:10000000F05B0120D1DD0000E1DD0000E3DD000058
:10001000E7DD0000E5DD0000E7DD0000E7DD0000D2
:10002000E7DD0000E7DD0000E7DD000041DF000064
:10003000E7DD0000E7DD0000F1DF000055E0000033
:10004000E7DD0000E7DD0000E7DD0000E7DD0000A0
:10005000E7DD0000E7DD0000E7DD0000E7DD000090
:10006000E7DD0000E7DD0000E7DD0000E7DD000080
:10007000E7DD0000E7DD0000E7DD0000E7DD000070
:10008000E7DD0000E7DD0000E7DD0000E7DD000060
:10009000E7DD0000E7DD0000E7DD0000E7DD000050
:1000A000E7DD0000E7DD0000E7DD0000E7DD000040
:1000B000E7DD0000E7DD0000E7DD0000E7DD000030
:1000C000E7DD0000E7DD0000E7DD0000E7DD000020
:0800D000E7DD0000E7DD0000A0
:1000E000F8B504461646F0070D461F4603D41D2EEC
:1000F00018BF1B2E09D16946204647F055FC17282A
:1001000011D0F00701D51E2E05D16946204647F0D3
:10011000BBFD172807D0069800903B46324629467B
:10012000204647F015FDF2BD2DE9F0410E46354958
:10013000054608781746984608B912205FE0002166
:10014000284647F0F1FC040008BF342057D03000A7
:1001500002D0012E08D01BE0606D417801F0120141
:10016000022926D0A06D04E0606D4178880720D573
:10017000E06D03214170A0F803703100C0F80580E4
:1001800002D13BF0FFF801E03BF0FEF8072801D177
:10019000182034E068B91C4F3868011D11F835206B
:1001A000500711D5206E01210170206E3BF0EEF852
:1001B00008B11E2023E03868011D001D11F835200C
:1001C00002F0FB0200F83520396801EBC500017927
:1001D000CA0704D5320008BF01F0FE0105D08A0726
:1001E00004D5012E02D101F0FD0101710749087803
:1001F00020B100220A70FF20054908700020BDE8E8
:10020000F08100BFA70F0020B00E0020A60F002035
:100210006402002038B505460F2D0C4616DA4FF65D
:10022000FF72914212D0022806D13C2014FB00F04C
:1002300080B247F0F9FD04E00E2804BFE0B201F0FF
:10024000D1F8034820F81540002032BD022032BD0D
:10025000CC010020F8B504460D4616461F460C207A
:1002600008F0D4FB010010D00698D0220A70488113
:10027000182306484C708B70CC708D80CE800F8117
:10028000BDE8F440007808F085BCF1BDB91100204C
:1002900010B5024601241078912804D0A2281CD061
:1002A000D02821D030E0517805290AD00E2904D079
:1002B0000F290AD03E290CD026E0104600F0D0F8D5
:1002C00010E0104647F0A8FC1FE0104600F012F9BD
:1002D00008E0104600F01CF804E050884FF6FF716B
:1002E00047F052FB044610E09078122802D0132801
:1002F00005D00AE05178506847F0A2FC05E051684B
:10030000D07847F01DFB00E00024204610BD00001F
:1003100038B5044686B0A07801250146012918D0D9
:1003200003292CD0062939D00A2912D00E291CBF46
:100330000F29102900F08980152918BF162979D0B6
:1003400017297DD0812975D0832918D0842974D0AC
:1003500080E0214647F048FB68462146162246F0D9
:1003600033FDBDF8040047F0B3FA040073D0002059
:1003700047F0BEFA0146608801F0D4F96BE0A0882E
:10038000224647F001FB0546E078002863D1238927
:100390006289E188A08847F073FB5CE0A0880122B5
:1003A000402147F059FB002047F026FCC0B202284C
:1003B00021D1102008F02AFBB8B1D0210170112101
:1003C000E27842708170A2888280E188C1802289AF
:1003D0000281618941810021A28981738281014664
:1003E0001E48007808F0D6FB35E0A08800224021A6
:1003F00047F032FB2FE0A188ADF80010012803D1AF
:100400000021ADF80A1011E080B9E088ADF80200D3
:1004100000212089ADF804006089ADF80600A089AC
:10042000ADF808008DF80A108DF80B50684647F0BB
:1004300077FA10E02246182104E022461C2101E050
:10044000224606213AF064FF02E020463AF097FF88
:10045000054600E00025284607B030BDB911002050
:1004600010B58388012442F20202991A1CD0891F18
:10047000012937D9891F1BD0193902291DD9891F94
:100480001BD01139022921D9C91F052921D90C39BD
:10049000062921D9C91F14D0491E1AD04DF61E4273
:1004A000891A01291ED921E0806847F091FC1BE0E0
:1004B00047F0F2FB47F04CFA19E081680878B0B1D8
:1004C00014E08268052142F2580008E03AF049FF42
:1004D0000AE03AF050FF07E08268032118463AF03C
:1004E00017FF01E03AF054FF044600E000242046E4
:1004F00010BD000070B58388012142F213041A1B5D
:1005000004D0921F12D02B3A1BD01EE0104D2E8823
:100510004FF6FF72964209D00E4B1A68002A1CBF94
:100520001268002A12D00146204608E00A4A1268E2
:10053000002A1CBF1268002A08D0014618469047BE
:1005400001E03AF01AFF014600E00021084670BDC4
:1005500058020020C40E0020C00E0020F8B50C4642
:100560001546002620B1012810D0042814D01DE023
:10057000162C19DA0F4F16220021384608F011FA0E
:1005800022462946384608F0DAF910E0022C0BD151
:100590002888094908800AE0082C05D1074829461F
:1005A000082246F011FC02E0182600E00226304640
:1005B000F2BD00BFDC210020F4210020E40F002068
:1005C00010B502460846002442B1012A0BD0042A85
:1005D0000DD0092A10D00A2A12D015E015220C4994
:1005E00008F0ADF911E00B4A118801800DE00A49CD
:1005F000082246F0E9FB08E008490A78027004E0A6
:10060000074B1978017000E00224204610BD00BF9E
:10061000DC210020F4210020E40F0020ED0F002059
:10062000F621002080B50021C00706D5044B0548FF
:1006300010220B2100F0FCF90146084602BD00BF64
:10064000287F0400F00F00202DE9F8430D46002715
:100650002878022814461E4663D168680178DDF8C0
:100660002080407801EB00205FEA080280B204D0CD
:10067000B0F5285F0ED00B2056E04FF42851401AF9
:1006800008D0401E24D0C01E2AD0A23843D0233820
:1006900041D046E0DDF82490E86808F04EF980B2D9
:1006A000A0EB08024A45BCBFA0EB08001FFA80F986
:1006B00009EB0800162809DAA6F800904A46E8680F
:1006C00000EB0801204608F03AF92CE00D272AE05B
:1006D000E8680088022131802070000A607022E002
:1006E000E868B0B1082131800288227003881B0AB3
:1006F00063704188A1704288120AE270818821717A
:100700008288120A6271C188A171C088000AE071F2
:1007100009E0308007E001213180E868027822702A
:1007200001E0378001273846BDE8F2832DE9F04724
:100730000F46814638780026022890461D4652D141
:100740007868089C01784078DFF8A4A001EB0022CB
:1007500092B24FF42853D21A06D0521E27D0A53A8F
:100760003FD0233A3DD03EE0F86808F0E6F880B28A
:10077000A0421AD3611916291CDAFB682A464146A1
:10078000181908F0DCF82D19F868ADB2C5F1160299
:100790000021401908F005F9DAF8000000281CBF14
:1007A0000268002A20D0002118E007261CE01CB9AE
:1007B000022D03D00D2617E00B2615E098F8000057
:1007C00098F8011000EB0122F8680280DAF80000C6
:1007D00000281CBF0268002A06D001214846904725
:1007E00002E0032600E001263046BDE8F08700BFA6
:1007F000D82100202DE9F843092986B0064617467E
:100800003FD196F8242039887888521C491E86F8F2
:1008100024204143786889B2425C08444178307BA7
:1008200002EB01240128A4B239D139887888002547
:1008300048431FFA80F93D80A846C8452FDA7888DA
:10084000D7F804C0B17C431FC4449BB20CF105022D
:1008500006F1130047F088F870B1A84506D0786813
:100860007A8800EB0801401908F069F8788839881F
:100870004519491CADB23980788840445FFA80F848
:10088000DBE738790A2818BF062802D196F8240039
:1008900090BB96F82400401C86F824007C884FF614
:1008A000FF70844218BF002C26D0308A844223DA9D
:1008B000307B641C0128F48112D1ADF80040022283
:1008C000318AADF802108DF80420032128228DF81A
:1008D00005108DF806206946308846F0CDFF04E00B
:1008E000308806F10E0146F0C7FF307A47F23051EA
:1008F00008F0ECFC162000E0002007B0BDE8F08313
:100900007CB504460D4647F037F906000AD101A828
:1009100021460090ADF804507F23034C207800223C
:1009200047F0F2F8304676BD720200202DE9F04122
:100930001F4C204F204D214E2070214801703A70ED
:100940002878C00008F0A8FD306070B338784FF602
:10095000FF7878B92878800008F09EFD1949086072
:1009600020B93068BDE8F04108F0A6BD0146404618
:1009700039F0AAFE3168002006E021F8308001EB52
:10098000C00300225A60401C2A789042F5DB052003
:1009900047F00EFA207847F04FF80B4847F09CF8E4
:1009A0002078BDE8F04147F083B9BDE8F08100BF91
:1009B000B40F0020A0100020C10F0020000F002065
:1009C000F721002018220020A512000038B50D469E
:1009D000290427D5144A107808F0F8F804001ED02E
:1009E0002078A2280BD0B02816D1204647F044F931
:1009F00090B1217904F1080047F0D6F80CE0607955
:100A0000652808BF47F0E0F808480078FF2803D0C1
:100A1000214608F0BFF810B1204608F009F885F427
:100A2000004032BD002032BDB40F0020760200200D
:100A30003EB504001D460FD0ADF800108DF8022021
:100A40000194684647F064F8010006D12DB1608931
:100A5000294646F041FF3EBD02203EBD3EB505465B
:100A60000C4646F0E1FF010008D16946284647F0F0
:100A700073F9010002D10CB1019921603EBD000063
:100A80002DE9FC47314C0F46994682469046ADF819
:100A900000900121257946F0B3FF18266D1C08B996
:100AA000142051E061888A4501BF207908282189F6
:100AB000894548D14B4642463946504646F058FF94
:100AC0002189491C21816A460146204600F080F8B0
:100AD000060038D016281E4F21D018281CBF607879
:100AE000142830D0E9B2384647F05EF82079BDF8D6
:100AF0000010387079803E713946608847F044F9BB
:100B000008B101251626217904F1080047F04CF8B8
:100B100020220021204607F044FF162E13D16088C2
:100B20003A46E9B246F09CFF18B1E9B2384647F0C0
:100B30003BF8217904F1080047F036F82022002123
:100B4000204607F02EFF3046BDE8F687F82100204A
:100B5000380C002080B50021C2070ED5084908785E
:100B600020B9084B08481022042103E0002310227A
:100B700001210648FFF75CFF0146084602BD00BFA1
:100B8000A01000203C7F0400A4100020E4100020EE
:100B900038B504460D4D47F0DBF8288029466088BB
:100BA00047F052F938B120892988884228BF084681
:100BB0002880162032BD21892888814228BF01461D
:100BC0006088FFF79DFE002032BD00BF380C00207A
:100BD0002DE9F44F054686B068888B4646F09CFFA9
:100BE0004549841E0878A4B288B144498D4204D096
:100BF00020222946414807F0A2FE414E0594414F6C
:100C0000DFF8F480DFF80091DFF800A117E005F1CC
:100C10000806F3E7BBF1000F49D16389BAF8002059
:100C2000D9F80010688846F0A3FE002883463ED11C
:100C300030884FF6FF71884239D0401C30800598CB
:100C40003989801E884232DBBBF1000F2FD104A806
:100C50000090337971883088721D46F059FE040087
:100C600025D0608930802146BDF81020688807F0C3
:100C700017F98346D8B928790599D9F80030039037
:100C80008A1E92B2002002920190CDF800A0BDF819
:100C900010206888214600F0A7F9834698F80000E4
:100CA0000028B7D0BBF1160FB4D1002021E039895C
:100CB0005846C1B17A8891FBF2F1398098F800006A
:100CC00050B10E4C217904F1080046F06DFF20224E
:100CD0000021204607F065FE6888394646F00CFE84
:100CE00038B1162005E032880100069908BF0A20B5
:100CF0000A8007B0BDE8F08FF7210020F82100201E
:100D000000220020380C0020080F0020840F002053
:100D10002DE9F84F074686B07888574DDFF85CB16B
:100D2000884646F0F9FE064604A800903B7B798988
:100D3000388907F10D0246F0EBFD00248246059646
:100D400049E06968FF208855A3B26868FF22C25451
:100D500034E0A0B2002877D1788800234FF6FF72E4
:100D6000112146F0F1FE0028686067D0BBF8000052
:100D7000001D6880641C6968BAF80A008855A2B230
:100D8000BAF80A006968000A8854BDF81020798909
:100D90000DF11203504646F017FE661C8246741C85
:100DA000BAF1000FB6B2CCD06968BDF81200885510
:100DB000A2B2BDF812006968000A8854641C304869
:100DC0006B680168BBF80020A6B2981907F0B7FD60
:100DD000BBF800000419BAF1000FA6B222D0BDF88A
:100DE00010207888514607F05BF88146A0B9387921
:100DF0000599234B1B6803908A1F92B20020029230
:100E00000190CDF800B0BDF810207888514600F070
:100E1000EBF8002881469CD0BAF80A10A8F8001018
:100E2000484600E00020A4B2CCB901003989A8F8F6
:100E3000001008BF0A2007B0BDE8F08FBAF80A001A
:100E4000A8F800001120F6E7BBF800006988021D31
:100E5000914204D10599891F801981428ADA6888F4
:100E600096FBF0F028802946788846F0B9FE0028E5
:100E700018BF1620DFE700BF380C0020840F0020C9
:100E8000080F00203EB54D681821144601916A886C
:100E90000092AB88AA682988408800F0A7F9162834
:100EA00002D10021A9603EBD01001CBF298821801C
:100EB0003EBD00002DE9FC4105460E46904600204F
:100EC00000270DE0019060880090A388A2686888E0
:100ED00000F08CF9162817D10021A1607F1CFFB209
:100EE0000D490A78974214DA71680C2313FB07F353
:100EF0000B441C46218861B1781C90421BBF988925
:100F0000002818201620DDE70028E7D02188A8F85F
:100F10000010BDE8F68100BFB50F002070B5054692
:100F20000C4646F0A1FE010006D14FF6FF7046F0D8
:100F30009BFE010017D00D80002200E0521C0B4BDD
:100F40001D78D0B2A8420ED24B68D6B20C256E43A3
:100F5000334418880028F1D10C222146184607F0A6
:100F6000EEFC002070BD092070BD00BFB50F002051
:100F7000F8B5054600260F4C0BE0B86808B108F03C
:100F8000EBF80C220021384607F00BFD00203880DA
:100F9000761C2178F0B2884207D26A68F3B20C213D
:100FA0004B43D71838880028E7D14FF6FF712980C6
:100FB000F1BD00BFB50F00207CB50C78022C11D11B
:100FC0004C682578647805EB042642F60215B6B223
:100FD000AE4207D1BDF8185000950224019439F0B3
:100FE000B9FB76BD012076BD2DE9FE4F0D46824648
:100FF000287AC10693461E464FF000090CD5584684
:1010000046F0F6FC030000F0EA800A22294650462A
:1010100098475FEA00094DD128780C9F0D9CDDF8B8
:10102000388002281AD168680178407801EB0022E4
:1010300092B24FF42053D21A012A10D9921E3AD0FC
:10104000521E14D0FD3A7BD0521E00F08280521EF8
:101050006ED0521E74D0521E00F09680ACE0002C70
:101060002AD1E868017839800278416888E0002C4C
:1010700022D101203880E9680A783270002168891D
:10108000401C80B246F004FD398860B10278921CA1
:1010900051183980418971704289120AB2704168D1
:1010A0000278F01C6DE0091D398004220021701CBB
:1010B00007F077FC95E0002C67D1E86804880421EC
:1010C00039803470220A72700DF10201204646F018
:1010D000DFFC5FEA000821D0D8F80C40BDF8022000
:1010E0004FF6FF756B46294646F06EFC50B998F8EE
:1010F0000030D8F804203C48022146F035FC08B9FD
:10110000ADF80050207802280AD161680222301D13
:1011100007F015FC3888801C388001E0ADF80040ED
:10112000BDF80000B070BDF80010090AF17058E079
:10113000002C2AD1E8680168504639F0F4FA02E040
:101140001CBBE8680088022139803070000A70708A
:1011500047E0E86807F0F1FB82B2A242B8BF4FF067
:1011600007093EDB944208BF002205D008EB0401CA
:101170009142B4BF4246121B3A8092B2E86801190C
:10118000304607F0DCFB2CE014B14FF00B0928E0EF
:10119000E86807213980027832704378737041889B
:1011A000B1704288120AF27001793171C28872718D
:1011B000C088000AB07114E0584646F059FC5FEA56
:1011C00000090CD09DF83C000290CDF804800094FA
:1011D0003B46324629465046C847814601E04FF01B
:1011E0000E094846BDE8FE8F0EFF04002DE9FE43C0
:1011F0008146884617461E4602A9404646F048FCEE
:1012000004002CD0BDF8080046F09AFD844620B3B7
:10121000BDF828100B9D0091334601953A462146B2
:101220004846E0470646D8B9FE2D19D02078022856
:1012300016D160680178407801EB002242F6021175
:1012400092B28A420CD13878797800EB012292B2BE
:101250004146484600F072F802E00E2600E0012602
:101260003046BDE8FE8300007CB505464FF6FF76AC
:1012700001AC009402230A4A3146012046F048FBA3
:101280000BE0E0680168284639F01EFABDF804203A
:1012900000233146204646F097FB0400F1D173BD90
:1012A000FEFE040038B50129044606D002293CD1CF
:1012B000012146F0A5FB002837D1204646F0D4FC9A
:1012C00008B1FFF755FE2046FFF7CEFF1749087813
:1012D00098B1174D6888A0420FD129791548491C4B
:1012E000C9B246F061FC297905F1080046F05CFCC2
:1012F00020220021284607F054FB0F4D284608F015
:10130000AFF810E0208958B12146284608F0B7F818
:10131000A17A04F10C0046F047FC204608F0CCF816
:10132000204608F09FF80400ECD131BDF7210020E1
:10133000F8210020380C0020180E0020F8B50D4CC4
:101340000E462178FF290546174611D00A2007F0DE
:101350005DFB68B1B12101700022427002714580CD
:10136000C680078101462078BDE8F44007F012BC32
:10137000F1BD00BF7302002038B51C460A4B1D7832
:10138000012D01D13A2032BD130018BF002C02D02C
:1013900010F47F4F01D0122032BD0B46214601B020
:1013A000BDE8304000F018BFB60F00200B4980B5F3
:1013B00009888DF8011000208DF80000090A8DF8C9
:1013C00002106A46064801788DF8031042F20200C6
:1013D000042146F0F5FC002002BD00BF38230020A8
:1013E000C60F002080B501F0BFF98DF800006A46F5
:1013F00001214FF6744046F0E3FC002002BD70B5B9
:101400004A1ED2B2002305E0D51AC45C465DC6541C
:1014100044555B1CB3EB510FF6DB70BD2DE9F8436F
:10142000054624480E46017801291746984608D1FA
:1014300021480188491E018089B211B9012046F076
:10144000E7FCDFF8789099F80000FF2478B10C20D1
:1014500007F0DCFA48B39021017002224470458005
:101460000271C7808660014699F8000019E00820E3
:1014700007F0CCFAC8B1012101704470711F4160BE
:1014800002220A7041684D702D0A416845EA08152C
:101490008D704268D7703F0A41680F710146084855
:1014A0000078BDE8F44307F075BB3046BDE8F24371
:1014B00007F052BEB70F0020860F00201F22002029
:1014C0001C220020F1B5234F0D4639781646A9B1EC
:1014D0000C2007F09BFA04003AD0912020703E21A6
:1014E00082226170A2700522BDF80000A080A67162
:1014F0002946E01D07F023FA387826E0142007F08B
:1015000085FA040024D001202070FF2104F1080294
:1015100061706260042010703E2260684270092190
:101520006068817082216068C170022260686946CB
:10153000001D07F004FA606886710522606829467C
:10154000C01D07F0FCF904480078214607F022FB93
:10155000F1BD00BF1E2200201C2200202DE9F04119
:1015600004462D480D46C179880616461F4650D5BB
:101570002A49487801074CD5200004D057EA0600D4
:1015800004BF01260127DFF8988098F80010C1B148
:10159000082007F03BFA00283BD0912101703E2241
:1015A0000C23042E08BF0326042F08BF0327427014
:1015B0008370C47085808671C771014698F80000F9
:1015C00023E0112007F022FA18B301210170FF2255
:1015D000427000F10801416004220A703E234B7002
:1015E00006228A704D710C22CA702D0A0C718D7101
:1015F000CA1D511C042E08BF0326042F167008BFF5
:1016000003270F70014607480078BDE8F04107F056
:10161000C1BABDE8F08100BF280E0020200E0020D6
:101620001E2200201C2200202DE9F0410446114812
:101630000D4601781646CA07984619D50E4F3978D7
:10164000B1B10C2007F0E2F990B106999122027035
:101650003E234370832282704181C4708580C6809E
:10166000A0F8088001463878BDE8F04107F092BA4A
:10167000BDE8F081212200201E22002080B50B4908
:101680000B4A087000200B49107008700A4A0B4979
:101690001070087046F090F909490A4B7F20887055
:1016A0000022094802701A7001BD00BF1C220020F0
:1016B0001D2200201E2200201F22002020220020A8
:1016C000200E002021220020B60F002038B50D4644
:1016D000290411D5094A107807F078FA040009D0D6
:1016E0002078032812BF0128E06807F035FD204666
:1016F00007F09EF985F40045284632BD1C220020E3
:1017000001490870704700BF1E220020014908707F
:10171000704700BF1F22002001490870704700BFBA
:1017200020220020F8B50C4F054638680E460624E6
:1017300040B90A49087810FB04F080B207F0ACFE0B
:10174000386040B13868654331462844BDE8F84008
:10175000062207F0F4B8F1BD24220020C10F0020BA
:101760000449096809B9002070470622504308441B
:10177000704700BF2422002078B587B00F9C250059
:1017800013D0BDF8485006950394BDF840509DF81D
:10179000384004950294BDF844600D9D0C9C05965C
:1017A0000195009446F070F900E0312008B070BD5A
:1017B000F8B5002500260C4C11E00C4801683422D5
:1017C00012FB06F288180379DF0706D506220021EE
:1017D000801D07F08CFC00B96D1C761CF6B22078D9
:1017E0008642EADBE8B2F2BDC10F0020180F0020EC
:1017F0002DE9F043A24CA349A34E20700A220020F9
:1018000008600D23A1484FF4097102704380818064
:1018100085B09F4A9F48106037789F480770FF2F18
:101820007178417008BFFF29B2788270F378C37075
:10183000357905717679467114D1FF2A08BFFF2BDF
:1018400010D1FF2D08BFFF2E0CD194490A780270E9
:101850004B7843708A788270CB78C3700A790271B2
:10186000497941718E4902788E4D8F4E8F4F0A70A3
:1018700043784B7082788A70C378CB7002790A7192
:1018800040798B4A4871FF2028706870A870E87012
:1018900028716871002087490880F06B864940787C
:1018A00008708649F06B0078087013888448854971
:1018B0000380F06BC06C08608349F06B90F83C00CB
:1018C00008708249F06B90F83D0008708049F06B19
:1018D00090F860000870F06B406901797D484A1EFD
:1018E0000270F06B7C49C0783870F06B80690860DA
:1018F00008B906F0E7FFF06B7849C069086008B9DD
:1019000006F0E0FFF06B416D75480C2207F017F808
:1019100045F0DAFFF06B7349006A086008B906F019
:10192000D1FFF06BDFF8C081406AC8F8000008B949
:1019300006F0C8FFF06B6D49806A086008B906F0D0
:10194000C1FFF06B6A49C06D002840D001220A75C2
:10195000F06BC06D02681378C3F3400048B1F06BC0
:10196000C06D02681378C3F3C00000280CBF0120CB
:101970000220487500208860C8600861F06BC06D67
:10198000426890780870F06BC06D4268D0784870FB
:10199000F06BC06D426813788B70F06BC06D42685D
:1019A0005078C870F06BC06D426810790871F06BA8
:1019B000C06D426850794871F06BC06D4268907993
:1019C0008871F06BC06D4268D079C87101E0002267
:1019D0000A7503F0C5FA07280AD103F0E5FB207861
:1019E0004FF4804107F07AF9002006F06BFF43E0E6
:1019F00040480168884781463AF0CAFBD8F80000A1
:101A000001688847684641F0B3FAD8F800200420FE
:101A10008DF80000694652F8043F00209847364987
:101A2000086003F079FDF068344A01883878344B57
:101A3000014311804846196888470C21314803F05A
:101A4000F4FC284646F0F4F845F0CAFF2E48002181
:101A50004FF6FF7201608280F06B90F858102B48AF
:101A6000006803F063FA0121FF2039F05CFC207864
:101A70004FF4005107F032F905B0BDE8F08300BF24
:101A8000C70F0020380F0020D04F0050700E0020EC
:101A90003C0F0020B63F0050400E0020E8120050DE
:101AA000500E0020480E0020B07F0400C40F00201C
:101AB000601100209E0F0020C60F0020D40F0020D0
:101AC0003823002058230020D4230020D5230020D1
:101AD00051230020CB0F0020200F0020240F0020D6
:101AE0003C230020280F00202C0F0020300F002066
:101AF000BC230020501B00204C230020A00F0020FE
:101B0000541B0020FC0D0020800E0020E02300204C
:101B1000704770472DE9F04F0F46380589B018D54A
:101B2000DFF8E4532888FF280ED0C0B203F006FA8D
:101B3000040009D0A079162145F02AFF204603F0C1
:101B40007BF8204646F06CF8FF20288087F4006080
:101B5000D6E1F80504D539F00BFC87F48070CFE1AD
:101B6000B80604D539F0CAFB87F02000C8E1F807B1
:101B70000CD505F023FB30B100218160DFF88C0328
:101B8000006800B1804787F00100B9E1380704D54B
:101B900039F0B6FB87F00800B2E1F8060FD5002156
:101BA0000022002306910592049103930291019271
:101BB0000091022046F028F987F01000A0E1B80754
:101BC0000FD5002100230691059104910393029102
:101BD0000191009101223C2046F016F987F00200A5
:101BE0008EE179074FF01E08C94EDFF828A340F1B7
:101BF000CD80C9480022002108920791007845F065
:101C000093FF0446C5488178FF2904BF002006F0F1
:101C100059FEA07A03F092F905469AF8000095F86B
:101C20002E91002805F5947B69D0606D807A02289A
:101C300018BF032807D130680D3045F0E5FF10B913
:101C40003068C11D07915946484646F055F8A0B383
:101C5000606D807C3368002818BF012804D11946C4
:101C6000584645F019FF04E05A464946184645F0E3
:101C70001FFFFF2843D018FB00F8306840440622BD
:101C80005946C01D06F05BFE306810F8081040444D
:101C900000F1010BC01D41F0020908900622616DA0
:101CA000C87A00F0010085F82E01606D00F10C018A
:101CB00005F5947006F043FE21E05946484645F08C
:101CC00053FFE0B130685A46494645F0F1FEFF281F
:101CD00015D018FB00F8306840440D3045F094FFF3
:101CE00058B9306840440D3045F08EFF002801BFE0
:101CF00030684044417F012901D149F0020905F1D2
:101D00002C004B4601780691428912090592012266
:101D1000698C0491C0880899029140080390CDF81D
:101D200000B0079801900020A97946F06DF8D5F829
:101D30009C017B498842A8790CBF0021012145F014
:101D400097FF7848AB7902682C214B43134401225A
:101D50001A73AB7904684B4323445A73AB79046814
:101D60004B4323449A73AB7904684B432344DA739F
:101D7000AB79006811FB03F10144002008740720CF
:101D8000A97939F0CDFA87F00400B9E038060FD50B
:101D90000021002306910591049103930291019182
:101DA000009101223B2046F02FF887F08000A7E049
:101DB000F8045DD55C4930680C680D3045F024FFAF
:101DC000002844D13068C11D0D3045F0F9FD3EE0DA
:101DD000606D4178480704F13E0526D52878022831
:101DE0001EBF03286878012830D16978306804F173
:101DF000380245F05DFE8146B9F1FF0F15D030681D
:101E000018FB09F948440D3045F0FEFE68B930680A
:101E10004844C11D0D3045F0D3FD30684844C11D14
:101E2000062204F1380006F08AFD2878022818BF3F
:101E300003280BD130680D3045F0E6FE30B930682C
:101E4000C11D062204F1300006F079FD2468002C43
:101E5000BED13648DAF8042000784FF4805107F0FC
:101E6000CBFB10B18E2045F03BFE87F4805047E05D
:101E7000B80505D544F012FD2D4901200860FEE7A4
:101E8000780504D506F058FD87F4806038E07804C2
:101E900005D5812045F024FE87F4804030E0B90468
:101EA0002DD5244C206810B1002006F00BFD4FF01A
:101EB000FF3020600020204C02F082FA216851F8A7
:101EC000202F684690471D494A6B086BC96A2468F1
:101ED0001B4B019200900293ADF810106B46194A0B
:101EE00019491A4803921A4A07922568194AA847BD
:101EF0001949086000F032F887F4005000E0002033
:101F000009B0BDE8F08F00BFF6100020480F002098
:101F1000680F0020880E0020D70F0020780E0020C8
:101F20004DE50110742300204C0F0020C70F002046
:101F30007C052043380F0020200F0020FC100020DB
:101F400025570000355700002822002038220020A5
:101F50001EFB0080EC0A00201C0F0020F8B5564C38
:101F6000564B2568186855F8183F00224FF0FF318E
:101F7000984705F0A9FB5249524AC86B406941791C
:101F800051481170002301680B8000244B800C71B4
:101F900000684371002002F013FA02F04DFA4B483A
:101FA000006845F081FE45F0F7FD4948006800B142
:101FB00004734848006800B1C4720026464C474D7F
:101FC00012E06068F1B24FF4D07251434218537975
:101FD000012B08D1F0B202F0B1FF074602F02CFE4F
:101FE000384645F01DFE761C2978F0B28842E8D3C9
:101FF00045F0C2FE3A483B4A0178117004F014FCE7
:1020000039F09DF93848394A8078C1074CBF07211B
:102010000521FF2400074CBFFF20FB20014034486E
:1020200001700021334811700023334A03700121ED
:10203000324811700370324A324811700370324ACC
:102040003248334913700370324A334813801B23DC
:1020500003804FF4A470314A314B088010804FF454
:102060002960304A1880FB212F4B1180198044F2DF
:1020700090202E492E4A0880108045F035FD45F00D
:10208000B3FD39F06DF939F07CF939F046F9294999
:10209000294A002008701F21284804704470847069
:1020A000C47001712648047044708470C47001715A
:1020B000252010700020F2BD200F00201C0F0020F2
:1020C000B07F0400CA0F0020400F00206C0F0020DA
:1020D000500F0020540F0020780E0020D40F002055
:1020E000C60F0020D30F0020C00C0020CC0F002012
:1020F000C50F0020CD0F0020CE0F0020CF0F0020F5
:10210000D00F0020D10F0020D20F00205C23002030
:102110008C0F00209C0F00208A0F00208E0F0020C3
:10212000900F0020920F0020960F0020940F0020A7
:10213000980F0020C80F002070230020602300208B
:102140006823002010B5040004BF002006F0BAFB8D
:102150001C490878052815D11B480168887A012890
:1021600018BF03282BD0194821780170627842707B
:10217000A1788170E278C27021790171627942712F
:10218000002010BD062807D111480168887A01286F
:1021900015D00328E7D112E01128E4D10D480068DA
:1021A0000028E0D0017A0129F9D1416D4A78D106A1
:1021B000F5D590F83E10012918BF0329EFD10C2066
:1021C00010BD00BFC80F0020500F0020480E002097
:1021D000540F00204C0F00202DE9FC410C00054657
:1021E0001646984605D05FEA080018BFB8F1010FFF
:1021F00001D0122045E024480188914204D28A206F
:1022000045F06EFC30203CE0284645F0BDFC010066
:1022100037D1E8B202F092FE1C4F0546387820B95B
:10222000012045F005FC07202BE01948016888478C
:102230003A781849531E3B70D1F800C0E047B5F812
:102240008E01B0420AD232462146284645F010FBA4
:10225000010016D1204606F07FFF07E01020009015
:102260004346F2B22146284645F0E2FD04F0A6FFBF
:10227000296800780A78824204BF284645F028FD84
:102280000020BDE8F68100BF38230020D30F0020D6
:10229000501B0020541B002038B5264C20780928FC
:1022A00018BF0A2801D0212032BD40F2014045F07C
:1022B00033FB207809280DD11F4A20481368018874
:1022C0001F489980007845F053FD0021002045F01B
:1022D000D3FB2BE00A2829D117481A4D02682B8816
:1022E0006988A888CB18C31893806988D180A97998
:1022F000802918BF81290FBF7F21134B93F900005C
:10230000091A11721149087838B1002288680A70D8
:1023100008B107F0D1F839F000F82888012145F01C
:10232000ABFB002002F04CF802F086F80020207091
:1023300032BD00BFC80F0020440F0020AC0E0020AB
:10234000CA0F0020E40D0020C90F00209C230020AC
:102350002DE9F84304460027002C894644D02C4D33
:102360002878884240D3227912F0E00F3CD12046F1
:1023700045F0EAFA012837D12978DFF898808945B5
:102380004FF4D07607D04F46D8F80420FBB2734301
:102390001A44507940B3D8F80400F9B271430844A4
:1023A0004279012A31D1F8B202F0C8FD00F1770379
:1023B0002A78197911B11978012902D0597E012999
:1023C00003D1914507D03A200CE001680B78802BAF
:1023D0000CD0914508D12878F9B2814201D28145CB
:1023E000D9D00020BDE8F2831220FBE70021625C17
:1023F0004318491C052983F86120F8DB818EC91D2B
:10240000A0F89210012145F0FBFC7F1CE3E700BF20
:10241000D40F0020780E0020A0F11B0210B5E12A95
:102420003EBFA1F5A47244F249139A4207D20D4A65
:102430001488844222BF0C4B1A888A4201D212208F
:1024400010BD0A4A53789A0601D4112010BD084ADB
:10245000084B094C10800948018019802180002018
:1024600010BD00BF920F0020940F0020C00C002070
:102470008A0F00208E0F0020900F00208C0F00206C
:1024800070B50446012045F0E3FB002500B10125AD
:102490001B4801680A7B012A0CBF0120002005436C
:1024A00018480168CA7A012A0CBF012000200543A0
:1024B00001D00C2070BD144D144E28787CB1012C35
:1024C0001BD1317849B972684FF4805107F094F804
:1024D00008B1032070BD01203070002070BD31783C
:1024E0000029FAD04FF4805107F0C6F828784FF44D
:1024F000805106F059FC0020EEE7122070BD00BFAD
:10250000500F0020540F0020C70F0020880E00201D
:1025100010B5010003D04AF2B911884201DB302026
:1025200010BD0A4A4FF47A71484350601078012870
:102530000AD1074C20784FF4805107F09DF820789D
:102540004FF4805106F0CAFB002010BD880E002019
:10255000C70F002018B591B04121684644F031FC06
:10256000684602F0B1FE044620210DF1010045F05D
:1025700023FC20210DF1210045F01EFC002C0CBF96
:1025800000201F200DF121020DF1010145F020FA7C
:10259000002012B010BD10B5A2B0014640220DF1CE
:1025A000010044F011FC04218DF800100DF1010030
:1025B000202145F001FC20210DF1210045F0FCFB1C
:1025C00011A9684602F0CEFE00280CBF00241F248B
:1025D00020210DF1450045F0EFFB0DF145012046AE
:1025E00045F0BEFB002022B010BD70B50D001446B2
:1025F00018BF002C064601D1122070BD00202870A3
:102600002070304645F0C0FA01000FD1F0B202F060
:1026100095FC90F89611042908BF0321297090F8C1
:102620009601042808BF03202070002070BD000020
:1026300083B24FF2FF52A3F20153934222BF8BB2F7
:10264000A3F20153934201D212207047094A136842
:10265000188059800A21B3F9000090FBF1F119713B
:102660001068B0F902100A2291FBF2F242710020C8
:10267000704700BF400F002008B9122070470D4A74
:10268000517809B10C2070470B4902784A704278A2
:102690008A708378CB70C0780871D1074CBF07204F
:1026A000052011074CBFFF21FB210840034908709A
:1026B00000207047780E0020C00C0020C50F0020BD
:1026C0002DE9F041064604F079FD0446304645F018
:1026D0005BFA010035D1F0B202F030FC050014BF06
:1026E000002C02202DD01848184F016888478046DA
:1026F0002078802811BF402815498A78964214D145
:1027000040F2014045F008F905F2171001211622A8
:102710000170427021780F48402902D10E4A0260B0
:1027200001E00E490160012103E00D4806804FF4ED
:102730000061387806F0D2FA0A490A6840469047A4
:102740000020BDE8F08100BF501B0020C70F002013
:10275000780E0020480F00203BB3030039B303007C
:10276000F6100020541B002010F0070001D11E209D
:102770007047024908700020704700BFF810002021
:1027800070B5094C094D2368286853F8186F00226A
:102790004FF0FF31B0472168286851F8042F904767
:1027A0000020286070BD00BF200F00201C0F0020FB
:1027B00038B5114C88B0002001F002FE216851F8B4
:1027C000202F684690470D494A6B086BC96A2468F8
:1027D0000B4B019200900293ADF810106B46094A22
:1027E00009490A4803920A4A07922568094AA847F4
:1027F0000949086009B030BD200F0020FC100020FE
:1028000025570000355700002822002038220020DC
:102810001EFB0080EC0A00201C0F0020F8B52948A0
:10282000294D0468296801F10D0045F0EDF90028F3
:1028300044D12868C11D0D3045F0C2F83EE0606DFE
:102840004178480704F13E0626D5307802281EBF9D
:1028500003287078012830D17178286804F1380293
:1028600045F026F90746FF2F16D01E20296847435A
:10287000394401F10D0045F0C7F968B928683844BA
:10288000C11D0D3045F09CF828683844C11D062252
:1028900004F1380006F053F83078022818BF0328F6
:1028A0000BD128680D3045F0AFF930B92868C11D4B
:1028B000062204F1300006F042F82468002CBED154
:1028C000F1BD00BF4C0F0020680F0020F8B5044692
:1028D00022480D4601780226052908D0062912D083
:1028E000112914D012291BD0132905D01DE01C4A30
:1028F000106890F8246018E0032038F03AFDA0B189
:1029000090F8B16011E0174801680E7E0DE016489E
:102910000078002145F008F938B190F8B86004E07B
:1029200038F01CFD08B190F8C660104F3868214699
:1029300003F06AFF08B9AE420ED20D48016888471D
:10294000012204463A7140F2014044F0E5FF094992
:102950000A68204690470120F2BD00BFC80F002042
:10296000500F0020540F0020D50F0020A823002076
:10297000501B0020541B00200249086000200871F1
:10298000704700BFA823002001480079704700BFAE
:10299000A823002030B501460B4BC8681C680A68A4
:1029A000A04208BF196003680B6085888B888C681B
:1029B0008D80838083688B6084600260C268CA6097
:1029C0000021C16030BD00BFB0230020F8B505462E
:1029D0002868416D4A78D10648BF40F6AC5465D4AA
:1029E000066D448B4CB9307CC0F3800100238722F4
:1029F00000F0030045F024F80446286800F1440183
:102A000004F2DC540A6953789A0728D4808C60B9A0
:102A10004A8802B9362296F84000C0F380010023AC
:102A200000F0030045F00CF83DE04A78012A14DD7F
:102A30000A7896F84000C0F38001002300F00300FC
:102A400044F0FEFF296822468C8C91F8451004F56D
:102A50009B74491E01FB042425E0241826E0243041
:102A60000023C27F96F84000C0F3800100F003000D
:102A700044F0E6FF0746286844304178012914DD18
:102A8000027896F84000C0F38001002300F00300B4
:102A900044F0D6FF2A6892F84530214607F59B742A
:102AA0005B1E03FB0414041900E03C19AC80F1BD6B
:102AB00030B5014609480A4C00682578002201E03B
:102AC000C068521CD3B2AB4205D20028F9D00368CB
:102AD0008B42F5D130BD002030BD00BFB0230020B7
:102AE000B42300202DE9F04706468946FFF7E0FFB2
:102AF00020B10020C9F80000012051E0102006F0AC
:102B0000CBFC040047D0274F26603968264E0029A9
:102B100004BF3078002808D13C60E46044F0C4FE73
:102B200000F5385000F1E0082EE0307801284FF42D
:102B30007A650ED10968086900F5FA5A02F070FC4E
:102B400000F00F083868E06015FB08A83968CC6011
:102B50001AE00868006900F5FA5802F061FC00F01C
:102B60000F0015FB00883D6800E00546E868026834
:102B70001069414603F048FE18B9E8683968884290
:102B8000F3D1E868E060EC603078401C3070C9F840
:102B90000040404604E000210E2045F0B1F800203E
:102BA000BDE8F087B0230020B423002070B50546AF
:102BB0000024287E85F87200012634E0686D427A90
:102BC00095F872002B7EA0F12501A3F1250006FAED
:102BD00001F106FA00F0014322EA01011C2212FB76
:102BE00004F201F00701A81841F02401242980F81B
:102BF000721016D1272180F8721012E0002C08BF45
:102C00000328DBD144F050FE297E00F0010041187A
:102C1000491C85F87210C8B22828A4BFC91E85F8BF
:102C20007210641CE4B2E87D411E8C42E6DB70BD8C
:102C300010B504460021207844F076FF08B9422000
:102C400010BD406DB4F8031043780022D80607D5B4
:102C500020290FDBA4F80320C4F80520122010BDA2
:102C6000074803888B4205D2A4F80320C4F8052046
:102C7000072010BD2046BDE81040002144F034BEBE
:102C80006002002010B504460021207844F04CFF7B
:102C900008B9422010BD406DB4F8031043780022FB
:102CA000D80607D520290FDBA4F80320C4F8052097
:102CB000122010BD074803888B4205D2A4F80320D8
:102CC000C4F80520072010BD2046BDE810400121B2
:102CD00044F00ABE600200202DE9F84F05004ED0F6
:102CE000DFF8E48298F80000092818BF0A2804D009
:102CF0000B281CBF0C280D2801D1212062E1A878E7
:102D0000002144F011FF040008BF4220F6D0AF4F6D
:102D1000A978DFF8BCA2397098F8000010B9A8783B
:102D20008AF8000004F14806F068417801F01201C9
:102D3000022902BF706900280C2012D0607AF0B11D
:102D4000A07B012804D1B5F8030008B1812816DA68
:102D50006878402813DA204644F092FDB06808B93C
:102D600007202FE1B561287801281FD1A07B00281A
:102D70001CBF0128042819D19648007808B91220F0
:102D800020E195494A78824208BF0920F8D0F068CE
:102D9000417848070AD504F1220180204A7F04F1D6
:102DA000380101F0B9FE08B10B200BE1687808B9D1
:102DB000112007E12878DFF82492DFF824B20128F7
:102DC00040F0AF8000212173F166217A012903D1FF
:102DD000B16968794871F4E0012000212072E17244
:102DE0006173254604F03CF96060DBF80000804721
:102DF0007C4A0146106802E06A6842600068002868
:102E0000FAD10846D9F800108847696876484861C1
:102E10000021387838F087FA39780122112038F00B
:102E20007FFAF0684178C80605D5284600F0E2FC34
:102E3000010024D0C6E0688C38F0B4FA85F821008F
:102E4000F068007838F07FFA04001CBF94F8B000F6
:102E5000002807D0E87F40F02000E877687D40F048
:102E600018006875284638F09BFA0100E2D134B1A9
:102E700094F8B000012804BF284638F06AFAF068D8
:102E80004178C8071CD505F14204A18800291CBF60
:102E90003068002814D022788A4211D20F2044F0E2
:102EA000ABFF68B1F06801788DF800100F20A288A0
:102EB000ADF8012021788DF80310694644F020FF19
:102EC00098F80000A0B94949087800281EBFF068AA
:102ED000417811F0030F03D04548006844F0E4FD49
:102EE000112088F800000121297238F00DFA68E0FD
:102EF0002846FFF7DDFD00281CBFB168002960D01F
:102F0000AA7B012A04D02A69808802EB800202E0B1
:102F1000486E2A69821895F8B8101046FFF7D6FC5B
:102F20004FE0207A00284CD0DBF800108847054697
:102F30003878012138F0F7F900202E4920720A680C
:102F40003E7811460B68187A002802BF586D037846
:102F5000B3421FD0C9689142F4D138789AF8001072
:102F6000884224D104F02AF9616888421FD104F014
:102F7000ABFB40F2014044F0CFFC1F491F4A204800
:102F800008600121107805F0A9FED9F80010284644
:102F9000884716E01B4E30780128DEDD0846FFF733
:102FA000F9FC06F089FA3078411E3170D5E72046E9
:102FB00044F0BAFCD9F8001028468847204601F0B2
:102FC000E1F90020BDE8F28FC80F0020D60F0020E5
:102FD000D50F0020D40F0020780E0020541B0020B5
:102FE000501B00204C0F002085720000880E00202E
:102FF0006C0F0020B0230020480F0020C70F0020D6
:103000006D400000B423002038B51048006800214E
:1030100001E0017200680028FBD10D480D4D0168E8
:103020008847044605E0C16829600022C26006F0B6
:1030300043FA28680028F6D1074A084B2860002187
:10304000117020461C68A04731BD00BF4C0F002006
:10305000501B0020B0230020B4230020541B00206C
:1030600070B51748174C007802280ED12068C46844
:1030700001688288A58883688580A668866025683F
:1030800005602160A280A36070BD032816DB206864
:10309000FFF780FC2668054600E00646F0680168F8
:1030A00028680969006903F0AFFB00281EBFF068BB
:1030B00021688842F1D1F068F560E86070BD00BF1A
:1030C000B4230020B02300202DE9F04144F0ECFBB4
:1030D000364D8046286800281DBF354E30780028C0
:1030E000002061D029680A68107A002841D132781E
:1030F000022A3EDB0846FFF74DFC06F0DDF930788A
:10310000411E317035E002F08BF9296809684B6D7A
:10311000D3F8037027F07F4740F6C4135F434FF0A6
:103120000B0C90FBFCFC0B2303FB1C0080B24FF448
:103130007A640A69604317FA80F082180A610AE02B
:103140000868827B012ADED144F0AEFB29680A6858
:1031500000F57A601061307802280ADB2868C168BF
:1031600000680A680069116903F04EFB08B1FFF7B7
:1031700077FF286801680969404603F045FB00288D
:103180002968DDD10A68107A0028ABD0506D094B50
:1031900002781A700868016D0069886029680868FB
:1031A0004168026D4A60006DBDE8F081B0230020E7
:1031B000B4230020D50F002010B5184C206844F02F
:1031C0000BFD48B30179032926D1007A10F00F0FC7
:1031D0001CBF00F00F01012908D000F00F02022AE5
:1031E0001EBF042900F00F00062815D10C48016805
:1031F0000A6A507880B1C8694078002818BF022850
:103200000AD10848006801784078814204D12068DA
:1032100044F03EFD012010BD002010BD8C0A0020AE
:10322000500F0020700F00202DE9F047804608F174
:10323000480517460E46AA68B00702F1A40408F133
:103240002A0918D5E968487810F0030F04BFB9F8C7
:103250001C1000290FD1286868B992F88A0000F084
:10326000FD0082F88A000622EB6803F10C0120467B
:1032700005F065FBA41D300708D5B9F8161004F851
:10328000011BB9F81600000A04F8010BF00608F15A
:10329000210A18D5B9F800109AF800303329E968E6
:1032A0008A7DB4BF40200020511E03F03F03184325
:1032B000C9B2C7F30C07207047EA413767703F0473
:1032C0003F0EA770E41CB00604D52146404638F0F6
:1032D00044F8123470060ED50849094BC86B416991
:1032E00008689AF8082002EB420281561A6892F99F
:1032F000040041182170BDE8F08700BFB07F0400D2
:10330000400F00202DE9FE4F0446002000900025CC
:103310000CB905F0D7FA04F1500841F62300D8F8AB
:10332000007038807D8002223A737A7369462046A5
:10333000FFF7D8FB08B9072051E2009901B1B86046
:10334000B8682061DFF89C04017884F8B810D8F8D8
:103350000400407A00F0D0FB25302076207EB87340
:10336000FD73D8F80400017D022904BF002005F098
:10337000A9FAD8F80400007D012802D1002000211C
:1033800004E083280CBF06200220202138747974C1
:1033900004F12406DFF850A4DAF83C00416908681B
:1033A000717901EB41010844B0F801207A82D8F824
:1033B0000400417848060AD5607DC10604D5E07F47
:1033C00040F04000E07702E040F04000607507F117
:1033D0005C0904F1300089F80050B17E890001F0E9
:1033E000040189F80010B866607DC10656D5D8F88A
:1033F000042051788A060CD500F0FE006075D8F8DC
:103400000400417811F0030F03D1E07F00F0FE00CB
:10341000E077607D44F044FAA075421C387CC0F32C
:103420008001002392B200F0030044F009FBA08366
:103430001E20A28B02F59B7393FBF0F01E2101FB73
:103440001030C0B208B1C0F11E00821802F59B72A4
:1034500062831E20A28B02F5967293B293FBF0F06A
:1034600001FB1030A283C0B208B1C0F11E00801869
:10347000A08380B2E27D618B521E5043401860836E
:1034800007F13005608BB43080003866062089F87B
:103490000300E17F41F00801E17720E040F0010006
:1034A0006075D8F804104A78510744BF40F0020014
:1034B0006075607D44F0F4F9A0750023401C82B271
:1034C000387CC0F3800100F0030044F0B9FAA08317
:1034D000A08B00F59670A0833D6689F80350A17D0E
:1034E000207D61F3050007F1880120750870032233
:1034F000607D48708A70B07E800000F0040040F06B
:1035000003008870F27ED20002F008021043887037
:103510000020C870C7F89000B08BC0F30B00B083D8
:10352000D8F80410CA7D40EA0230B0830022617DE1
:1035300001F0FE012046FFF777FE019700271EE00D
:103540001C2010FB07F004EB000B01991C220BF16F
:10355000640005F0F4F90BF16C00052101717F1C8A
:10356000A28B92000260FFB2DAF83C104A6911683F
:10357000737903EB43031944B1F801204281E07DE4
:10358000401E8742DCDB019F2046FFF70FFBE07DFA
:10359000012809D013D3032808D03EBF04F16400EA
:1035A0007860C8F818500AE07D6008E004F1640013
:1035B000786004F18001C8F81810C8F8345041F65A
:1035C000240038860021798607F13C05B868618BB4
:1035D00000EB8100B863022182202870697000210D
:1035E00094F82100E97000F03F00A870D8F80400BA
:1035F000807D012818BF022803D100F07F00401E03
:1036000004E083280CBF0620022020212871697164
:103610004FF0000BDAF83C0041690868727902EB60
:1036200042021044B0F80110E980C7F86CB0D8F835
:103630000400417811F0030F20D044F0ADF9F86692
:10364000DAF818000078C107DAF8181009784CBFCA
:103650001F200F208A07DAF81810097848BF40F0B9
:1036600020004A07DAF81810097848BF40F04000F7
:103670000A0748BF40F0800089F8140089F815B0A7
:10368000D8F80410594A897C01F0030189F8151013
:10369000B07E800000F00400014389F81510F07E30
:1036A000C00000F00800014341F0100189F8151036
:1036B000107838B199F8140000F0FE0041F0400194
:1036C00089F8140089F81510E07F44F0E9F884F8CF
:1036D0002000204644F044FAE07FC10636D5D8F8F1
:1036E000040094F820204178521C88074EBFD21E57
:1036F000F07F12182879C0F380010023D2B200F0C5
:10370000030044F09DF930801E22308800F5967049
:10371000C0F11E0190FBF2F21E2000FB021131717C
:10372000D8F804104878810731884CBF00204FF446
:103730009B70401830807080B86B31883279521895
:10374000A63200EB82007867022002E0C7F874B06E
:10375000002089F8170004F13000C7F8800007F155
:103760008400D8F804104A78510707D504F13802CC
:10377000026099F8150040F0200007E01C490A6833
:103780005168016099F8150000F0DF0089F8150014
:10379000A17F94F8200060F30501A17740F60B00AB
:1037A0002882A5F812B0DAF8380000888000786521
:1037B000DAF83800008800B10720287702206877FF
:1037C00094F84510E983D8F804004178880744BF8D
:1037D0000121E983009808B1FFF7F8F80020BDE85F
:1037E000FE8F00BF50230020B07F0400880E002011
:1037F0006C0F00202DE9F84F0446002000900CB912
:1038000005F060F804F1500569462E682046FFF780
:1038100069F908B9072015E1A04641F28839DFF8B7
:1038200028B2DFF828A2002469684A7A1820604389
:1038300001233718A3401A420AD098F80E103AF81C
:103840001100388000211BF80420BA73F97302E0DC
:1038500040F6010038800021798007F11800786077
:10386000387B00F0EF00387340F08000387398F830
:103870000E10012916D1397B002C0CBF0220052027
:1038800001F0F0010843387324B944F00DF800F555
:103890007A6000E04846B860787B00F0F00040F0C5
:1038A000020017E0002C0CBF0221002100F0F00004
:1038B0000843387324B943F0F7FF00F57A6000E05D
:1038C0000020B860022C797B0CBF0120022001F09F
:1038D000F00108437873641C06F14800386106F172
:1038E0006801032C79619FDB98F80E000024012801
:1038F00008F1A80718D108F19C007063182231461E
:1039000005F01DF806F118002865C5F854903978BF
:1039100001F0F00141F005013970787800F0F00015
:1039200040F00200787000E07463B068C8F81000DE
:1039300047480178397444F02FF8B06445488169EC
:103940000978CA07826912784CBF1F210F2193079B
:103950008269127848BF41F02001530782691078CC
:1039600048BF41F04001020706F14C0248BF41F058
:103970008001117054706968887C00F0030008F1C0
:103980003E0150700B7863F3820050704978947058
:1039900061F3C3005070D47040F010005070346573
:1039A000746508F13800F06598F80E00012818BF1A
:1039B000042815D0A86830B1B0F803009070A96849
:1039C000D1F805003065E86830B1B0F80300D07078
:1039D000E968D1F8050070651F4801684868F0651E
:1039E00008F13000B065D07D00F0EF00D07540F0F8
:1039F0008000D07500F0F00040F00600D075286916
:103A0000B0F8030000280EBF144849F6404148436F
:103A100070661349087838B15078117840F040004A
:103A200001F0FE01507011700E498B7850785906E4
:103A30004CBF40F0200000F0DF0050700098FEF70F
:103A4000C5FF0020BDE8F28F506E0210F46B02102B
:103A500050230020B07F04006C0F002000204E0097
:103A6000880E0020C00C002070B5214B214D197824
:103A700001F00104C1F340010C191978C1F3800170
:103A80000C190022A97B2539060018BF0128C9B2EC
:103A900001D01E2070BDE4B2012C11D0040003D16E
:103AA000022910D04A1C05E001280CD109B90222D4
:103AB00009E04A1ED4B2022C05DDD0B2032815D18C
:103AC000084670BD00221C78012595402C42F4D197
:103AD000040004D1D4B2022CF4D0521CEAE701282D
:103AE000E8D1D4B2002CE2D0521EE3E770BD00BF93
:103AF000F8100020E80B002038B5044601F090FCD7
:103B000004F00102C4F340018A18C4F380018A184A
:103B1000D2B290FBF2F102FB11010025C9B20020E4
:103B200001228240144203D0EAB28A4204D06D1CC2
:103B3000401CC2B2032AF3DBC0B232BDF0B5124B57
:103B40001B7890FBF3F403FB1400FF2100220023F9
:103B50000E4C0025E65CEE40F70704D5D6B287B2DE
:103B6000BE4209D0521C6D1CEEB2082EF2DB5B1C6B
:103B7000052BEEDBC8B2F0BDD90051FA85F1CDB20C
:103B8000FF2DF7D1F3E700BF70230020682300204A
:103B900038B504460D4600210C4A2172107810B148
:103BA000204643F0C1FE204600F0ECFB3C2D18BF40
:103BB000432D0AD106488178880706D52946204634
:103BC000BDE83840FF2243F0DBBF31BDB423002005
:103BD000200E00202DE9F84F054605F14C0AE87D3E
:103BE0009AF80010DAF8047081424FF00008C0F033
:103BF000938105F1280407F1900907F17306C34684
:103C000040F08C80A87F7075E97FB175DAF80820E4
:103C10005278930710D5EA7FD30604D5C01E70757D
:103C200001F0EF01B175C7F874B086F8008000228A
:103C3000B17D01F0FE016AE1910608D4E08B00B18C
:103C4000E07E3076E08B00B1206AC9F80000DAF837
:103C500008004178CA070DD5E08B00281CBF206AF8
:103C6000002807D0C9F80000A17EE08B814238BF50
:103C700008463076E87FC1060CD5B86B217800EB9A
:103C80008100B863B86BA98CA63100EB810078671E
:103C9000022002E0C7F874B000203070DAF80800A3
:103CA000417811F0030F22D1007837F04CFB5FEA26
:103CB00000081CD098F8B000032809D1E87F8106DD
:103CC00015D440F02000E877B07D40F020000DE0F2
:103CD00068B9E87F81060AD500F0DF00E877707DDB
:103CE000A0F112017175B07D00F0DF00B075E97FC1
:103CF000002201F0FC012846FFF796FAB8F1000F08
:103D000036D0E87F810633D598F8B00002282FD14D
:103D100041462846BDE8F44F37F019BBE87F8106DD
:103D20000AD500F0DF00E877707DA0F1120171750F
:103D3000B07D00F0DF00B075DAF808004178C80700
:103D400017D5B07D717D00F0F700891E01F03F01AD
:103D500082075CBF891D40F00200420644BF491E35
:103D600000F0BF00B0757175C9F800B086F8188012
:103D7000D2E09AF80020E87D121AD2B289070092A8
:103D800040F18280012A07F140083FD1B86BA98C2D
:103D900000EB8100B863A87F00F03F00A877707542
:103DA000E97FB175DAF8082053785A0703D5801FE8
:103DB000707501F0FD01B1750023707DE17E00F0AA
:103DC0003F00421898F80000521CC0F3800192B2E4
:103DD00000F0030043F034FE00F59B70A8841E2120
:103DE000A88C90FBF1F18AB2B17D01F0FE0128466A
:103DF000FFF71AFA86F800B0E08B00B1E07E30766B
:103E0000E08B00B1206AC9F8000085E0B86BA98C8E
:103E1000022A00EB8100B86326D1E87FC10706D5EE
:103E2000707D811F7175B07D00F0FE00B0750023BC
:103E3000707DE17E00F03F00421898F80000521CAF
:103E4000C0F3800192B200F0030043F0F9FD00F5E9
:103E50009B70A8840022B17D01F0FE012846FFF787
:103E6000E3F9607FA8F81A00617F0098491C081ADE
:103E7000C0B201281CDDB96BAA8CA63201EB82010D
:103E800079670221317014E0B86BA98C00EB8100D6
:103E9000B863617F0098081AE97FCA06C0B207D5E7
:103EA000B96BAA8CA63201EB8201796702213170CD
:103EB00090B395F81F80A97FD9F80020E37E1A44BB
:103EC000C9F8002028F00108DAF8082052785307D2
:103ED00048BF28F00208920748BF28F008080128C8
:103EE00007D1207F3076C7F874B028F0100886F824
:103EF00000B001F0C004404643F0D2FC00F03F00A7
:103F00002043707586F81680002208F0FC012846D0
:103F1000BDE8F84FFFF788B9BDE8F18F2DE9F04112
:103F2000044604F1500500202E68708006F17308E5
:103F30006968487AFFF7E0FD2530207604F1220712
:103F4000207EB0732046FEF731FE207D88F81500F4
:103F50000020617D88F8161088F81800C6F89000D7
:103F60003888401C388080B237F01CFA84F8210071
:103F70006868417811F0030F42D1007837F0E3F917
:103F800000283DD000F1B0010878032806D1E27F77
:103F9000930603D442F02002E27731E001280ED1EB
:103FA000E07F40F02000E077607D40F01800607511
:103FB000204637F0F5F9204637F0CBF920E008B17C
:103FC0000879E8B1E07F00F0DF00E077A86800281A
:103FD00004BFE868002810D16868007D83280CD0F1
:103FE000617D03280A4607D0C80648BF01F0EF02EA
:103FF000100748BF02F0F7026275204637F0D0F98B
:10400000617D002201F0FE012046FFF70DF900203E
:10401000708606F13E0094F8211001F03F01017016
:10402000B168628B01EB8201B1630021018294F8D7
:104030004520828369684A78910709D5BA887A80D1
:10404000A17F01F03F0141F08001A177012181832F
:10405000E07FC10608D5B06B7988A63100EB8100FE
:104060007067022088F80000BDE8F0812DE9F0417A
:10407000DFF85C8198F80000002143F055FD040052
:1040800004F1500602D104F01DFC91E0207A08B939
:10409000002140E0217B491C21733069407920B127
:1040A000C9B2814208BF432135D004F13E07002048
:1040B000B8730B2501F0B4F97168D1F80320D4F876
:1040C00010E022F07F4240F6C41303FB02EE90FBA7
:1040D000F5F50B2202FB1500D6F800C080B24FF4B4
:1040E0007A6148431EFA80F0CCF8080033683948FA
:1040F0009968216133690268B3F8030000281FBF83
:10410000706E0028A37B012B0CD0938801EB8301F8
:10411000814207D33C212046FFF73AFDBDE8F0413C
:1041200037F0F2B82C4D2878012809DDD0680168F5
:1041300010680969006902F067FB08B1FEF790FF9B
:1041400070684178C8061BD5A17B01290CD10022DB
:104150002272287810B1204643F0E6FB1F48007811
:10416000022104F0BBFD0EE0306890F8631001F00E
:10417000E00141F0860180F863101949416602E0D0
:10418000204637F013F91749087888B138780228A3
:1041900018BF03280CD1144F38680D3043F034FD9C
:1041A00030B93868C11D062204F1300004F0C7FBA5
:1041B00037F0AAF84CB17068017E480605D5414633
:1041C000BDE8F041032043F09BBDBDE8F08100BF96
:1041D000D50F0020B0230020B4230020C70F0020FB
:1041E00000204E00880E0020680F00202DE9F843C3
:1041F0004F4C2168087B68B943F042FD2168096A89
:104200000878002804BF8888002840F080800021BA
:1042100009207AE0474D484E0020688043F044FB77
:1042200000F6C410009020683278C16902EB820267
:104230008818C1888088814202BF404908790128D6
:1042400065D03F4F0099386A02F0DEFA68B1786AAB
:1042500018B1009902F0D8FA38B10098A860216826
:104260000868BDE8F24303F047BA0020FFF7FCFB03
:104270002530A87340F6C4122168C86990F802C0BE
:104280003378BCF1050F48D183F00103337003EBA1
:104290008303C86903447879DB7863F3410078715C
:1042A0003078D1F81CC00B6900EB80080CEB0809D2
:1042B000B9F804C002FB0C3CC5F808C0C1F810C036
:1042C00043002B7438BB6874A8683578CB6905EB5C
:1042D00085055E19F38802FB03023A62194A1078D9
:1042E00088B1887A022818BF03280CD1164D286897
:1042F0000D3043F089FC30B928682368C11D0622BF
:10430000181D04F01CFB00210A2043F0F9FCBDE855
:10431000F14336F0F9BF2020D5E703EB83031844BF
:10432000D1F810C0808802FB00C0A8600861CBE70C
:10433000500F0020E80B0020D80F0020A8230020F9
:104340008C0A0020880E0020680F002001780129C7
:1043500008D002290AD004290CD0082904D0102939
:1043600006D009E0FEF7B0BE36F0F5BF034870474F
:1043700036F0FCBF0248704740687047E80B0020E9
:10438000040C002010B50446A07A00F0E1FD50B105
:10439000617B8A0707D5017B41F001010173607BD6
:1043A00000F0FD006073616D087E020607D5607B3A
:1043B000C20704D4BDE81040012043F0A1BC10BDE9
:1043C00010B5010018BF012803D002281CBF062821
:1043D000002015494FF4C1520A8000234B8000226F
:1043E0004A608A600A73CA7301234B7388730F4A49
:1043F0000F4813880B82C26B0E4B52684A61C26B26
:1044000092688A61C26BD268CA61C26B12690A6221
:10441000C26B526910681C7804EB44042044B0F865
:1044200001204A8210BD00BFEC0A0020A00F00202E
:10443000B07F0400CA0F0020F8B58AB002A81C495A
:104440001C4D1D4C202242F0BFFC0026CDE9006629
:104450001A482E68006856F8607F002302AA214699
:10446000B847174AC2E900016188ADF80010BDF8ED
:1044700000000028F9D0B1F5A05F05D0002004F0BD
:1044800021FA892043F01CFB0E490F4BC8680F4CE2
:104490004288187802432280C868007881060C4957
:1044A00043BF0C480068400A002008700BB0F0BD04
:1044B000487F0400200F0020EC0A00201C0F002081
:1044C000600E0020B07F0400C40F0020A00F002069
:1044D000C90F002080130050F8B590B004460D4677
:1044E00008A82049202242F06FFC0020ADF80A0005
:1044F000039040F603079DF815109DF81400ADF8E1
:10450000087001F0F001002200F0600041F00101AC
:1045100004928DF814008DF81510ADF81650ADF812
:1045200018208DF81A408DF81B200792CDE9002243
:104530000D4C0E482568006855F8606F002308AAE6
:1045400002A9B0470A4AC2E90001BDF80A00B0F565
:10455000806F05D0002004F0B5F9882043F0B0FA50
:1045600011B0F0BD687F0400200F00201C0F002058
:10457000600E00201CB50F490F4CCA6B53691A68B6
:1045800000EB40000244B2F8013063821022ADF823
:1045900000200A4BCA6B52691168094A1C6808441A
:1045A0006946B0F80100ADF80200106854F8242FF5
:1045B000904713BDB07F0400EC0A0020200F0020BC
:1045C0001C0F0020F8B504461646FF2730000D46A4
:1045D0001DD0104908688047014604202318421E58
:1045E00093F87630FC2B08D1F3B22B44204413F817
:1045F000013C80F87630761E1746D0B200281CBFEA
:10460000F2B2002AEAD1084603490A689047F8B294
:10461000F2BD00BF501B0020541B00202DE9F041CB
:10462000054614480E460168904688470124002735
:10463000291991F87710FF2916D0002200E0521CAA
:10464000D3B216F803C0BCF1FF0F0AD06145F6D112
:104650002A19FC2182F87710F9B2F35C08F80130CE
:104660007F1C641C042CE3DB03490A689047F8B202
:10467000BDE8F081501B0020541B002070B504469B
:1046800004F1380004F190060178174D417030783C
:1046900001281AD120897288401C904215DB04F150
:1046A0006101204643F048F9D4F89C112046884720
:1046B0002A68A1795054A0792A68125C04F161013A
:1046C000FCF700FF0220307006E0D4F89C11204671
:1046D00088472A68A17950542868A179425C2068EB
:1046E00041688A7370BD00BFB823002070B50446CE
:1046F000C0B200F023FC0546E0B200F029FC0646FB
:1047000005F5CB700178012916BF02294C1E8C1EBD
:1047100001796879022908BF002108B9FF2070BD1E
:10472000307CC2070FD495F894300022E0B243F0F9
:1047300087F9716980B241F6583201F0004102EB0D
:10474000C00211437161002070BD0000F8B58B48B4
:104750008B4D01782A788A4200F00E816A68002425
:1047600000E0641C8C4280F204814FF4D0736343F8
:10477000134418790028F4D1E0B200F0DFFB0121E6
:10478000017100224271426200F1610184710122D3
:1047900000F168034A711A71012400221A609A60BC
:1047A00000F1900602814281047480F83920826110
:1047B0000277C283327000F592749A762275802750
:1047C0001F739A730027FF22DF741A7600F20D130D
:1047D0001F70DF70BC46BE4600F5897783F801C0C4
:1047E00083F802E0A7F800C0A7F802C087F805E048
:1047F00000F1E70386F804C083F800C083F801C025
:1048000000F1EC03C3F800C0C3F804C083F80AE069
:1048100083F80CC083F808C083F80DC083F80EC07D
:1048200083F80FC0A7F808C0A7F80AC0A7F80CC003
:10483000A7F80EC047F23057A76100F5C676C4F856
:1048400000C02273A4F80EC084F81CC084F81DC0F8
:10485000A2770127B7720227F77286F80EE086F872
:104860000CC0484FDFF820E13F78777386F806C028
:1048700084F80AC084F804C084F805C084F806C02F
:1048800084F807C084F808C084F809C000F5B37440
:104890003E4F84F800C086F800C04FF01B0C3F88E4
:1048A000E7803B4F3F882781BEF800706780394F13
:1048B0003F88A780A4F80AC04FF4A477E781278235
:1048C000A4F80CC0E7822783A4F812C0A4F814C08F
:1048D0006783A783E78327846784A784A6F802C039
:1048E0000127377100240719641C042C87F87720EE
:1048F000F9DB294A14780C7057784F7094788C70D3
:104900000446D778CF7012790A710021234A5018D3
:104910006718407887F8FD00491C0829F7DB204814
:10492000306100211974A07900F012FB0646A079CD
:10493000FFF7DCFE1B480178307C717300F0FC004F
:1049400030740022B069F28100F0004040F48530FC
:1049500040F04000B061307F00F0F80030772878F8
:10496000401C2870C0B2012804BFA079A87020465E
:10497000F2BD002003F0A6FF0020F2BDD40F0020FE
:10498000780E0020C50F00208A0F00208C0F002019
:10499000980F0020960F002060230020C00C0020FC
:1049A0004DE50110F410002070B5254E0446306826
:1049B000A2792C2500F11C016A43885808B104F043
:1049C0007BFDA179306869430144886A08B104F02D
:1049D00073FDA17932686943505C00281EBF194BF2
:1049E000D869002803D00023535436F096FCA379ED
:1049F000306815FB03F52C220021284403F0D1FF79
:104A000011480078082818BF072803D1A17901228E
:104A100036F086FC60790D4D40B1002161716878F7
:104A200008B903F04FFF6878411E69702878401E6E
:104A30002870C0B208B9FF20A8700021217170BD94
:104A40007423002078230020C80F0020780E002057
:104A500038B50446C0B200F071FA0546E0B200F085
:104A600077FA697909B9FF2032BD017CC1F34001B1
:104A700039B96A8E40F6C4114A43816962F31E0156
:104A80008161002032BD0000F8B542F00DFF0546FF
:104A900005F6C41500261E4F00E0761C3978F0B2EA
:104AA000884232D200F04AFA044660790028F4D0F5
:104AB00018490A68A07910702946204643F040F84A
:104AC00020680178402902BF04F1820001780129A1
:104AD00002BF41886289914205D1A169C088091845
:104AE000204600F0B9F9A079FF2136F055FCE089A5
:104AF000B4F862114008884205D3207C18B9A07927
:104B0000012136F017FCA079F2BDFF20F2BD00BFF5
:104B1000D40F0020340F00202DE9F04705460E4643
:104B2000924680281EBF4028002003F0CBFE3C495F
:104B3000487850B33B480078002142F0F5FF04006C
:104B400004BF002003F0BEFE802D21D1616D4878A6
:104B5000C20604D5A27B012A18BF042A1FD000F088
:104B60001402042A1BD0C20606D5A07B20B9887C7B
:104B7000022818BF032816D0487810F0140F04D16B
:104B8000887C022818BF03280DD00020BDE8F087DC
:104B9000402DFAD1244801684A69107808B90124E7
:104BA00002E00128F1D100240027204DDFF88080A9
:104BB000DFF880901BE08879504502BF0B78307891
:104BC000834213D148787278904202BF8878B278D5
:104BD00090420BD1C878F278904202BF08793279BE
:104BE000904202BF48797179884217D07F1C99F8AA
:104BF0000010F8B28842C8D200F0A0F90146487906
:104C00000028F3D0002C01F59471D4D18A79D8F81A
:104C1000000043F025F829788842E7D20120B5E763
:104C2000780E0020D60F0020540F0020D42300203F
:104C30006C0F0020D40F002003490A78022AA4BF79
:104C400000210167704700BF780E002038B50400CE
:104C50000D4608BF03F036FEA079294642F098FEC3
:104C60002046FFF7E9FF204642F0DAFFBDE8314079
:104C700036F04ABB30B50F4800210022431CCCB2AD
:104C8000491CCDB21A55082DF9DBD02141723022D2
:104C900082727821C17208220273002141738173EC
:104CA000C1730174FF218278417042F05902827011
:104CB00030BD00BFC00C002038B504460B4A6088E8
:104CC00013880025834238BF8A200AD3884238BF20
:104CD0008B2006D342F090FEA06008B1012502E0CF
:104CE000812042F0FDFE284632BD00BF382300205F
:104CF0002DE9F84F07460C4615469A46C0B200F01B
:104D00001DF98346F8B200F023F9074601263879E9
:104D1000DFF83C81DFF83C91012802D0022859D00D
:104D200094E0BAF1020F0AD1002078803880022284
:104D30003A71B86804F010FA0020B8604DE0388885
:104D400002280FDB7A8841198A420BDA002078802A
:104D5000388002223A71B86804F0FEF90020B86089
:104D60008B203DE001280CD128000AD079882078DA
:104D7000091D41EA0021798038462946FFF79CFF4A
:104D80000646B868002861D0012E5FD13B882A46CC
:104D90002146184403F0D3FD38882D183D80ADB26C
:104DA0007A88954252D19BF87410802917BF8129C7
:104DB0007F2199F80000091A49B200915346B96859
:104DC00098F80200FCF72AFB002078803880022245
:104DD0003A713BE0BAF1020F38D1280004D18C209F
:104DE000BDE8F24F42F07CBE012D03D13D80217819
:104DF00079802AE021786078091D41EA00217980D4
:104E000038462946FFF758FF0146B868F0B1012936
:104E10001CD12A46214603F092FD7A88954211D191
:104E20009BF87410802917BF81297F2199F8000011
:104E3000091A49B200910223B96898F80200FCF7F8
:104E4000EDFA03E038882D183D803E71BDE8F18F02
:104E5000780E0020C90F002010B50268536814694D
:104E600040F6C41202FB01449C6081614FF4C87398
:104E7000428A5143B1FBF3F1491C416101684B681F
:104E80009A684169521A9A6001684B689A688A6008
:104E9000BDE8104000F000B87CB5044604F186017E
:104EA00042F092FF04F18205002168896084217735
:104EB000E18304F12E066189E0894118A1812A89E4
:104EC000B188A8898A4204BF3389984202BF6B899E
:104ED000F1888B4206D0000900906B89A1795208B5
:104EE000002004E0000900905208A179302042F02F
:104EF00017FFB088A4F86401297931702889B0803F
:104F00006989F180A8893081204642F0F1FD0220B4
:104F1000287073BD044B1B6D2BB143F8220001F1C7
:104F2000045141F8280F7047FC100020024A5268D3
:104F30000AB142F821007047FC100020034A536870
:104F40004FF4D07148431844704700BF780E0020DA
:104F500002490A6802EB4010704700BF542300204A
:104F600038B5784D687904F097FA774900280860D9
:104F700063D00022026002730868C2610262A879ED
:104F800004F08AFA71490028086056D000220260B5
:104F9000C27200200A681074052308684374002256
:104FA00009684A61E87A04F077FA694900280860DC
:104FB00043D0684C21782878491D10FB01F080B25D
:104FC00004F06AFA64490028886036D02078002806
:104FD0006FD0698811FB00F080B204F05DFA5F4A7F
:104FE0000028506029D05E482278017811FB02F039
:104FF00080B204F051FA5B49002808601DD00025FA
:105000000AE0E8B2FFF7A4FF00214180816001803F
:105010000223037101736D1C2078E9B28142F0D341
:1050200004F03AFA50490028086006D02078400081
:1050300004F032FA4D49002808607CD020781C2109
:1050400010FB01F080B204F027FA494A00281060F2
:1050500071D02078400104F01FFA4649002808600A
:1050600069D0102004F018FA43490028086062D083
:105070002078000104F010FA4049002808605AD056
:10508000302004F009FA3E490028086053D0207807
:105090002C2110FB01F080B204F0FEF9394A0028FF
:1050A000106048D0207804F0F7F9374900280860EC
:1050B00041D0364C364D2178287800EB4100C000B5
:1050C000103080B204F0E8F932490028086032D08C
:1050D00000F1080141602878227800EB4200C0000E
:1050E000103080B204F0D8F92B49086018B300F1F1
:1050F000080141601E212078401C10FB01F080B2A5
:1051000004F0CAF9254A1060A8B1082004F0C4F9D7
:10511000234C206078B1062004F0BEF921680860B5
:105120002168086838B100204860062004F0B4F90E
:105130001C49086008B9072032BD36F0F7F800B105
:10514000002032BD64110020500F0020540F0020B9
:10515000440F0020D40F0020E4230020780E00200C
:105160007411002054230020340F00204823002015
:10517000980E00209C0E0020A00E0020A40E0020FF
:10518000A80E002074230020B8230020D52300207F
:10519000D42300206C0F0020700F0020680F002027
:1051A000E0230020400F002010B53448006808B10B
:1051B00004F082F93248006808B104F07DF9314802
:1051C000006808B104F078F92F48806808B104F04D
:1051D00073F92E48406808B104F06EF92C48006855
:1051E00008B104F069F92B48006808B104F064F9CB
:1051F0002948006808B104F05FF92848006808B140
:1052000004F05AF92648006808B104F055F9254819
:10521000006808B104F050F92348006808B104F0B0
:105220004BF92248006808B104F046F920480068AC
:1052300008B104F041F91F48006808B104F03CF9D6
:105240001D48006808B104F037F91C4C2168086853
:1052500010B1086804F030F9206808B104F02CF9A6
:105260001748006808B104F027F91648006808B12B
:1052700004F022F9BDE8104036F057B8500F002076
:10528000540F0020440F0020E4230020780E00205B
:1052900054230020340F002048230020980E0020C3
:1052A0009C0E0020A00E0020A40E0020A80E0020BE
:1052B0006C0F0020700F0020680F0020E0230020FA
:1052C000400F0020742300202DE9F0411C4CDFF832
:1052D00074801D4D07462021404600F0A6F8236843
:1052E00053F8386F202241462846B0472368174EAE
:1052F000174C394653F83C7F41223046B847154F8A
:10530000396851F8102F204690471349134AC86B4B
:10531000006C20606560A66021463B68106853F809
:10532000182F0F4D9047286010B1002003F0CAFAE3
:105330002021404642F040FD286840B2BDE8F0819F
:10534000280F0020540B0020340D0020440D0020B5
:10535000F00D0020240F0020B07F0400580F002023
:105360005C0F00202DE9F843234D244C2B68DFF817
:10537000909053F8386F07468846202249462046C9
:10538000B0472B681F4E394653F8387F41223046CC
:10539000B8472B681C4F53F83CCF41224146DFF8F9
:1053A0006C801B4D3846E047D8F8001051F8142F98
:1053B000284690471749C86B006C28606C60AE6047
:1053C000EF602021484642F0F7FCD8F80020124850
:1053D00052F81C3F0068114C294698472060202154
:1053E000484642F0E9FC206810B1002003F06AFA58
:1053F000206840B2BDE8F283280F0020340D002061
:10540000540B0020540D0020640D0020240F0020B8
:10541000940D0020B07F0400580F00205C0F002086
:1054200080B536F0EDFEC0B202BD00F01DB8000040
:1054300038B50A4B1C680A4684B0014654F83C5FF4
:105440006846A847064A07481368006853F8084F9B
:105450006946A047C0B205B030BD00BF280F00208C
:105460002C0F00204C2300202DE9F041264D0E4644
:1054700029688CB0044611B9002003F023FA234BAD
:10548000234F21461C68324654F83C6F6846B047AB
:10549000204E3068804780462868694637F06CFDAA
:1054A000044639684046884714F1030F24D120216F
:1054B00004A8FFF7BDFF10B1002003F003FA306825
:1054C0008047804628680023002204A937F05EFD4B
:1054D000044639684046884714B1002003F0F2F9C9
:1054E0003068804706462868694637F045FD04461F
:1054F00039683046884703E014B1002003F0E2F930
:10550000E0B20CB0BDE8F081D8230020280F0020C5
:10551000541B0020501B0020114800B501688FB0BB
:1055200011B9002003F0CEF9202107A8FFF780FF72
:1055300037F0AAFC684637F025FC102042F21071C3
:105540008DF80000019107AA02926946002037F009
:1055500011FC0449086008B903F0B4F90FB000BDAC
:105560004C230020D823002073B501F023018DF8CF
:10557000041001AD0E490F4CCA6108611A448B60DA
:10558000CB604A610D20012681F8200004230A4ADD
:105590000C604D608E6181F82130084B1C681068EA
:1055A00054F8142F904710B1002003F08BF973BD0D
:1055B000100B0020D40D0020600F0020280F0020C9
:1055C000F2B501F023018DF8001014461D46069A2D
:1055D0001349144B08610B604A610D20012781F8C3
:1055E00020000422104BC1F804D08F618D60CC6183
:1055F000CD6081F821200D4A1668186856F8183FCA
:10560000984748B122460021284603F0CAF90020F5
:1056100003F058F9002000E0012005490870F1BDB1
:10562000100B0020D40D0020600F0020280F002058
:10563000DC2300202DE9F843044618480D46016894
:1056400016461F468847226880461078802804F155
:10565000BA0902D14A46012103E0402806D14A4650
:105660000021D4F8EC0042F063F902E0002003F0DE
:1056700029F904F1C70042F0D3F93B4632462946E6
:105680004846FFF771FFD4F8EC000549401CC4F808
:10569000EC0040460A68BDE8F2431047501B00206A
:1056A000541B00202DE9F843074615460C461E46BC
:1056B000280004BF002003F005F918490868804756
:1056C0003A6880461078802807F1BA0902D14A4624
:1056D000002103E0402806D14A460121D7F8F00016
:1056E00042F026F902E0002003F0ECF807F1C700D1
:1056F00042F096F97019009033462A4621464846F2
:10570000FFF75EFFD7F8F0000549401CC7F8F0002E
:1057100040460A6890470120BDE8F283501B0020F4
:10572000541B0020024940F649600880704700BFC2
:10573000F000002170B5024CA56B2E68B04770BD1B
:10574000FC10002010B5044600F06CF8012807D0CA
:10575000204600F06DF801281CBF204600F0ACF890
:10576000002010BD38B514461D46E00648BF00F0C5
:1057700099FB600548BF00F0C7FB60030BD500F044
:10578000D3FB012805D000F0D7FB012818BF00F09B
:1057900007FD24F40024200348BF00F011FD20027F
:1057A00003D5002000F0C2FD04E0A00344BF0120A7
:1057B00000F0F2FD14F0030F0DD000F0B5F8012851
:1057C00009D000F0B9F8012805D000F01FFA01282F
:1057D00018BF00F0A9FA200405D5114890F8201050
:1057E000491C80F82010002C48BF00F091F815F0FB
:1057F000E24113D015F0045314BF012400242046C5
:1058000000F010F8012809D0204600F011F8012816
:1058100004D02046BDE8324000F04EB831BD00BF94
:105820007823002080B501F04FFF002002BD00006A
:105830002DE9F04104461948194E0278194F012507
:10584000112A02D0122A1AD024E0DFF85C8098F8DE
:105850000000002142F068F9144A117811B10020CB
:10586000107018E0B8B114B9FDF78EF898B198F837
:1058700000100022112035F053FD0D4804E014B94A
:10588000FDF782F838B10B4838600121307803F019
:1058900025FA00E000252846BDE8F081C80F002069
:1058A000C70F0020480F0020D50F0020DD23002067
:1058B0006D4000004DB3030010B50F490A78012474
:1058C000072A16D10D4A117811B10020107011E08D
:1058D0000B498A78FF2A0DD010B9FDF755F848B169
:1058E0000849094A094808600121107803F0F6F9CF
:1058F00000E00024204610BDC80F0020DD2300205A
:10590000780E0020480F0020C70F00203BB3030093
:1059100080B5002002F0D6FF822042F0D1F8BDE829
:10592000014042F03DBA000002480178481E804123
:10593000C00F7047C80F00202DE9FE4F01200190D5
:10594000A74EA848A84F0278112A02D0122A0DD0DB
:1059500040E1A64C2078002142F0E6F8A449054633
:10596000087810B100220A70FCE0002D00F02581BB
:10597000A048DFF88482DFF8849238600122217821
:10598000112035F0CDFC286D696D009141F60802BB
:10599000009B9B495C78E30640F1E680044641F2B7
:1059A0000443B4F802C09C451FBFB4F81AE09E45FA
:1059B000B4F832C09C454FF4A05A1CD095F80EC0E4
:1059C000BCF1010F04BFB5F89EE09E4513D0B4F8BA
:1059D00002E041F20A439E451FBFB4F81AB09B454E
:1059E000B4F832E09E4506D0BCF1010F04BFB5F813
:1059F0009EC09C4503D13380C7F800803DE0002362
:105A000040F2FE3B4FF0180C0CFB03FCA444BCF826
:105A100002E0A6F800E0BEF1010FF3D0BEF1000FE6
:105A20005FD0AEF1020EBEF1010F5AD9BEEB0B0EE4
:105A30001AD04FF48063BEEB030363D04FF4406B86
:105A4000B3EB0B034DD09B1E012B4AD91B1F48D033
:105A500040F2FA3BB3EB0B0379D05B1E6BD0D81E40
:105A600050D0001F4ED077E0B4F800C040F6010ED1
:105A7000F44536D15B1C022BC4DD386840452FD17C
:105A8000A06C0168A06C01F1080501680879032881
:105A900004BF94F86C0001281AD1D5F80E00002834
:105AA0001CBF288B002813D095F8220010F0E00FBF
:105AB0000ED105F11E0041F047FF012808D1688B87
:105AC000298BAA8B401C89004843B0EB021F70DB76
:105AD000A6F800A0C7F80090A06C0168002008712B
:105AE00067E0A87B01281CBF0428A6F800A0C7F81F
:105AF0000090087D0028C0D08868401C0022886083
:105B00000A82BAE7A87B012806BF41F20243ACF83B
:105B10000230ACF802A03088904215D1CA68088AD9
:105B20004D8A521CCA60401C82B2AA4238BF2A4623
:105B30004A82088208E000994A78D1064CBF816CFD
:105B4000C16E086800210171C7F8009095E7002038
:105B500002F0B8FE832003E0002002F0B3FE8420B0
:105B600041F0AEFF012038E0438E41F204455C1B5A
:105B70001CD0A41F1AD03380408890420CD1CA6830
:105B8000088A4C8A521CCA60401C82B2A24238BFAA
:105B900022464A82088206E0087D20B18868401CBF
:105BA000002288600A8241F20643C846C7F8008096
:105BB000338001211348007809E035F0CFFB58B15C
:105BC000C08811490F4A308039600121107803F0F4
:105BD00085F801E0002001900198BDE8FE8F00BF2C
:105BE0009A0F0020C80F0020480F0020D50F00207A
:105BF000DD230020756B0210598000006D4000000D
:105C0000BC230020C70F00204DB30300F8B53C486B
:105C100001780124072970D13A49087810B100228F
:105C20000A700FE0384EB078FF280BD072684FF43E
:105C3000D071484311188879FFF78AF920B1007BA9
:105C4000C10701D50120F2BD304D314828603148EF
:105C500031490A68B3781C214B4313445F8807809D
:105C600017F47F4FF4D02D4A2D494FF40066BF1B27
:105C70001CD00A3F012F1DD940F6F636BF1B032F5B
:105C800084BF7F1F012F09D940F2FF36BF1B05D00B
:105C90007F1E012F0ED9FF1E0CD020E0107D28B3EF
:105CA0009068401C0023906013821FE041F2014085
:105CB00058801BE04FF4A0565E8041F60803008830
:105CC000984213D1D068578A401CD060108A401C7B
:105CD00083B2BB4238BF3B465382108206E00020AD
:105CE00002F0F0FD852041F0EBFE29680D482960A7
:105CF0000121007802F0F2FF00E000242046F2BD0E
:105D0000C80F0020DD230020780E0020480F00205F
:105D1000756B02109A0F0020980E0020BC23002003
:105D20003BB30300C70F00202DE9F0474E4E4F4C08
:105D300096F800904E4FA9F10905042D8AB000F2A3
:105D40008980DFE805F003036767710002A849490D
:105D5000202241F039F8788810F47F4F2080FBD062
:105D6000454C464DDFF81881DFF818A14FF4A051DB
:105D7000401A14D0C01E12D040F20141401A4ED138
:105D8000414A2D68D8F800000023CDE9002355F8DA
:105D90005C8F534602AA3946C047208060E0B9F1C3
:105DA000090F0FD139490A685089002837D038497E
:105DB000087841F0DDFF0021002041F05DFE002069
:105DC00030704DE0B9F10A0F29D1324E307830B33E
:105DD0007078002844D101212F4A717092F8200078
:105DE00030B1B078012803D10021032035F08EFABC
:105DF0002A482D680021CDE900015346D8F800005B
:105E000055F85C8F264902AAC04720800020707098
:105E1000B07025E0788810F47F4FFBD02080002000
:105E200002F050FD852019E078882080022807D9EB
:105E30004FF4A051401A03D040F20441401AEED171
:105E4000B87B801CC1B2B529A8BF6620B8730020FA
:105E5000788005E0002002F035FD842041F030FE1E
:105E600001200AB0BDE8F087C80F00209A0F00207B
:105E7000940B00200C800400880F0020200F0020CD
:105E80001C0F0020F9B2030002000080440F002024
:105E9000CA0F00209C2300207823002002808080ED
:105EA000500C002080B516480278112A02D0122A20
:105EB00020D001BD134B1878002141F035FE48B9C0
:105EC00002F000FD002002F0FDFCBDE80240FF20D2
:105ED00041F0F6BD00F14C02117809B90123C372FB
:105EE000491C117092685178CA0607D4BDE8024077
:105EF00035F05ABABDE8014035F027BA01BD00BF00
:105F0000C80F0020D50F002006488078FF2800D158
:105F1000704780B5FFF712F8BDE80440002141F05A
:105F200023BF00BF780E002002480178481E804140
:105F3000C00F7047C80F00202DE9FE4F8D48027832
:105F40000024521E032A4FF0010A0AD9103A40F0E9
:105F50000C81894C2078002141F0E6FD040000F01E
:105F6000058114B9002002F0ADFC606DDFF80C82F1
:105F70004178DFF80C92834DC806216D4CBF886CC8
:105F8000C86E0622016801F10806B11C01A802F0E2
:105F9000D6FC3078C0F380108DF800004FF01E0B57
:105FA0003778794E07F00F0103292FD101A941F06D
:105FB000A3FE002829D0606D807C012818BF03282B
:105FC00023D1296801A841F067FDFF281DD01BFBE4
:105FD00000FB286810F80B205844411CD9F8000039
:105FE00041F03EFE98F8001088420ED028685844D0
:105FF000C11DD9F8000001AA41F026FE28685844C6
:10600000062201A9C01D02F09AFC9FE007F00F00D4
:106010000528FAD19DF8000001A941F06DFE7F0925
:1060200090B3296801A841F037FD616DFF2823D0A6
:10603000897C022918BF03291BFB00FB0CD12868AF
:1060400010F80B205844411CD9F8000041F008FE1C
:1060500098F80010884279D028685844C11DD9F8B2
:10606000000001AA41F0F0FD28685844062201A969
:10607000C01D02F064FC24E04878C2066FD5887C1D
:10608000F8B1012862D11CE03A48017802295DD1BB
:106090009DF80010286801AA41F00AFDFF2855D09C
:1060A00029681BFB00FB01EB0B00427F012A04D097
:1060B0000D3041F0A9FD002848D040F2014041F0E8
:1060C0002BFC606D4178C80649D530498878410677
:1060D00005D5F80703D4206D41F20A4102E0206D96
:1060E00041F2044141804183418629480180206D6D
:1060F000816C0A68816C08680079032802F108073E
:1061000024D1D7F80E0000281CBF388B00281DD0E2
:1061100097F8220010F0E00F18D107F11E0041F0AF
:1061200013FC012812D1788B398BBA8B401C890063
:106130004843B0EB021F09DA164A1749174886F898
:1061400000A011600121007802F0C8FD606D417867
:10615000CA0604D5307848B9216D886C01E0216DFC
:10616000C86E01680020087100E0A2465046BDE8F4
:10617000FE8F00BFC80F0020D50F0020D4230020C1
:106180006C0F0020680F0020DD230020C00C0020D1
:106190009A0F0020480F002059800000C70F0020F0
:1061A00080B506480178C91F012905D9002002F0F1
:1061B00089FB862041F084FC012002BDC80F00202D
:1061C0002DE9F8434D480278012A1CBF032A112A01
:1061D00040F092804A4F3878002141F0A5FC04003D
:1061E00039D004F15008D8F804004078810740F114
:1061F0008380D8F80060C00604D5B06C016801F156
:10620000080524E0F06E016801F108054FF4966975
:10621000287C03280FD8DFE800F002050B084FF4B4
:10622000EE690BE04FF4C46908E040F6E86905E068
:1062300041F6F03902E0002002F044FBB06B484424
:10624000B06394F845000228A8BFA6F85A000620BB
:1062500041F0D2FD00284FD0D8F80400017EC807D5
:1062600040D50B2003F020F9040037D01320207014
:10627000062239786170A91C2878C0F38010A070BC
:10628000E01C02F05CFBE87B00F03F006072A97B41
:10629000802918BF81290FBF7F211A4A1078091A57
:1062A000A172E11CA07841F027FDA0B1164F39681A
:1062B000E01C41F0F1FBFF280DD01E213A68484355
:1062C000135C43F00203A370062239684B1C1918B3
:1062D000E01C02F034FB2146062001E000210E20E4
:1062E00041F00EFDD8F804004178C8064CBFB06CF0
:1062F000F06E016800200871BDE8F183C80F00202E
:10630000D50F0020C90F0020680F002020B50146DE
:1063100000200A680860134615791268032D08BF2B
:10632000401C9A42F8D10B60C0B220BD70B5044643
:1063300016480178491F15D0891E012920D8144B11
:106340009878FF2821D0FEF7F9FD0026006FFFF7AF
:10635000DDFF0546F0B2A84217DA204600F01CF82F
:10636000761CF7E70B490868FFF7D0FF05460026C3
:10637000F0B2A84209DA204600F00EF8761CF7E7E2
:106380002046BDE8704000F007B870BDC80F00207F
:10639000780E00208C0A00202DE9FE4F0546DFF81C
:1063A0002404DFF824640278002A4CD0052A73D034
:1063B000062A00F08080072A18BF082A00F0F7801C
:1063C0000A2A00F0D381112A02D0132A70D0F1E1F9
:1063D000DFF8F8331878002141F0A6FB04001EBF57
:1063E000606D407810F00C0F2DD0216DC0064CBFB1
:1063F000886CC86E0622016801F10805A91C684670
:1064000002F09DFA287800F00F0105291BD14509FB
:106410006946C0F3801041F06FFC002813D031684A
:10642000684641F039FB0746316804F1380041F015
:1064300033FB87420DD0606D4178C80604D440F22A
:10644000014041F069FABBE1607B40F002006073FB
:10645000B6E133681E2010FB07F69819062269463C
:10646000C01D02F06CFA606D4178C806F0D5A17BC2
:106470000129EDD1DFF858038178480605D5E907F1
:1064800003D4206D41F20A4102E0206D41F2044143
:1064900041804183418693E134F065FF0028FAD1C1
:1064A000FCF78AFE012802D0012041F0ADFA87E115
:1064B00034F05BFF84E1DFF81C53286841F08CFB6B
:1064C0000400F7D020790328F4D1207A00F00F01DE
:1064D000072937D1C04800684169497A4A1E1142EC
:1064E0005ED0617A04F10A035A5C02F03F02252A69
:1064F00056DBA17A8A09012A52D111F03F0F4FD001
:10650000007CFEF71BFDE17ACA074CBF04F11102C3
:1065100004F10B028B0748BF921D0B0748BF921C6A
:10652000C90648BFD21C1621127852094A43AB490A
:106530008B180A31EB608A5A428699898186DA89FA
:10654000C2862DE000F00F00082829D1A17A880921
:1065500026D129B3A0480168087CFEF7EFFCE17A58
:10656000074688071CD5062201F001015143601837
:1065700000F10C01684602F0E2F9207AC009FF2818
:106580000ED0694641F0B8FB50B1306800F10D0102
:10659000684641F055FC18B905213846FEF756FB10
:1065A0002079032802D0002002F08CF9FEE0DFF809
:1065B00030B29BF802000024FF281BD0FEF7BEFC7F
:1065C000804608F16C09D9F8040041F005FB2A4621
:1065D0000179032901D011000CD08368197801F0EA
:1065E00003008D06009003D50124009818B9BAE085
:1065F0001000FAD0E4E05D7803F1020A34B31AF82F
:10660000010B784B01902C2098F806C01F6810FBF6
:106610000CFC67444FF0010E87F805E0002A1F6864
:1066200098F806E007F11A0C019F10FB0EFE07F028
:106630001F070CF80E7098F806701B6810FB07F027
:106640001844019BC3F38113C3761AD10098032821
:1066500008F217171AD0ADB199F8000068B108F127
:10666000F4000278012A0DD1564B1A78072A04D07B
:10667000082A04BFC078012804D13D217970012087
:1066800038709DE0584A1378012BFAD098F894009E
:1066900070B32D1FEDB253462A464046FFF702F86D
:1066A00000281EBF51490878002807D13D21797084
:1066B00001203870306841F0FFF881E04C480168F3
:1066C0008847064698F80610DBF804204FF4D0708F
:1066D00041435018002280F8412108F59E7001685E
:1066E0008079490802F0F2FD42490A683046904735
:1066F0000098032819D04048416909788A0708D5CD
:1067000041690878C1074CBFE81C28461AF8000008
:1067100000E0812089F808002A460098C3B29BF85F
:1067200002005146FEF7E4FA1DE09AF800001CB1A1
:106730001B2804BF022D01251C2803D22F490B5C06
:106740009D4205D0B8700721404641F059FB0AE050
:106750001C48017808295146404602D134F0D2FD48
:1067600001E001F02FF9D9F8040020E0244C207852
:1067700030B3244D286841F02FFA08B3017903297A
:106780001ED1017A8A0611D5807AE178C0F3811290
:10679000914202BF217900F01F00814206D1A0780A
:1067A000002801BF607800280121A170286841F00D
:1067B0006FFA05E0002002F085F8862041F080F9AC
:1067C000BDE8F78FC80F0020680F0020D50F00200C
:1067D000C00C0020BC0A0020540F0020E00700205D
:1067E000780E002074230020D20F0020DC2300202C
:1067F000501B0020541B0020B07F0400F07F0400D9
:106800009C230020AC0C00208142064A03D2401A8F
:106810009042804103E0081A90428041C043C00F7B
:10682000704700BF01E07072F0B50023FF200F49F0
:106830000F4A002711E01C248E6814FB03F4264441
:106840005B1C7770DBB28D6828558E6834446761B5
:10685000A7616760A760E76027611478641DA342A1
:10686000E9DBCF700F804F608870F0BDE42300201B
:10687000D40F00202DE9FE4FDFF81883D8F804600C
:106880001EB9BDE8F74F41F03BB83078DFF8089308
:10689000C24FDFF80CA3012818BF02280AD0042831
:1068A0001CBF0828102805D0402818BF802800F0F9
:1068B000A08068E100F0E0FC0028FAD0012000F0A0
:1068C0009FFC20B1012000F0BDFCFDF73FFD08203A
:1068D00000F096FC20B1082000F0B4FCFDF736FD76
:1068E000307800F0D9F905009AF8010014BF6C68FF
:1068F000002400284ED034F04DFDFEF71FFB064665
:1069000030680090D0F804B0B0798AF80300BCB1C8
:106910000099284634F042FD022811D02978012937
:1069200002D0082963D02EE128B940F0BDFF00F560
:10693000E8504C30A060012088F8020011211CE1D1
:106940000098017880290CD10820964938700A787F
:10695000DBF81400012A1ABFD9F8241009780121A4
:1069600013E007203870B079FEF7F2FA0446207B76
:10697000C10748BFB0795DD48A480178DBF81400BC
:1069800001291CBFD9F824104978C172B0798AF85E
:106990000200BCE0002D11D02878AE420AD10128B7
:1069A00018BF082802D1002C03D1F1E0002001F02B
:1069B00089FFE3E0012802D0082816D0E3E0002C8C
:1069C000F3D040F071FF0146A06801F5C241A83143
:1069D000FFF71AFF28B940F067FF00F5E8504C3088
:1069E000A060112038700121C0E0002CDDD008200B
:1069F000C0E09AF80100002800F08B8034F0CAFC57
:106A0000FEF79CFA054628680090D0F804B09AF882
:106A10000200FEF793FA0190A8798AF80300317812
:106A2000402911D1A879FEF793FA0446207BC107CB
:106A30000AD5A879FEF782FA0521FEF707F9207B2F
:106A400000F0FE002073A3E000F0F6FB10F01F0F33
:106A50003AD0012000F0D4FB20B1012000F0F2FB7D
:106A6000FDF774FC082000F0CBFB20B1082000F0FB
:106A7000E9FBFDF76BFC98F8020000F00DF9064603
:106A800074680CB3009934F089FC02281CD031786A
:106A9000012902D008290DD013E028B940F004FFE5
:106AA00000F5E8504C30A06011203870012188F8C2
:106AB000021004E0082088F80200122139703046E4
:106AC0005DE0002001F0FEFE0198A8421FD0009971
:106AD00034480A78802A0BD10821397000780128BF
:106AE000DBF814001ABFD9F82410097801210AE054
:106AF00007223A7000780128DBF814000EBF01214C
:106B0000D9F824104978C172A8798AF8020000984F
:106B100035E000F091FB10F01F0F39D0012000F09C
:106B20006FFB20B1012000F08DFBFDF70FFC08206A
:106B300000F066FB20B1082000F084FBFDF706FCA6
:106B400098F8020000F0A8F8054628786C6801283B
:106B500002D008280DD01BE0D4B140F0A5FE00F50E
:106B6000E8504C30A06001211120387088F80210E4
:106B700004E06CB188F80200122139702846BDE8A3
:106B8000FE4F00F0B9BDBDE8FE4F002001F09ABEF7
:106B9000BDE8F78FE4230020B07F0400C80F002079
:106BA000780E0020CC0F00202DE9F041040048F6BB
:106BB000B80564D04E68676840F076FE804620785D
:106BC000022808F6C4180DD12E4908682E49C2695A
:106BD000087800EB800010448188C088814211D180
:106BE000C7F80880207804280CD12849086828496B
:106BF0004269087802EB001041898089814208BF10
:106C0000C7F80880B0684146FFF7FEFD012808D0AC
:106C1000B0684146FFF7F8FD012818BF002001F0D9
:106C200051FE2078012804D11A4801688D88AD00F2
:106C30000FE0082804D134F091FB08B1D0F890504F
:106C40002078102805D1032034F093FB08B1D0F848
:106C50009850B068414640F0ABFF85420FD2B06813
:106C6000411BB868FFF7D0FD48B9B86808F58842FD
:106C700002F15C01FFF7C8FD10B1012000E0022025
:106C8000BDE8F081500F0020D80F0020540F0020E5
:106C9000D90F0020B02300202DE9F041FF28054640
:106CA0002AD100F0C9FA10F01F0F22D0042000F002
:106CB000A7FA08B1042016E0012000F0A1FA08B1FB
:106CC000012010E0022000F09BFA08B102200AE047
:106CD000102000F095FA08B1102004E0082000F020
:106CE0008FFA20B10820BDE8F04100F0ABBA01F006
:106CF000E9FD0020BDE8F08100F0A4FA5FEA000899
:106D000014BFD8F804400024012D46F2A81740F61D
:106D1000C4160BD0022D63D0042D00F0A280082DE4
:106D200000F0EF80102D00F05181E2E7012000F02B
:106D300067FA00281EBFDFF81403006800281CBF94
:106D40008788BF00102000F05BFAE0B1102000F04F
:106D500079FA05466E6846B9022000F051FA20B172
:106D6000022000F06FFA05466E68012000F048FA34
:106D700038B1B068C11BA068FFF746FD08B94046AE
:106D8000B8E72846B6E7022000F03AFA88B10220B8
:106D900000F058FA06460120756800F031FA30B16B
:106DA000A868C11BA068FFF72FFD0028E7D0304678
:106DB000A0E7042000F024FA08B10420E8E7082046
:106DC00000F01EFA30B1082000F03CFA41680029BA
:106DD00090D1D4E7012000F013FA00288AD0CEE742
:106DE000022000F00DFA58B1994801689948CA6923
:106DF000017801EB81015318DF88774307F51667A7
:106E0000042000F0FDF928B1042000F01BFA06462A
:106E10000220C1E7082000F0F3F980B1082000F05B
:106E200011FA05466E6846B9012000F0E9F920B173
:106E3000012000F007FA05466E68022096E701205F
:106E400000F0DEF928B1012000F0FCF9064602202E
:106E5000A2E7102000F0D4F908B11020B4E7022016
:106E6000B9E7042000F0CCF950B17B4801687B48B9
:106E70004A69017802EB01139F89774307F516678A
:106E8000082000F0BDF980B1082000F0DBF90546CC
:106E90006E6846B9012000F0B3F920B1012000F07E
:106EA000D1F905466E68042060E7012000F0A8F9DA
:106EB00028B1012000F0C6F9064604206CE7102036
:106EC00000F09EF988B1102000F0BCF905466E680C
:106ED000002EE8D1022000F093F90028E3D0022030
:106EE00000F0B0F905466E68DDE7022000F088F991
:106EF00028B1022000F0A6F9064604204CE7042041
:106F000069E734F02BFA08B1D0F89070042000F053
:106F100077F9A0B1042000F095F9064608207568BD
:106F200000F06EF9002818BF002C16D0A868C11B0D
:106F3000A068FFF769FC00287FF439AF1FE7012044
:106F400000F05EF960B1012000F07CF906460820EF
:106F500000F056F9002818BF002C3FF428AF0EE7C8
:106F6000102000F04DF9F8B1102000F06BF9054643
:106F70006E6846B9022000F043F920B1022000F00B
:106F800061F905466E68082000F03AF9002818BF3C
:106F9000002C3FF4F6AEB068C11BA068FFF734FCCC
:106FA00000287FF4EEAEEAE6022000F029F958B19D
:106FB000022000F047F906460820756800F020F925
:106FC000002818BF002CB0E7082004E7032034F0A5
:106FD000D0F908B1D0F89870022000F011F950B142
:106FE000022000F02FF90646102000F009F90028D1
:106FF00018BF002CB1E7042000F002F928B10420EA
:1070000000F020F906461020C6E6082000F0F8F847
:1070100080B1082000F016F905466E6846B90120D7
:1070200000F0EEF820B1012000F00CF905466E6882
:1070300010209BE6012000F0E3F828B1012000F0C9
:1070400001F906461020A7E61020C4E6B023002070
:10705000500F0020D80F0020540F0020D90F00201F
:10706000F8B52B4C2B4D217806462878491D8842CF
:10707000A4BF002001F026FC2178491D1C22012E0E
:107080001CBF082E102E0DD1AB68002002FB00F4AF
:107090005F1C3F5D012F04BF1F5DB74217D0401C2E
:1070A0008842F3DB0023AC6802FB03F73C446078C2
:1070B00028B92778FF2F0CD06868844209D15B1C5F
:1070C0008B42F0DB002001F0FDFB0020F2BD18191F
:1070D000F2BD002060606061267001206070287839
:1070E0006978401C28703143C0B201281CBF802E33
:1070F000402E697000D16C60EA7891421FBFE97040
:107100000548426C002A1CBF806C90472046F2BDA7
:10711000D40F0020E4230020FC100020F8B5050067
:107120001FBF2C68002C2078FF283CD0012803D1F9
:1071300040F08EFD002836D12078012802BF1A4E7B
:107140003078012806D1194F386802F0B5F90020CF
:107150003860307000222A6062702078144D402818
:1071600018BF802802D100F06DF818B9697820782E
:1071700081436970287800281FBF401E2870C0B264
:10718000002803D100200B4A686010706978E87805
:1071900081421FBFE9700848426C002A03D0BDE855
:1071A000F840806C1047F1BDB4230020B0230020CC
:1071B000E4230020C80F0020FC10002002490878BA
:1071C00000B14868704700BFE423002030B50A4A88
:1071D00092680021CBB21C246343D55C854208D061
:1071E000064C2578491CCBB26D1DAB42F2DB00206A
:1071F00030BDD018407830BDE4230020D40F0020EB
:1072000010B50B4A926800211C234B43D45C844286
:1072100002BFD3185B78012B07D0064B1C78491CA2
:10722000641DA142F0DB002010BD012010BD00BF95
:10723000E4230020D40F002001484078704700BFAD
:10724000E423002050B501460948836800221C2031
:1072500050431C5C8C4202BF18184678012E06D0A1
:1072600004480478521C641DA242F0DB002050BD8B
:10727000E4230020D40F002001480078704700BFAD
:10728000E42300202DE9F843DFF88C91804699F83B
:107290000000002140F048FC98F800100446012945
:1072A0001CBF002001F00EFB14B9002001F00AFB06
:1072B00004F14C060020B1684A787768D10641F69F
:1072C0004C551DD507F1680108808870C870087199
:1072D0004871C88008818872C872786740F0E4FA03
:1072E000B9682818FFF790FA28B140F0DDFA2D1898
:1072F000BD60B868206194F82900FDF73BF93AE0D9
:1073000007F1940108808870C87008714871C880BE
:1073100008818872C872C7F8A00040F0C5FAB96841
:107320002818FFF771FA28B140F0BEFA2D18BD6099
:10733000B8682061607DC1060BD5B868618B00EB31
:107340008100B86397F84000012802D1B86BC01DD6
:10735000B863E07F81060ED599F8000033F0F3FFA3
:1073600000281EBF00F1B0010878002803D08879FA
:1073700008B902228A7161687068284A8A61486087
:10738000B2685078C3065CBF1020886150788307CC
:1073900003D5886940F4002088615078430703D5FD
:1073A000886940F4000088611D4B187800281CBFD4
:1073B000507810F0030F03D0886940F48020886172
:1073C0000020B1683070087E10F0300F1CBF4046BE
:1073D00000F04CF91349C86948B10522D0210020BA
:1073E000FDF798FD0622D4210020FDF793FD0E49FC
:1073F0000A68206990607169B1F8030048B1B06E05
:1074000038B92269B1F8031049F6404000FB012267
:10741000B266BDE8F18300BFD50F002002000080F6
:10742000880E002078230020B023002038B500F01B
:107430004BF90F4801688847044640F035FA054685
:10744000FFF7BCFE68B10178802918BF402908D138
:1074500081682846FFF7D8F918B140F2014040F0A2
:107460005BFA04490A682046BDE83240104700BF75
:10747000501B0020541B0020FEB5C0B2FDF768FD74
:10748000124A92E83800694681E838008069104D58
:1074900020F0004002906FF0010495F90000A04236
:1074A00018BF00F011F90B4B0B481E68006856F826
:1074B0002C7F00226946B847A042287005D1902051
:1074C00040F0FEFA002001F0FDF9F7BD4C80040009
:1074D00075110020200F00201C0F00202DE9F04125
:1074E000394E0546B078FDF729FD0446B078FDF722
:1074F0002FFD07462068D0F80480287880281EBF1A
:107500004028002001F0DEF9304800210170417070
:107510008170C170017141718171C17101724172DB
:107520008172C17201734173C173016180228273E0
:10753000707802280EDBD8F80800B9690818A0F5A1
:10754000965060F31E01B961A0797178884238BF06
:10755000FFF792FF002C1EBF1D4EF069002830D0AF
:107560001C490868A1792C235943425C012A18D18F
:10757000A96941F42031A9610522A47913FB04F320
:107580001844D021C069FDF7C5FC0622D42106F1BC
:107590001000FDF7BFFC0020012186F82000F174E7
:1075A0000FE0A86920F42030A8610522D021002036
:1075B000FDF7B0FCBDE8F0410622D4210020FDF724
:1075C000A9BCBDE8F08100BF780E0020980C002017
:1075D000782300207423002038B500F075F8204887
:1075E000017805291DD0112938D11E4D2878002198
:1075F00040F09AFA04001CBF616D00292ED0E07A99
:107600000028087E08D1C10628D52946002040F070
:1076100077FB0120E07231BD81061FD5294602208B
:1076200016E0114C2068017E19B1022914D00DD347
:1076300031BD026A51880A204143202040F0F0FB0E
:107640002168012008760021082001E000210B209C
:10765000BDE8344040F054BB0121017631BD00BF8C
:10766000C80F0020D50F0020500F0020FEB5124A91
:1076700092E83800694681E8380046680F4DB068E6
:1076800002906FF0010495F90000A04218BF00F0CD
:107690001BF80B4B0B481E68006856F82C7F002225
:1076A0006946B847A042287005D1902040F008FAFA
:1076B000002001F007F9F7BD588004007511002083
:1076C000200F00201C0F002070B5084C94F900100A
:1076D0006FF00105A94207D0054B064A1E681068E5
:1076E00056F8342F9047257070BD00BF75110020EB
:1076F000200F00201C0F0020F8B58AB0044602A815
:10770000324920223FF060FB1CB9002001F0DAF87A
:107710005AE02F4D2F48304E304A446000212B68EC
:10772000306853F8487FB8476168087B00F00F0065
:1077300002280CBF886840F0B7F86169A06009B101
:10774000204688476068008833F0EBFD08902449A4
:10775000087D78B1487D022818BF01280AD16068E9
:10776000008833F0EEFD28B101788DF824104078C0
:107770008DF8250061688868FBF7FEF8A069002194
:1077800041F0E243CDE9000361682C68306854F8A9
:107790005C5F144B02AA6FF00106A847124C6FF011
:1077A0000205B04218BFA842208006D1012033F064
:1077B000BFFDB4F90000B04203D0B4F90010A942F3
:1077C00002D1012033F0B4FD0BB0F0BD2C800400D9
:1077D000200F0020E42300201C0F00202C1100208B
:1077E000BC230020F9B20300880F0020F8B505463D
:1077F0000E4640F0DDF8144F04463868C08840F06B
:1078000067F808B91420F2BD3A684088117861B170
:10781000F9F7A6FF01460622284601F090F840F04D
:1078200037F800B10120A8710BE0F9F799FF014684
:107830000622304601F083F840F02AF800B101201A
:10784000B0712046F2BD00BF740F0020F8B50246AB
:10785000042AD8BF04291CDC104C2568EE783707B1
:107860000AD5042818BF012806D1042918BF012908
:1078700002D1062028710EE0094801EB8103C118EE
:107880008A5C2A7100F00EF828B12068017901297C
:1078900001D11820F2BD0020F2BD00BF740F0020FE
:1078A000A860021001480078704700BFF023002054
:1078B00001480078704700BFB8110020F8B50446B1
:1078C000104A206F05685169B4F87A314978EA881E
:1078D000C918891D8A4213DA002606602F46B86847
:1078E00020B1B86801F038FCBE60FE803F68AF424E
:1078F000F5D1206F05602046BDE8F24040F074BA33
:10790000F1BD00BFB07F04002DE9F047FDF716FB85
:10791000294D2A68116819B10267FFF7CFFF48E0C7
:107920000024264E264F4FF00C088146396808FB8C
:1079300004FA514400200871022238685044641C43
:10794000427172693868B9F87A31527800EB0A01ED
:107950009A18921DCA80631004EB93729310A4EBE3
:10796000830208FB02F2104408607069B9F87A11CA
:1079700040780818001D80B240F03EF8396801F1E7
:10798000080242F80A00386800F10801514408680A
:1079900010B10868801E0860042CC7DB28683968AD
:1079A000016000202A68506029683A688A60296866
:1079B000C8602868BDE8F087A00E0020B07F0400F2
:1079C000A80E00202DE9F043044685B0084611F8C2
:1079D00001CBDFF8A883DFF8A8332C22BCF1030F1A
:1079E0004FF0000904F5A47704F1660504F1F406EC
:1079F00000F0C380BCF1070F00F08381BCF10F0FD2
:107A00000CD0BCF1110F00F02781BCF11A0F00F06F
:107A10003981BCF11B0F00F0648191E1707A82071B
:107A200003D40F2184F8191159E008784A7800EB43
:107A300002233B808878CA7800EB02237B80087998
:107A40004A7900EB0223BB808879CA7900EB0223D4
:107A5000FB80087A38724A7A887A02EB00237B81AD
:107A6000C87A0A7B00EB0223BB81487B8A7B00EB50
:107A70000223FB81C87B0A7C00EB02233B82487C0B
:107A80008A7C00EB02237B82C87C0A7D00EB022308
:107A9000BB82487D897D00EB0122BA48FA820178D9
:107AA0008A0658BF4FF01A0913D504F5AA7004903E
:107AB00079890391387A029021890191F8880090A0
:107AC000BB887A88398820463FF0FAFEC8B14FF06B
:107AD0001E09707A410706D40F2084F81901204648
:107AE00040F0F2F8F3E04A460F2120463FF094FFC1
:107AF000F8880090BB887A88A1794846F9F794FD08
:107B0000ECE004F1860079888180BA88C280022284
:107B1000F98801810270A0F80290A18EC91DE98345
:107B2000628E8188B1EB520F02BFC188A28E914252
:107B300002BF0089E18EB0EB111F1CD0287C012808
:107B400004BF687C0F2809D0687D00281CBF687CB2
:107B50001A2803D00F21A976FE2179E0FC212046C6
:107B600040F04EF9F8880090BB887A883988A0796F
:107B70003FF0A2FFB2E010216AE0707AC20709D498
:107B800031781A200129707002D1FF220D213BE0CB
:107B90000D215DE085F8009085F806900123337192
:107BA000082204F1B0003FF017FF0146022204F161
:107BB000B8003FF011FF04F1A80801460822404632
:107BC0003FF00AFF07460821404640F0F5F804F16F
:107BD0009C080422394640463FF0FEFE0421404600
:107BE00040F0EAF804F1A0003FF04EFE04F19800E6
:107BF0003FF03AFE6448018841F08001018030780E
:107C0000012805D1FF22042120463FF02DFF65E029
:107C10006E7C0F2E18BF142E07D00E2E18BF0C2E00
:107C200003D01A2E18BF162E11D12F7C20463FF0FC
:107C30003FFE0421204640F0E3F8012F05D11A2E23
:107C4000AE7614BFFD21FB2102E0314600E00421A5
:107C5000204640F0D5F841E00E783E761A2E49785D
:107C600079766DD11868A679411C564301F80690C3
:107C70001968A37912FB03F20A4482F80490A179EF
:107C8000787E56E0A77918680E785743074406F0C7
:107C90001F0117F8210FB60938B17878F040C007F6
:107CA00003D594F89601042805D120221A212046F4
:107CB0003FF0B2FE12E0F970A179186812FB01F2F0
:107CC0008118204681F82360002133F024FB28B975
:107CD00098F800004FF4804101F000F84FF00109DE
:107CE00032E0A179186851430144C88808B981F885
:107CF0000190A179186812FB01F2811881F80490B3
:107D0000ECE709780F2917D01A2919D1A179186839
:107D1000514301441A2081F80190A1791B6812FB9C
:107D200001F2991881F80490F17A01F0FB01F172E7
:107D3000A17933F0F4FAD1E7717A01F0FD017172A3
:107D4000014620463FF064FF687C1A2812D1A87CC7
:107D500017281CBF1028FC280CD12E7C20463FF091
:107D6000A7FD012E03BF1A20A876FB211A21204669
:107D700040F046F8484605B0BDE8F083C70F002044
:107D800074230020200E00209C0F00201CB5114CF5
:107D90000346E079042818BF002B0A4616D01F2A94
:107DA000A8BF1F22694601203FF07AFF00B100788A
:107DB000E17988420AD0012918BF032902D110F0C5
:107DC000030F03D1022903D1C00701D5012016BD3D
:107DD000002016BD2002002070B5002408380528B8
:107DE000264D4AD8DFE800F00F150306090C4FF4C2
:107DF000001039E04FF4801036E04FF4002033E0FB
:107E00004FF4802030E02868C10336D54FF480302D
:107E10002AE01B4C206880B31A49086808B13FF07B
:107E2000A7FE02203FF084FF2068174E01F044FBBC
:107E3000306801F041FB0020206030602A68900328
:107E40001BD51249087801F027FB040008D010491F
:107E5000104B0A7822704FF40030597A617003E0B9
:107E60003FF0BAFF4FF000400B490B682BB10B49B4
:107E70000A682146BDE87040184770BD1002002016
:107E8000D40E0020D00E0020D80E00206C0200205E
:107E9000AD0F002020020020E40E0020E00E0020A4
:107EA00070B50D460446287A4107164604D530467B
:107EB0003FF0B2FF012205E0410609D530463FF010
:107EC000ABFF002201462046BDE870403FF028BECF
:107ED000C10617D530463FF09FFF014601222046DC
:107EE0003FF01EFE60B930463FF082FD030005D032
:107EF00029462046BDE870400A2218470E2070BD72
:107F0000082070BDC00701D4022070BD002070BDE4
:107F1000F8B50E460546307A810617461C461DD533
:107F200038463FF079FF0146012228463FF0F8FD30
:107F300030B1607A10B1207A012801D00820F2BD5A
:107F400038463FF055FD030006D03146284601B0C3
:107F5000BDE8F040122218470E20F2BD010609D5F7
:107F600038463FF059FF01462846BDE8F840002258
:107F70003FF0D6BD01070FD538463FF04DFF014613
:107F8000012228463FF0CCFD010009D0617A41B1C1
:107F9000217A012904D0F2BD800701D40320F2BD6B
:107FA0000020F2BD1CB504460846694600883FF033
:107FB0006FFD010001D1012016BDBDF80020204653
:107FC000FFF76EFF16BD7CB506460D46002409E09E
:107FD000BDF8002001463046FFF762FF01001DD1C9
:107FE000641CA4B2A888844222DA286810F81420FD
:107FF000401C694610F8143002EB032290B23FF0A7
:1080000047FD0028E4D1286810F814100170286892
:10801000421C12F814104170012076BD296811F835
:1080200014200A7029684B1C13F814204A7076BD7E
:10803000002076BD38B504460D46694628883FF0D5
:1080400027FD08B9012032BDBDF8002001462B46AE
:108050002046FFF75DFF32BD2DE9F84F0120FFF705
:10806000B5F8012816D1DFF89866307800213FF086
:108070005BFD040004BF002000F024FC00202072FF
:10808000201DFFF74BF8FCF761FB050003D18120B1
:108090003FF016FD30E301206871DFF86826DFF855
:1080A00068064178491C4170A879A0724020317857
:1080B0001170FEF7D5FF2860616D4A78206DD106FA
:1080C00020D5816C0A681179032908D0816C086871
:1080D000007903280CBF0120002000F0F3FB206D85
:1080E000816C0A6890F86C0002F1080701281CBF37
:1080F000002000F0E7FB216D486F296800F5B060B3
:10810000C8604AE0C16E0A681179032908D0C16EBF
:108110000868007903280CBF0120002000F0D2FB82
:10812000206DC16E0A6890F8980002F108070128D6
:108130001CBF002000F0C6FB226DB5F87401D2F818
:10814000A0102A68DFF8C435DFF8C465D16097F85D
:108150002690B9F1030F1BD8DFE809F002050E11D4
:1081600001F5B06101E001F53471D16005F59A7156
:108170001888088718880EE001F5355101E001F6EE
:10818000B871D16005F59A7130880887308802E0AF
:1081900001F5B061D160A5F8740106222868DFF806
:1081A0007465C168DFF8708501F59071C160B91C14
:1081B0003878C0F3801085F82E0105F5947000F032
:1081C000BEFB042207F10E0105F1240000F0B7FB0D
:1081D000306895F8069000F10C03042207F10E01B7
:1081E00003EB491000F0ABFB3068AB7900EB4313B5
:1081F000032207F1120103F1100000F0A0FB05F1CA
:108200002C09787D89F80200022207F1160105F198
:10821000300000F094FB022207F1180105F1320052
:1082200000F08DFB022207F11A0105F1340000F085
:1082300086FBB9F808006884022207F11C0105F1E9
:10824000360000F07CFB99F80200B9F80A104000F3
:1082500089F802000901B9F80400A9F80A104000E1
:10826000A9F8040089B2B9F806004000A9F8060090
:1082700003046A8C521CDB0B5A438A4201D280B23F
:1082800030B998F80000802100F028FD3B2133E14F
:1082900005F12E0128463FF097FD0520A8814FF0FB
:1082A0001C0A28463FF024FC052207F11E0105F1B7
:1082B000610000F044FB97F82300400989F80000B2
:1082C0003FF06EFB688205F59A72618D401AD0808E
:1082D00005F1610197F82300DFF8407400F01F00FA
:1082E00089F80F0028463FF027FB616D4A78206D22
:1082F000D1064CBF816CC16E41F621020868002195
:108300000171A97938681AFB01F142520021AB7959
:108310001AFB03F303445980AA791AFB02F21044B2
:108320004160616DDFF8F8034A78D1060DD5DFF8BA
:10833000F4138A7851060AD5DFF8EC23138841F24A
:108340000A418B4208BFDFF8E403C5F89C01D5F869
:108350009C11284688473A68A97902F10E031AFB56
:1083600001F15854AA7938681AFB02F2024400203D
:10837000D0733968A87901F10E021AFB00F0115C84
:1083800089F80D10606D4178CA061DD595F89601E3
:1083900008B900F097FAA97938681AFB01F101448D
:1083A00095F89601421E0A74A87939681AFB00F004
:1083B0000844002141743A68A97902F112001AFBBD
:1083C00001F1002242522BE0A97938681AFB01F131
:1083D0000144206D90F840200A74A87939681AFB8E
:1083E00000F00844216D91F841204274206D3968F5
:1083F000AB79403001F112021AFB03F34188D152EC
:1084000005F5CB710078012200F0030082400A706C
:10841000226D92F84000800814BF012002200871EC
:108420003968A879DFF808B301F1140231681AFB42
:1084300000F301EB4010D050A87939681AFB00F026
:108440000844BC498161DBF814000078C107DBF8FF
:10845000141009784CBF1F200F208A07DBF8141076
:10846000097848BF40F020004A07DBF8141009786B
:1084700048BF40F040000A073168AA7901EB421377
:1084800048BF40F080001872A979306800EB4112B3
:108490000B2050723168AA7901EB42100421A64AE0
:1084A00081721078012806D13168A87901EB401259
:1084B0000121D17207E0DBF824003168AA79407805
:1084C00001EB4213D8723168A87901EB40121F21E9
:1084D00011763068AA7900EB421100204876A8791D
:1084E000FFF712FAAA79316852018850AA793168E7
:1084F0005201885820B907212846FCF7A7FBFBE06A
:108500008E48AA79016801EB02103FF045FCA8797A
:1085100031688A4B01EB4012196801EB0010506082
:10852000A979306800EB41125168C9F83C10AA796A
:1085300052018158C9F84410042198F8000000F055
:10854000CDFB616D4A783868D10648BF02210AD454
:10855000A9791AFB01F101440A7C02F00302022A04
:1085600014BF04210621B9F8042095F806C04FF481
:10857000C8738A18698AAA615143B1FBF3F35B1C83
:108580006B611AFB0CFCD5F800E06044DEF80CC00F
:1085900040F6C41101FB02C2D21AA2F5A8628260A1
:1085A000AA7938681AFB02F283189A682B689A60D5
:1085B00000F10C03AA791AFB02F20C309B5C03F069
:1085C000EF038354A8793A681AFB00F002F10C0318
:1085D0000C321B5C03F07F031354A8793A681AFB32
:1085E00000F002F10C030C321B5C03F0F00343F0CB
:1085F00002031354AB7938681AFB03F31844427B27
:1086000002F0F00242F001024273AA7938681AFBC4
:1086100002F2024490682B6818613068AB7999F8CF
:1086200002C000F11402686940005B0111FB0C00FC
:1086300000F5F660D05095F8960104280DD1306809
:10864000AA7900F114034FEA421C143053F80C20AD
:10865000AB795B0102F56162C2503068AA7900F122
:1086600014034FEA421C53F80C20C5F83421AA79B0
:1086700000EB4210C37C03F0F00343F00403C37427
:10868000DBF830003268AB79006802EB431CB9F8C4
:10869000062042436423B2FBF3F35943A1F59661EC
:1086A000CCF81C103068A97900EB4110C27E02F0B2
:1086B000F00242F00402C276A97938682A681AFBEF
:1086C00001FA00EB0A01516028460E213FF098FBA9
:1086D0001B49072008702046FBF754FE1948817893
:1086E000880704D5AA79002120463FF049FA286876
:1086F0001549164A41618261BDE8F14F32F004BE6E
:10870000D50F0020D70F0020780E00208E0F0020FC
:10871000900F00209C0E0020C70F0020980E002014
:1087200081010210C00C00209A0F00204DE50110BD
:10873000B07F0400980C0020CC0F0020A40E002075
:10874000C80F0020200E0020DD740000020480808D
:10875000F8B5054617461C463FF02EFA02260228B9
:1087600001D11220F2BD042F1EDA012F18BF032FF2
:1087700002D1CCB1012F01D0032F17D10522002146
:10878000204600F0B4FC18B1607910F03F0F0BD018
:108790000622FF21204600F0AAFC002802BF6079D3
:1087A00000F0C000C02801D00220F2BD6D1E032DD4
:1087B00006D96D1F04D0AD1E012D01D92D1F00D18A
:1087C00000263046F2BD10B5044614F00C0F04D05C
:1087D0003FF01EF900213FF073FA3FF079F93FF0C6
:1087E000BFF814F00A0F07D03FF0AEFA200703D508
:1087F0003FF07AFA3FF088FA14F0050F09D03FF005
:10880000F7F9600705D53FF067FABDE810403FF083
:10881000A3B910BD2DE9F84384B004460D46904637
:108820009946FFF795FF070026D1154E86F8008080
:10883000B8F1010F12BFB8F1030F4846F9F782FCF7
:108840001048114905700D7020463FF0D1FA07001D
:1088500012D16846002100220023002580E82E0066
:108860003078002818BF012803D1694600203FF066
:1088700013F82046FFF7A7FF384605B0BDE8F083A0
:10888000A90F0020BA110020B911002003460022D0
:10889000002100203FF0DCB8F9F772BFF9F788BF7C
:1088A000F9F7BCBF0200034A117008BF0248034930
:1088B00008607047C0110020F1880000BC11002042
:1088C0007047000080B5010002BF06490A78012AFE
:1088D00004D00549054A097813689847BDE8014066
:1088E000FFF7EEBFC0110020F1230020BC110020D3
:1088F0007047000010B50C460168084A11604368D3
:108900000749084A0B608068106000F06BFF32F086
:10891000CBFC2046BDE8104032F0B6BB4C1B00201B
:10892000501B0020541B002080B5022168463FF0F8
:10893000FBF9BDF8000002BD704702F054B803E037
:1089400011F8013B00F8013B13465A1E002BF7D1EA
:10895000704711444B1E03E013F8011900F8011B86
:1089600011464A1E0029F7D1704770B505460E46DC
:10897000B0B200F091FD040003D032462946FFF763
:10898000DEFF204670BD10B513465A1E3BB110F8ED
:10899000013B11F8014BA342F6D0002010BD01208D
:1089A00010BD10B5044610460A460146204601F0A7
:1089B000C3FF204610BD02460229107803D151782A
:1089C00000EB01207047032906D15178927800EB23
:1089D000012000EB02407047042908D151789378B8
:1089E00000EB0120D17800EB034000EB0160704701
:1089F000FFF79ABF10B5034A034C13692278801819
:108A0000195410BDC41100203800050010B5040031
:108A100001D1002010BD04F10C0080B200F03CFD3B
:108A200028B100210160FF22048182720C3010BD48
:108A300080B508B9052002BD10F8021CFF2901D03D
:108A4000042002BD0C3800F037FD002002BD0000FC
:108A50002DE9F04104460E46904600F057FB46498A
:108A6000FF2808BF4F7804D0444A13780969C0181A
:108A70000F5C434DFF2F04D1286850F8081F88472A
:108A800013E0304600F052F80146FF2008F8020CCF
:108A900022002E680CD156F83C4F4346002238463F
:108AA000A04770B14046FFF7C3FF0120BDE8F08149
:108AB000012CF7D13468434600223846A0470028ED
:108AC000F0D10020F2E770B50C00064615461AD02A
:108AD000300604D52A490A6852F8080F804727490A
:108AE0000A78964204D32046FFF7A2FF032070BD08
:108AF000A4F10C010868002804BF887AFF2804D07C
:108B00002046FFF795FF052070BD8E72012D1D4890
:108B1000214602D100F0B0F801E000F08FF84FF4E8
:108B20000041304600F0DAF8002070BD10B580F04A
:108B30008004042C04DB1248016851F8082F904788
:108B40000D482044007910BD38B504460E48016830
:108B50008847094A0546D068844206D1084A0B492D
:108B60001368086853F8241F88472846BDE8324038
:108B7000074A136818470000C41100203800050098
:108B800030900020F4230020501B002000240020FF
:108B9000541B002080B5020606D50A460146012076
:108BA000FFF756FFC0B202BDBDE808400022FFF744
:108BB0008ABF80B50A46010605D501460020FFF7A9
:108BC00047FFC0B202BD012002BD00002DE9F04107
:108BD00005461748174F01688847804638680026C1
:108BE000002405E014B9064600E0044650F80C0CD9
:108BF00058B110F8021CA942F4D1002CF5D04FF462
:108C00000041284600F06AF805E04FF4004128468C
:108C100000F0CAF824B132462146384600F040F848
:108C200005490A68404690472046BDE8F08100BFEC
:108C3000501B0020F4230020541B002038B50446AC
:108C40000B480D4601688847002245F80C2C226825
:108C500012B9256006E00A4652F80C1C0029FAD128
:108C600042F80C5C03490A68BDE83240104700BF77
:108C7000501B0020541B002038B5044606480D4602
:108C8000016888472268054945F80C2C25600B6867
:108C9000BDE83240184700BF501B0020541B002085
:108CA00070B504460B480E46016815468847A6F184
:108CB0000C0123680A689E420CBF226045F80C2C08
:108CC0000022FF230A608B72BDE8704002490A68E7
:108CD000104700BF501B0020541B00202DE9F0411D
:108CE00080462A482A4D06780F465FEA086132D549
:108CF0000420FFF78BFE040008BF042043D04FF68A
:108D0000FF702080678000F001FA2249FF280FBF22
:108D10004E78096980190E5CFF2EA4F10C0707D16B
:108D20002046FFF785FE286850F8081F884710E0A6
:108D30004046FFF7FBFEFF21B97201462D68D5F8CA
:108D40000080234600223046C047E0B12046FFF7AE
:108D50006FFE012017E0B04514D20F480168884724
:108D60000E4A116831F818301F4321F818700C4969
:108D70000A68904729680B4851F8242F00689047EB
:108D8000002000E00320BDE8F08100BF38000500AE
:108D900030900020C4110020501B00207052012090
:108DA000541B00200024002038B50D460B490A78DA
:108DB000904204460FD20A4801688847094A116860
:108DC00031F8143023EA050521F8145006490A68E1
:108DD0009047002032BD032032BD00BF380005009F
:108DE000501B002070520120541B002038B50F4941
:108DF0000F4D0020086000F087FB00F065FB0D4878
:108E00000478600000F048FB28616200FF21FFF752
:108E1000C8FD0422FF21281DFFF7C3FD32F0F4F83E
:108E200005480168891E0160002032BDF42300203E
:108E3000C4110020380005000C240020024A1060F4
:108E400002480160704700BF082400200C24002065
:108E500070B50C4C0C482568C26855F8106F0B496A
:108E600000F108030120B04718B1206850F8081F2E
:108E7000884700F043F8216851F8142F4FF0FF3075
:108E80009047F6E730900020C4110020498B000085
:108E900080B5014600200B4A02441379FF2B0BD00A
:108EA0008B420AD0401C0428F5D30748016851F8CA
:108EB000082F9047FF2002BD117140F08000C0B222
:108EC00002BD00BFC41100203090002010B5044640
:108ED000608850B9A079FFF7DBFFFF28E07102D16D
:108EE0006FF0030010BD002010BD6FF0010010BD39
:108EF00001490860704700BFFC2300202DE9FE4FA8
:108F000000F05EFC00255FEA000903D000F040FBA2
:108F10004FF0FF396348006828B1804703E03068AC
:108F200050F8081F8847604EDFF88081336853F897
:108F30001C7F01AA69460DF10100B84700285C4F6B
:108F40002FD10198A0F10C07B979032906D159480E
:108F500001680029E7D001988847E4E79DF8000000
:108F6000002400E0641C54490A789442D7D2D8F80F
:108F700010100A5D8242F5D1E0B2FF28CFD03879D7
:108F8000FFF786FFB979012902D10199087003E042
:108F9000022904BF019988700199E0B2FFF7FAFD38
:108FA000C1E73968EAB231F8120028B942480278BC
:108FB0006D1CE9B29142F4D33F49404C0878DFF888
:108FC00000A18DF80000E9B2814226D2DAF8001043
:108FD000884739685FFA85FB31F81B20ADF802201D
:108FE000002321F81B3021688847364ABDF802105B
:108FF00088F80050E8B252F82B3098470546FF2019
:1090000088F80000DAF800108847396831F81B202A
:10901000154321F81B502168884700F0D1FB054615
:109020004D4520D005B9284D28480068DAF80010D1
:10903000A84238BF05468847316851F8202F81463D
:10904000D8F808009047D8F80C202149521CC8F8DD
:109050000C202846356855F80CCF08F10803E04786
:109060002168484688471B4A1B4C106828B1316864
:10907000206851F8242F904711E000250AE0396854
:10908000EAB231F8120020B13168206851F8242F7B
:1090900090476D1C9DF80010E8B28842EFD3BDE800
:1090A000F78F00BFF823002030900020C41100206B
:1090B00070520120FC23002038000500541B0020C2
:1090C000501B0020140005008EC2F5280C2400203F
:1090D000498B0000F42300200024002001700A0ABC
:1090E0000B0C090E42708370C170001D704710B5E3
:1090F00040B1002300E05B1CDCB2944204D2045D6A
:109100008C42F8D0002010BD012010BD014800782D
:10911000704700BFC411002070B505460B480168B8
:109120008847064605F1080080B200F0B5F9040052
:1091300005D00748A5800168216004600834054A0D
:10914000116830468847204670BD00BF501B002084
:1091500010240020541B002070B5044610480168FC
:109160008847104A05461068002101E00146006862
:1091700080B100F108039C4221BF00F108068388FA
:10918000F318A342F2D3036800290CBF13600B60ED
:1091900000F092F92846BDE8704003490A6810477C
:1091A000501B002010240020541B002038B504461A
:1091B0000D4600F011F868B16D42611900F1080325
:1091C000994221BF00F1080580882818884201D300
:1091D000084632BD204632BD38B505460B48016809
:1091E00088470B4A146800E024684CB104F1080178
:1091F0008D4221BF04F10802A1885118A942F3D37E
:10920000044A13689847204632BD00BF501B002017
:1092100010240020541B002005490A88FF2A05D18C
:109220000880782200210348FFF7BBBB704700BFCE
:10923000D8110020142400202DE9F04104460D46E9
:10924000280448BF85F4004030D428002DD01848A9
:10925000016888472E468046002725FA07F0C00798
:1092600008D47F1C0F2FF8DB12490A68404690474C
:10927000B0B21BE01049114B0A88121BC2EB02125C
:10928000BA1803EBC206012101FA07F7316809B1E8
:1092900070688847B9B2204600F00AFA10B9306009
:1092A0000021716087EA0506DEE70020BDE8F08155
:1092B000501B0020541B0020D81100201424002033
:1092C0001CB50024009400F073F816BD2DE9F0479A
:1092D00006461848184D8A46016888470F2E814671
:1092E00021DA164951F83600E8B10F21144F96FBE8
:1092F000F1F8C8EB08140120341B00FA04F4388894
:109300004044A1B2C0B200F0D3F960B138888044C3
:109310005246A1B25FFA88F000F06EF9296848461B
:109320008847002003E02968484688470220BDE8B6
:10933000F08700BF501B0020541B00201424002085
:10934000D8110020F8B504461548164E0168884724
:109350000F2C05461EDA144F57F83400D0B10F21F8
:1093600094FBF1F0C0EB001C0123A4EB0C018B403B
:1093700099B20E4B1A881018C0B200F07DF9002087
:1093800007EBC40247F8340050602846336898471A
:109390000020F2BD3168284688470220F2BD00BF98
:1093A000501B0020541B002014240020D811002042
:1093B0002DE9F34F81462148214E016881B0904646
:1093C0001D4688475FEA090203D1316888470220B9
:1093D00025E01C49DFF870B0009100270C9C824604
:1093E0005BF83700A0B9012C0CBF184B184B0F20AD
:1093F00097FBF0FCCCEB0C1E0121A7EB0E0081408B
:10940000009800886044424689B2C0B2984740B193
:109410007F1C0F2FE4DB3168504688470820BDE8E9
:10942000FE8F02994BF837900BEBC7025046516004
:1094300005B12F70316888470020F0E7501B0020ED
:10944000541B0020D8110020142400203D96000059
:10945000F9950000006808B90120704700207047A6
:10946000006870470068704700220A6043684B60DC
:109470004268002A14BF11600160416070470A68A9
:109480004B68002A0CBF436053604A6809680AB9F8
:10949000016070471160704702490A6852F8343F12
:1094A000184700BF3090002002490A6852F8443F34
:1094B000184700BF3090002002490A6852F8383F30
:1094C000184700BF309000200349044B002008805B
:1094D00001221A70704700BF8C2400208E240020C7
:1094E00038B5074D074CA96920463C223DF06CFC7D
:1094F00020462EF0B1FA2168BDE83440002008472C
:109500006CFE04009024002080B50549054A002027
:109510000860136853F8180F80470349086001BDBD
:10952000D424002030900020D024002070B50446C0
:109530000D46164600F01AF808B1466070BD1020BE
:10954000FFF7AAFF78B184720581466000210160AF
:10955000C16005490A6812B9086070BD0A46116801
:109560000029FBD1106070BDCC24002020B502463C
:109570000448006828B103898B4204BF857A95426C
:10958000F7D120BDCC24002008B100210181704713
:109590002DE9F8451548164D016851F8182F9047E8
:1095A0002E6807461348D0F80080BC1BB8F57A7FB8
:1095B00015D0A8FB04014FF47A72002301F040F8A3
:1095C0003746044606460A464FF47A7AAAFB060155
:1095D0000AFB02114246002301F032F8C7192F603E
:1095E0002046BDE8F24500F0FFB800BF30900020F3
:1095F000D024002008240020F8B50D460C4904466C
:109600000868164608B9FFF7C3FF0A48016888478B
:109610000746324629462046FFF788FF06490A6872
:109620000446384690470CB10020F2BD0820F2BD38
:10963000CC240020501B0020541B0020F8B5044609
:109640000B480D46016816468847074632462946AC
:109650002046FFF76BFF0400064918BFE6600A6862
:10966000384690470CB10020F2BD0820F2BD00BF83
:10967000501B0020541B002070B504460A480D46BC
:1096800001688847064629462046FFF76FFF040019
:1096900018BFFFF779FF05490A68304690470CB1BB
:1096A000002070BD062070BD501B0020541B002000
:1096B000F8B5054608480E46016888470746314612
:1096C0002846FFF753FF002400B1446803490A68A5
:1096D000384690472046F2BD501B0020541B002006
:1096E0002DE9FC47324FDFF8CC80DFF8CC90044600
:1096F0003868804731490A68A2180A60D8F8001013
:109700008847D9F80050002D42D0002600943868D0
:1097100080478246BDF802000024002804BF9DF85F
:109720000100002807D128799DF80010884202D353
:10973000401A287106E06868009981423ABF401AD1
:1097400068606C60A88860B9E88860B9E86800283B
:109750001CBF298900290AD0A87AFFF7BFFAE86858
:109760006860A88808B9E88808B1288938B92868E5
:10977000002E0CBFC9F8000030602C4600E02E46D9
:109780002D68D8F80010504688471CB9002DBED16E
:10979000BDE8F387A088002804BFE088002803D133
:1097A0002189A07AFFF79AFA2046FFF785FEEDE7B8
:1097B000501B0020541B0020CC240020D424002067
:1097C0000648016841B106484A680968824298BF64
:1097D00010460029F8D1704700207047CC240020A3
:1097E0008EC2F5287047000070B504460E48016827
:1097F00088470E4A1368E318B3F57A7F0BD30C49F8
:109800000E684FF47A75B3FBF5F5AE190E604FF4A0
:109810007A7101FB15331360064A13689847204696
:10982000BDE87040FFF75CBF501B0020D82400202B
:10983000DC240020541B00201CB501240246032A0E
:10984000084613D0832A08D042F219018A4214D064
:109850004FF6FF718A420CD014E0428900920389CE
:10986000C2888188C078F6F7F5FC0CE03EF09CFADF
:1098700009E03EF045F9044605E0807818B13EF075
:10988000E3F800E00024204616BD1CB50124024682
:10989000032A08460ED0832A13D042F213018A42CB
:1098A00004D04FF6FF718A4207D013E0807800F0B1
:1098B00014F810E000F01AF80DE03EF061F80446EC
:1098C00009E0418900910389C2888188C078F6F750
:1098D000C1FC00E00024204616BD0C281CBF112846
:1098E0001A2801D13EF024B9704700007CB5044627
:1098F0000121E078134E1A284FF6FF7506D1A08893
:109900003288904205D13EF013F90146E0781A28DA
:1099100008D1A0883288904218BFE07808D10800AA
:109920000FD006E0302801BFA28833889A423580E4
:1099300039B13580618900912389E288A1883EF0A0
:10994000AFF873BD580200202DE9F84F0422FF2123
:109950006846FFF726F8DFF88C63B0780024FF280C
:1099600000F0BE81FBF7EAFA0546B078FBF7F0FAA3
:10997000064605F217100178012908BF417800F06A
:10998000008105F1740005F5927A817B022904BFFC
:1099900005F174018C7395F89201022805F17400A9
:1099A00008BF85F89241017F022904BF05F17401C7
:1099B0000C77BAF80E1019B19AF80C00FFF78EF96F
:1099C0006889C94F288105F58D7BBA7AF879397B8A
:1099D00080184118F87A0818797B00EB0109BBF868
:1099E0000400BBF80010401CABF804004944BBF86D
:1099F0000200ABF800101018ABF80200DAF8000013
:109A0000F0B1BA4995F806E00B681C2103F10E0C81
:109A100011FB0EFE0E331CF80E1030F811C0CC44B2
:109A200020F811C01C2195F806C011FB0CFC13F89E
:109A30000C3000EB4300B0F84A105218A0F84A204E
:109A4000FDF742FEF879002804BFF87A002805D116
:109A5000387B002804BF787B002840D0F481A046E2
:109A6000F07EC00910D0307F00F00701022907DA2C
:109A700000F0F802401C00F007001043307703E0CC
:109A8000A879002131F056FC2989E8892C74411805
:109A9000287FA981012804BF688CE883A979012265
:109AA000072031F03DFC787805F1740658B10121AA
:109AB0002977B078002804BFB07B002803D1307F1D
:109AC00008B9688CE8839AF81400002862D002284C
:109AD00004BFF87A002858D18AF814405AE0A979CE
:109AE0000022072031F01CFCEC83317F11F0070FBE
:109AF00002D1F07EC00903D0A879002131F01AFC10
:109B0000B87A38B1287F01284FF0010827D1688C36
:109B1000E88324E0BBF80600401CABF806004FF0D9
:109B20000208287CD8B172490868AB7995F82E6094
:109B300000F1140268694FEA400C40F6C4105B0162
:109B400010FB06CC0CF5F660D0500968A87901EB43
:109B50004010C17C01F0F00141F00401C174A889FA
:109B60002989814206D088429DD2081A41F2AB026F
:109B7000904298DA287C08B1052901D0082100E03C
:109B80003E212846FBF762F8AAE0787A10B102215C
:109B90008AF81410F87BC1070DD538692968C860A8
:109BA00000F59070C86052480168A87901F114026C
:109BB0004001145014E04E48AB79026802F11401E0
:109BC0005B01C858CAF810004848AB7901681C20EE
:109BD00001F108024343D0582968C860EC832C7710
:109BE000444A50690078810702D5B87B802800D1AB
:109BF00081203070404991F8200018B12946012099
:109C000031F084FB284600F0C5FA02281BD1F07918
:109C1000022805DB6A4639492846FAF7FFFC044664
:109C200028463DF089FF01285AD020000DD0224659
:109C300069462846FAF7C6FC38B9284600F0AAFA61
:109C4000012802D14CE001284AD0012128463EF0EB
:109C50008BF800F05BF8012842D0284631F05AFB1F
:109C600031F052FB264F3868002839D0B888AA79DD
:109C700090421CBF4FF6FD71884231D12148007BD4
:109C8000FFF712FC04002BD084F80080A8791E494D
:109C900060800A68A879115C217105F5C972107994
:109CA000607196F90010A171A4F80890BBF8020049
:109CB0006081FDF783FA050005D1FF204FF0FF31E9
:109CC0002073216109E0287820733DF0EDFD014605
:109CD000A8683DF06DFF80082061204639688847FC
:109CE000BDE8F18F780E0020980C0020980E00201F
:109CF0009C0E0020B07F040078230020DC1100209F
:109D0000800E002064110020B82300202DE9F84FB8
:109D1000DFF85854A9780024FF2904BF0020FEF77B
:109D2000D1FDA878FBF70AF9054605F1680605F5A7
:109D3000C9773168086805F1900808B1EC8311E033
:109D4000B07B002804BFB07E00280BD198F800102B
:109D5000002904BF3878002804D1287F012804BFD7
:109D6000688CE8832989E88B4118491C6981284659
:109D70003DF072FF01281EBFDFF8F40301780129CE
:109D800003D12989EC83491C69814FF6FF79B07EA4
:109D900001280DD1B28B698928893DF0ADFE38B11B
:109DA000298968894A1C93B298422FD0B08B23E04E
:109DB00098F8000001280FD1B8F802206989288995
:109DC0003DF09AFE40B1298968894A1C93B29842B5
:109DD0001CD0B8F802000FE03878012816D17A8834
:109DE000698928893DF088FE80B1298968894A1CE3
:109DF00093B298420AD0788892B2904206D04844F2
:109E0000688180B23DF0E4FE4844E8833878012858
:109E10000FD128897988401C80B2884209DB7C797F
:109E20003C71022038702346A97922460020F7F7BA
:109E300095FB05F59A71087920B128890021401C0D
:109E4000E9836881B07E012813D12989B08B4B1C2E
:109E50009BB298420DD168813DF0BAFE804605F173
:109E60002E008188308C01FB08082846FBF714F887
:109E700003E005F12E01B1F80480EA8BDFF8F492DB
:109E8000501C00FB08F040F6C41808FB00F10091DC
:109E90002B68D3F80CE07144D960B74B1968097886
:109EA0008909032940F0168199F80F30B349DB077F
:109EB00040F10081B5F812C000230CFB00FC4FF408
:109EC000C87EBCFBFEFC0CF1010C0B80A861C5F840
:109ED00014C085F820204FF01C0BDFF8A4A2AB794A
:109EE000DAF8000000F108021BFB03F3D1582A68DE
:109EF000116100F10801AB79D26868691BFB03F3BB
:109F0000121ACA50DAF80000AB7900F108021BFB04
:109F100003F3D1582A68916000F10C02A9791BFB68
:109F200001F10C30535C03F0F00343F0020343549F
:109F3000DAF80010AB798A1C1BFB03F30021D15225
:109F4000387908B9FEF7BEFCDAF80000AA7900F10A
:109F5000100138791BFB02F240088854A879DAF81E
:109F600000101BFB00F008440021417438790428DC
:109F700014D1A879DAF800101BFB00F001F11002EF
:109F80001031135C3A7A43EA82030B54AA79DAF867
:109F900000001BFB02F2024420205074DAF800108B
:109FA000A87901F112021BFB00F000211152754942
:109FB000A8790A6802F114034FEA401C143253F8DE
:109FC0000C00AB79D5F814C05B0100EB4C00D0500D
:109FD000B07E02280DD10A68AE7902F11403760131
:109FE00014329859AB7995F82E605B0118FB060086
:109FF000D05005F12E0299F80F00C30773D5DAF897
:10A000000000AE7900F108041BFB06F60830A359E6
:10A01000AC791BFB04F4A3F5A8630351DAF8000044
:10A02000AE7900F108041BFB06F6A3592C68A36067
:10A0300000981B1A23610868AE7900F114047601B8
:10A040001430A359AC79640103F5F66303513879F0
:10A0500004280BD10868AE7900F11404760114309D
:10A06000A359AC79640103F5616303510868AC79C5
:10A0700000F1140364011859C5F83401424B186B00
:10A080000C68AE799288006804EB4617424364245A
:10A09000B2FBF4F408FB04F0A0F59660F8613B48CD
:10A0A0000278012A48D10868A97900EB4112012001
:10A0B000D07248E00B885B1C1FFA83FCBCF1010FD7
:10A0C00011BFB5F812C005F59A7EBEF806C00CF2B5
:10A0D000DC5CF2E6698A41434FF4C873B1FBF3FCE0
:10A0E0000CF1010CF2E6042C0BD10868AE7900F1FA
:10A0F000140476011430A359AC79640103F561634B
:10A10000035138790B68AE7904280CBF4FF4AA507C
:10A110004FF4E66003F114047601A359181A9388EA
:10A1200008FB03F3A3F516739842A7D3082128462A
:10A13000FAF78CFD012016E0586A0968AA79407880
:10A1400001EB4213D872A879DAF800102A681BFBD9
:10A1500000FB01EB0B00506007210D480170284601
:10A16000FAF78CFA0020BDE8F28F00BF780E0020CD
:10A17000D10F0020980C00203C0F0020E02400208C
:10A18000980E00209C0E0020B07F0400CC0F002011
:10A19000C80F002070B504000AD10020FEF792FB22
:10A1A00006E0A97EFF2220463DF05EFC01202874D7
:10A1B00004F16605687D002841D0687C112823D011
:10A1C0001A2802D0FB28ECD039E0297C012912D1D1
:10A1D0001C48A27901682C235A438B18187930B394
:10A1E000288B401E288380B260B922212046FAF7CE
:10A1F0002DFD012070BD0121204631F08CF828741E
:10A20000E88A2883002070BD287C012813D10E4ED7
:10A21000B07848B1002184F89410012028702046BD
:10A220003DF08AFD0121A971F0780028D8D02046A0
:10A230003DF03EFBBCE720463DF05AFDDFE7022043
:10A2400070BD00BF74230020980C0020017A1029F3
:10A2500008DA054A11688B6E93F83310012901D191
:10A26000062070473DF0CCBC740F002070B50E4E38
:10A27000336804461022214603F11800FEF783FBE1
:10A28000002508B1082070BD306810222146383002
:10A29000FEF755FB3DF010FD00B1082531680520A3
:10A2A0004870284670BD00BF740F002070B5144D73
:10A2B00029680446886FD8B1124E202231462046C4
:10A2C000FEF761FB60B1202206F1200104F12000BD
:10A2D000FEF759FB20B1FDF7EBFA58B90A2070BD23
:10A2E0002868416F202220312046FEF74CFB08B140
:10A2F000082070BD2046BDE870403DF09DBC00BF09
:10A30000740F002078110020F8B588B007460D467C
:10A310001646102200216846FEF743FB374C2068A2
:10A32000002848D0C288BA4204BF0178002942D12F
:10A330004178062927D1C1780A0733D400F14802B1
:10A3400000F1280104AB08303DF04AFD002832D16D
:10A3500038463DF0BDFA04002DD0E06A18B91C2043
:10A36000FFF79AF8E062E06A28B33DF005FBE16A86
:10A37000887604A9E06A827E6846FEF7E0FAE06A21
:10A38000102269462DE0806DA8B1112913D1028AEF
:10A3900096420DD100F1120108222846FEF7F3FA89
:10A3A000012805D13DF0E8FA02462068816D17E0EA
:10A3B00032203DF049FB38463DF08AFA04001CBFCC
:10A3C000E06A002814D0018A8E4211D100F11201F6
:10A3D00008222846FEF7D7FA012809D1E16A8A7EC9
:10A3E0006846FEF7ACFA694638463DF0B5FA02E039
:10A3F00038463DF0C5FC012009B0F0BD740F0020C7
:10A4000038B50C4B1B688BB1DC884588AC4201D059
:10A41000082032BD1B78012B01D1072032BD0C2949
:10A4200004D1BDE83240104630F0C6BFBDE8384028
:10A430003DF06ABA740F0020017A102908DA054A43
:10A4400011688B6E93F83310012901D106207047F3
:10A450003DF0F2BC740F002038B504461348006884
:10A460004178132903D114214170002032BD1529F0
:10A470001AD1FDF71DFA80B90D4D2022294620463C
:10A48000FEF781FA48B1202205F1200104F12000F5
:10A49000FEF779FA08B10A2032BD20463DF020FAD5
:10A4A000BDE831403DF01CBC082032BD740F0020D7
:10A4B0007811002038B5012815461C4602D0022824
:10A4C00009D00DE0049B0A462146284601B0BDE8AC
:10A4D00030403DF039BB0846BDE832403DF01CBC81
:10A4E0000846BDE83240FEF717BE0B46012811466C
:10A4F000184608BF3DF058BBFEF72EBE014611F8C6
:10A50000060C032803D1024A1078FEF743BB7047BC
:10A51000E224002010B50C46210409D5054A107824
:10A52000FEF754FB08B100F00DF884F4004010BDB4
:10A53000002010BDE224002001490870704700BFD0
:10A54000E2240020F8B5044684B0656823682668D4
:10A550002768D4F800C0D4F800E022682168206899
:10A56000DB690393B66902967B690193DCF810609E
:10A570000096DEF80C30926849680068A8472168A8
:10A58000086014F8080CFEF783FC04460120FEF76F
:10A590003DFA010007D04220087005B02046BDE812
:10A5A000F040FEF706BB05B0F0BD000070B50546F3
:10A5B0000E466320FEF72AFA040020D0C220207045
:10A5C0000022E9786170A270E87888B920223146CB
:10A5D000E01CFEF7B4F92022291D04F12300FEF748
:10A5E000AEF9202205F1240104F14300FEF7A7F99A
:10A5F0002146BDE8704002480078FEF7CBBA70BD36
:10A600007902002038B505462320FEF7FFF9040043
:10A6100013D0C22020700122E9786170A270E8781E
:10A6200020B92022291DE01CFEF789F92146BDE84A
:10A63000344002480078FEF7ADBA31BD79020020FF
:10A6400053B94AB9002908BF00281CBF4FF0FF3199
:10A650004FF0FF3000F06EB9ADF1080C6DE904CE9B
:10A6600000F006F8DDF804E0DDE9022304B07047ED
:10A670002DE9F047089D04468C46002B40F083806E
:10A680008A42174647D9B2FA82F242B1C2F120009B
:10A6900024FA00F09140974040EA010C94404FEAC0
:10A6A0001748230CBCFBF8F61FFA87FE08FB16C1FF
:10A6B00043EA014306FB0EF1994209D9FB1806F162
:10A6C000FF3080F01981994240F21681023E3B44EE
:10A6D0005B1AA4B2B3FBF8F008FB103344EA03445E
:10A6E00000FB0EFEA64509D93C1900F1FF3380F0AE
:10A6F0000581A64540F2028102383C4440EA06400A
:10A70000A4EB0E0400261DB1D4400023C5E900438C
:10A710003146BDE8F08702B9FFDEB2FA82F2002AC4
:10A7200050D1CB1B4FEA174E1FFA87F80126B3FB17
:10A73000FEFC210C0EFB1C3341EA034108FB0CF329
:10A740008B4207D979180CF1FF3002D28B4200F20C
:10A75000E9808446C91AA3B2B1FBFEF00EFB1011CA
:10A7600043EA014408FB00F8A04507D93C1900F171
:10A77000FF3302D2A04500F2D9801846A4EB0804AA
:10A7800040EA0C40BFE78B4209D9002D00F0B180B0
:10A790000026C5E9000130463146BDE8F087B3FA2E
:10A7A00083F6002E4AD18B4202D3824200F2B88057
:10A7B000841A61EB030101208C46002DA8D0C5E965
:10A7C000004CA5E7C2F1200320FA03F6974001FAF6
:10A7D00002F04FEA174ED9403043030CB1FBFEF6AE
:10A7E0001FFA87F80EFB161143EA014306FB08F136
:10A7F000994204FA02F409D9FB1806F1FF3C80F0F3
:10A800008D80994240F28A80023E3B445B1A81B2BD
:10A81000B3FBFEF00EFB103341EA034100FB08F3EB
:10A820008B4207D9791800F1FF3C73D28B4271D962
:10A8300002383944CB1A40EA064678E7C6F1200CC4
:10A8400003FA06F422FA0CF31C4320FA0CF701FA7F
:10A8500006F34FEA144E21FA0CF11F433B0CB1FBF7
:10A86000FEF91FFA84F80EFB191143EA014109FBB6
:10A8700008FA8A4502FA06F200FA06F308D96118C6
:10A8800009F1FF3048D28A4546D9A9F1020921448D
:10A89000A1EB0A01BFB2B1FBFEF00EFB101147EABB
:10A8A000014700FB08F8B84507D9E71900F1FF3167
:10A8B0002ED2B8452CD90238274440EA0940A7EBEC
:10A8C0000807A0FB02894F45C64649461AD317D050
:10A8D0005DB1B3EB0E0267EB010707FA0CFCF24027
:10A8E0004CEA0202F740C5E9002700263146BDE8E0
:10A8F000F0872E4628460BE70646E9E61846FDE6B1
:10A900004345E5D2B8EB020E69EB04010138DFE7FD
:10A910000846D2E760468DE78146B9E7664675E7A7
:10A9200030464AE7ACF1020C394413E702383C44A4
:10A9300024E700BF704700BF70B4840746D04C1EA8
:10A94000002941D0D5B2034602E0611EE4B30C46B3
:10A9500003F8015B9907F8D1032C2ED9D5B245EA4B
:10A9600005250F2C45EA054519D9264603F11001A6
:10A97000103E0F2E41F8105C41F80C5C41F8085C69
:10A9800041F8045C01F11001F2D8A4F1100121F0AA
:10A990000F0104F00F041031032C0B440DD91E4697
:10A9A00021460439032946F8045BFAD8211F21F017
:10A9B000030104310B4404F003042CB1D2B21C4453
:10A9C00003F8012BA342FBD170BC70470C46034631
:10A9D000C2E710F8012B11F8013B012A28BF9A4267
:10A9E000F7D0D01A7047034613F8012B002AFBD189
:10A9F000181A013870470000000000000000000035
:10AA000001F0FF01102A2BDB10F0070F08D010F81F
:10AA1000013B013A8B422DD010F0070F42B3F6D123
:10AA2000F0B441EA012141EA014122F007047FF03C
:10AA300000070023F0E80256083C85EA010586EA93
:10AA4000010685FA47F5A3FA87F586FA47F6A5FACF
:10AA500087F68EB9EED1F0BC01F0FF0102F00702DB
:10AA600032B110F8013B013A83EA010313B1F8D186
:10AA70000020704701387047002D06BF3546033867
:10AA8000073815F0010F07D1013015F4807F02BFA0
:10AA9000013015F4C03F0130F0BC0138704700BFF1
:10AAA000054B1B6ADA0702D50123036070479B0739
:10AAB000FCD50223F9E700BFE424002007B501908C
:10AAC0008B8900930B79044A0021084630F02EFE52
:10AAD00003B05DF804FB00BF6480040007B5838900
:10AAE00000930379034A0021022030F01FFE03B0D7
:10AAF0005DF804FB958004001FB5DFF858C0DCF852
:10AB000000C0CDF80CC04FF0000C02928DF804107C
:10AB10001A46B3B100236A4601A9009301F0DCFA9A
:10AB2000009B3BB10A4B4FF080521A60BFF34F8F2E
:10AB3000BFF36F8F074B1A68039B5A4005D03CF058
:10AB4000F1FA01A901F0CEF9F4E705B05DF804FBD4
:10AB500004ED00E0B48004000348012300680022F3
:10AB60000621FFF7C9BF00BF3826002010B40C46ED
:10AB700000220346114660685DF8044BFFF7BCBF36
:10AB80002DE9F041404BDFF8148198B000240546D0
:10AB90001022002106A81B6817934FF000030FAF87
:10ABA0003CF050F901261C22214610A801960F9472
:10ABB0003CF048F92022394606A83CF03FF82946E7
:10ABC00006A807F02CF9314B0293099B8DF80C4035
:10ABD000FF2208F1540106A8CDE904373CF02EF815
:10ABE00004AA02A906A807F043F89DF9187067B1F6
:10ABF000274A3B462146204630F098FD224B1A68F2
:10AC0000179B5A403CD03CF08DFA01A8FFF748FF53
:10AC1000142239460AA83CF015F94FF48C70019CB7
:10AC200002F0E0FF054620B91A4A014630F07EFDE9
:10AC3000E4E7099A426108F1540118303CF0DAF86F
:10AC400040F201334FF0020CADF836303C230A9449
:10AC50000C96ADF838308DF82CC00AAC0FCC2E46CF
:10AC60000FC623683360394660460B4A30F05EFDFC
:10AC7000D8F804003B462A460721FFF73DFFBDE711
:10AC800018B0BDE8F08100BF248104000103000179
:10AC9000B8800400E98004000D810400E424002051
:10ACA000F7B5134C237E278B012B4EF660224FF015
:10ACB000000541F2883143F6982018BF114640F252
:10ACC00001320CBF052603262B46974214BF0A46C5
:10ACD00002460095A068042102F0F6FD6068012399
:10ACE0002A46314603B0BDE8F040FFF705BF00BF7C
:10ACF000E424002038B5044600236168994200D856
:10AD000038BD03F1500522688D421A4486BFCB1A24
:10AD10009BB250230021022030F0E6FB2B46ECE7EB
:10AD200010B5104C637E032B1AD10B0718D594F87D
:10AD30004210626C012303FA01F10A4204BF0A4384
:10AD4000626494F84C2018BF00234AB943B1064806
:10AD5000012300680221FFF7CFFE012384F84C3065
:10AD600010BD00BFE4240020382600208B0706D544
:10AD700003480123006800221946FFF7BDBE704753
:10AD800038260020012808B5034606D900210846C8
:10AD9000074A30F0CBFC002008BD064B0E3053F8BC
:10ADA000200031F04DFA431E58425841F4E700BFED
:10ADB00028810400E424002070B504461248037E74
:10ADC00003F0FD03012B0D4617D14069224605F023
:10ADD00031FE014638B100210346BDE870400B4A00
:10ADE000084630F0A3BCA389094A022030F09EFC3B
:10ADF0002846BDE87040FFF77DBF0021BDE87040E8
:10AE0000044A084630F092BCE42400203B81040050
:10AE100058810400728104002DE9F0415E4B5F4EC1
:10AE2000A4B00746102200210DA800241B6823931C
:10AE30004FF0000301253CF005F81022002111A875
:10AE400004953BF0FFFF1C2221461CA8CDE90744D6
:10AE50001B943BF0F7FF70698DF84C7007AA2146F0
:10AE600005F036FF5FBB8DF8455038F077F88DF868
:10AE70004C70ADF84600079B129304A80DF16C08C6
:10AE8000FFF70EFE049B8DF84430202241460DA8AA
:10AE90003BF0D4FE11A90DA807F084F89DF93440C9
:10AEA000002C35D03E4A23460021084630F03EFCB7
:10AEB000394B1A68239B5A406BD03CF033F996F813
:10AEC0004220716C8DF84C50954029408DF84540DA
:10AED000ADF846401AD0B36C1D4212D11D43F06844
:10AEE000079B33658DF86820B56402F05FFE03466A
:10AEF00030B90090F06847F23052042102F0E4FCCF
:10AF000001241AAB14938DF84D40B4E70C46F8E7D2
:10AF1000109B0594CDE90938DFF894808DF818402E
:10AF2000FF2241460DA8022501268DF815508DF807
:10AF300017603BF083FE05A909AA0DA806F098FE4C
:10AF40009DF9341011B1174A0B46ADE7109B0C93D5
:10AF5000102216A8CDF82C8003913BF073FF049BC0
:10AF600015938DF85850179687B140F20133ADF81C
:10AF700062300D4A03993C23ADF86430284630F026
:10AF8000D5FB0BA915A8FFF717FF91E7074A39462C
:10AF9000F4E724B0BDE8F081E8810400E424002057
:10AFA000AE860400B88004008D810400BA810400DC
:10AFB0003825002030B5244B244ACBB01B68499378
:10AFC0004FF0000390F91230049390F9113003937D
:10AFD0004B68029383890193836800930379044645
:10AFE0000D460220002130F0A1FB2846FFF782FE2B
:10AFF0002379032B0ED1A37B63B1A389144A0021CB
:10B00000022030F093FB104B1A68499B5A4018D02D
:10B010003CF088F84FF48472002107A83BF012FF3F
:10B02000A3896A682968ADF81C3009A808923BF02A
:10B03000E1FE084800231A4607A9006800F052FF05
:10B04000E1E74BB030BD00BF50820400EC8104004A
:10B05000358204003C26002008B5054A0021022064
:10B0600030F064FB3BF01AFC024B01221A60FEE751
:10B07000548204007C0520432DE9F047AB4BAC4FD4
:10B08000AC4CDCB006461B685B934FF0000330F01D
:10B09000F1F970684FF0FF3217A901F0E7F80128C5
:10B0A000F5D10025DFF8A092A1480795FF22294697
:10B0B0008DF820503BF0C6FE189A19A94846CDE9F4
:10B0C00009573BF0BBFD09AA07A9484606F007FE51
:10B0D000099B04939DF8203003939DF81C30029344
:10B0E0009DF81F3001939DF81E300093924A9DF801
:10B0F0001D302946022030F019FB99F9003013B1B8
:10B100008E4A29466BE09DF81C309DF81DA0002B4F
:10B1100067D0BAF1030F64D19DF81F209DF81E304F
:10B1200013439DF82020134308D1099931B9844A6B
:10B13000022030F0FBFA84F819A0A8E79DF81F80E0
:10B14000B8F1010FA3D19DF81E509DF820301D438A
:10B150009DD17C4A2946022030F0E8FADDE9092138
:10B1600079483BF06BFD1822294610A88DF86851EC
:10B170003BF068FE5AAB10A97348169306F0B0FE78
:10B1800099F9001011B1714A0B46BAE79DF84030A9
:10B19000022B23D19DF85530FF2B03D1C4E91111A7
:10B1A000216574E7012B12D8002B3FF470AF16987D
:10B1B000037808FA03F2636C23EA020363640278FB
:10B1C00008FA02F8A26C22EA0802A264E8E7604AE0
:10B1D00000934346084630F0A9FA58E75D4A08460E
:10B1E0008EE0BAF1010F7FF452AF9DF81E80B8F1E6
:10B1F000000F7FF44CAF9DF81F30012B7FF447AF59
:10B20000554A4146022030F091FADDE909214E48C5
:10B210003BF014FD59AB4C48ADF864810DA9CDF855
:10B220003480CDF83C800E9306F0C5FD99F90050AE
:10B230001DB14A4A2B464146D1E79DF834305A1E8B
:10B24000012A00F2CD801C22294610A8ADF86851D1
:10B250003BF0F8FD5AAB0BAA606914932946CDE97F
:10B260000B558DF840A005F033FD0B9B0F9A129300
:10B2700093421CBF9B1A11939DF83530FF2B42D18E
:10B280009DF83450A06B022D27D1642131F026F8AF
:10B29000E06B642131F022F8DFF8CC908DF84C504F
:10B2A0004FF00008022D19F8010B1FD1FFF76AFDBE
:10B2B00048B19DF84D3019F8012C01338DF84D300F
:10B2C000149B03F80820B8F1000F0CD09DF84D3006
:10B2D00093B110A8FFF754FCD9E630F0E1FFE06B22
:10B2E00030F0DEFFD8E74FF00108DBE7FFF74AFD5B
:10B2F00080F00100C0B2DBE70023194A1946184666
:10B3000030F014FAC3E6022B60D90093154A0223E9
:10B3100000215FE70E9B022A5B5D4FD1012B25D9EF
:10B3200000214246084630F001FA25E0508404002E
:10B3300058260020E424002085820400D0820400E6
:10B34000F482040011830400482600202A830400AC
:10B350004D830400818304009E830400B6830400AF
:10B36000DC830400FD830400242500200E336421C7
:10B3700054F8230030F0B2FF01359DF835309DF8C8
:10B3800034209D42C6D38DF84C2000259DF83530E1
:10B390009D429BD20E9B585D9DF83430022B19D1F3
:10B3A000FFF7F0FC40B19DF84D3001338DF84D3082
:10B3B0000E9B5A5D149B5A550135E7E7012BAFD818
:10B3C0000E3354F8230030F06BFFD5E7DFF8188018
:10B3D0000025D2E7FFF7D6FC80F00100C0B2E1E71C
:10B3E000004A8EE630840400288104001FB5CDE9B0
:10B3F00001210021074A0090084630F097F930F00B
:10B4000039F84FF0200383F31188BFF36F8FBFF338
:10B410004F8FFEE7548404002DE9F7430546037877
:10B42000494A0C460220002130F080F92B78032B8A
:10B4300005D8DFE803F0026D6F7F01232376AB6848
:10B4400001936B7900932B79404ADFF81891002122
:10B45000022030F06BF9AB6823626B79237705F13A
:10B460000C0704F1240800263B6848F8043B57F811
:10B47000043B00934A46334600210220013630F057
:10B4800055F9032EF0D1637E1BB92B790BB901233B
:10B490006376237E012B1ED1627E012A4CD10223CA
:10B4A000637641F288342A4EB06802F07FFB0128AF
:10B4B00006D100230093B0681A46032102F004FA73
:10B4C00000234FF47A7200935443B068B4FBF2F255
:10B4D000042102F0F9F9AB68DB0716D4AD88A5B9F1
:10B4E0001B4CA06802F062FB012806D10095A06801
:10B4F0002B462A46032102F0E7F900230093A068B7
:10B5000041F28832042102F0DFF903B0BDE8F08394
:10B51000022393E7606905F057F90E4A03460021BC
:10B52000022030F003F90C4B0C4A0D484FF488719F
:10B53000FFF75CFF032381E741F2883443F6982349
:10B54000032A08BF1C46AEE771840400B8840400D7
:10B55000E4240020848404009784040054890400B7
:10B560009D840400028504002DE9F04F974BB1B093
:10B570001B682F934FF00003954B054693E8070097
:10B580002CF0E0FA2BF0E4F80446002800F00382E7
:10B590002FF03CFF012805D98E4A234601210220C5
:10B5A0002FF03AFF2FF066FF8B4B8C4A40F276313A
:10B5B0008B48FFF71BFF1B986861194604F00AFFD0
:10B5C00001230446F0B92FF055FF864B009341F25A
:10B5D000883185486F692346224602F04FF90146BB
:10B5E000A86098B9814A30F0A1F8002F00F0C98115
:10B5F0001699384604F09EFF384605F05BF80023A4
:10B600006B61BEE17A4A00903146B2E1794B00931A
:10B6100047F2305178482346224602F02FF901467E
:10B62000E86008B9754ADEE70223754C2B762FF0E7
:10B6300021FF68684FF0FF3208A900F017FE0128CB
:10B64000F5D19DF82030072B00F26081DFE813F080
:10B65000080011002600430152012D00EA005201AA
:10B66000384605F0A3F809980028E0D002F0F9FA6E
:10B67000DDE7606905F0CEFA014650B10021614A6C
:10B68000084630F053F83BF009F95F4B01221A608D
:10B69000FEE75E4A022030F049F8E4E70120FFF7B8
:10B6A000BBFB002384F84C30DDE794F818A0BAF116
:10B6B000010F0FD0236ADB07D5D4637E012BD2D1D3
:10B6C000237F002BCFD152481A4600680321FFF791
:10B6D00013FAC8E794F81980B8F1020F6ED110225E
:10B6E00000210EA83BF0AEFB4A4ECDF814A010226C
:10B6F000002112A83BF0A6FB4FF0000B40F2012303
:10B700001C225946ADF8483028A8B31E14938DF872
:10B710004AA01396CDF89CB03BF094FB05A8FFF728
:10B72000BFF9059B8DF8543027AB194620220EA88F
:10B730003BF084FA12A90EA806F00AFB9DF9389096
:10B7400027ABB9F1000F03D0334A4B46002119E073
:10B75000119ACDF818901236CDE90A233146FF220E
:10B760000EA88DF81C908DF819803BF067FA06A999
:10B770000AAA0EA806F07CFA9DF9381031B1274AC2
:10B780000B46494608462FF0D1FF6CE7119B0D93FD
:10B7900010221CA803910C963BF054FB059B0399C7
:10B7A0001F4A1B9340468DF87080CDF874A02FF08F
:10B7B000BDFF0CA91BA8FFF7FFFA54E7B8F1030F70
:10B7C0007FF451AF0020FFF727FB4CE74C880400C3
:10B7D000B889040012850400388504006F890400CC
:10B7E0009D840400A1AC0000A7850400E585040049
:10B7F000B685040059AB00000586040018860400D5
:10B80000E42400203A8604007C0520436B86040073
:10B810003826002026250020AE860400A5860400D8
:10B82000D8860400684A002102204FF000092FF05A
:10B830007DFF1BAA60694946CDE91B9905F048FACE
:10B8400094F84260A36C4FF0010808FA06F616EA75
:10B850000302266D3AD0CEB11B9A961BB6B25B4A54
:10B860000096494602202FF061FF1D2E27D994F83B
:10B870004230C4F8509008FA03F8A36C23EA080396
:10B88000A364636C23EA080363644E460096A36CCA
:10B890004F4A002102202FF049FF2FF0EBFD002E30
:10B8A0003FF4E1AE4B4A002300935643E0684FF467
:10B8B0007A720421B6FBF2F202F006F8D3E6226DAA
:10B8C0001B9B9B1A9E42E1D99EB2DFE7002EDDD082
:10B8D00022651646DAE7404A002102202FF026FFB3
:10B8E0000121384605F0A6F9034600283FF4BBAE17
:10B8F0003A4A2BE7099830B100F118031B934369CA
:10B900001C931BA957E7364A0146C4E6099B0093DE
:10B910000021089B334A08462FF008FFA3E6324B6C
:10B920002193324B2293324B2393324B2493324B4D
:10B930002593324B26934FF4E153179320AB189382
:10B940002095169400F04CF92D4B19902D481A9320
:10B9500005F0D4F901231BA916A816931B9404F033
:10B9600087FA0123064600283FF425AE264A0096B2
:10B97000214608462FF0DAFE2FF07CFD00236B6194
:10B980001693002001F030F9204B1A682F9B5A4083
:10B9900017D03BF0C7FB2EF059FF04460028BED05D
:10B9A0002FF034FD012805D9194A23460121022030
:10B9B0002FF032FD2FF05EFD164B174A40F27D311D
:10B9C000F6E531B0BDE8F08F038704002A87040054
:10B9D0007C87040040420F00CF870400E687040004
:10B9E00016880400348804006DAB0000B5AF000079
:10B9F000DDAA0000BDAA000019B4000059B0000083
:10BA0000AC89040084890400748504004C88040017
:10BA100053850400388504006F89040070B5564BC7
:10BA2000564C8EB01B680D934FF0000303F0CFFB14
:10BA300030F0D4FE37F050FA514A07CA05AB83E81C
:10BA4000070018462FF080FE4E4A002102202FF0FA
:10BA50006DFE2FF00FFD08A830F06CFF4A4B0C93E1
:10BA600008A9002030F0BCFE206330B9474B484A9B
:10BA700040F265414748FFF7B9FC474B0C9308A9D2
:10BA8000012030F0ADFE606320B9444B404A40F2E3
:10BA90006941EFE703A830F0D7FB03A9002030F09D
:10BAA00087FCA06320B93E4B394A40F26E41E1E782
:10BAB00003A9012030F07CFCE06320B9394B344A03
:10BAC00040F27141D6E7082100220A2000F0A8F9CF
:10BAD000354E0146306038B9344A2FF027FE344BDA
:10BAE0002B4A40F27641C5E701234FF48072CDE93D
:10BAF000003400252377A4F8402060602D492E48AB
:10BB0000258323464FF4806284F8425001F03EF8CA
:10BB1000012809D0294A294628462FF007FE244B40
:10BB20001B4A40F28941A5E72A464FF484710A2056
:10BB300000F076F9224B1860336823B91C4B144A85
:10BB400040F28E4196E71F4B1F4958600222009237
:10BB50001E4801934FF4806201F018F8012804D0C8
:10BB6000134B0B4A40F2944184E701F029F9104B42
:10BB7000074A40F29A417DE750890400E4240020FE
:10BB8000587E04005088040021AD0000698804003C
:10BB90007F8904009D8404006DAD00008888040046
:10BBA000A7880400DC8804003826002011890400DE
:10BBB000978404002789040069B500002C890400DB
:10BBC0003C260020402600204689040079B0000071
:10BBD000024849F2880103F0B7B900BF349F002042
:10BBE000004870472C8A040010B5044602F0BAF9E8
:10BBF000A46B02F0DDF9B4FA84F0400910BDF8B589
:10BC00001546026C866B044652B9076847BB8068CC
:10BC100001F0EEFCA76005460136A6632846F8BD94
:10BC200065B940683BF0E6F86368226C1344A2688B
:10BC300063609342F0D323686360EDE7C0683BF034
:10BC4000D9F8226CE36851429B1A2268E360934260
:10BC50003EBFA3685B18E360022D01D116B1013E1F
:10BC60000025D9E73546D7E7034610B41A6C0846D5
:10BC70006AB1DC68996814448C4228BF1968DC609A
:10BC800028BFD960D9685DF8044B3BF0B3B85DF8C4
:10BC9000044B704770B5044602F064F994F84550BF
:10BCA00004F124066DB2002D14DCFF2384F8453026
:10BCB00002F07EF902F056F994F8445004F11006AF
:10BCC0006DB2002D12DCFF2384F84430BDE87040D3
:10BCD00002F06EB9636A002BE7D0304601F066FBD4
:10BCE00008B101F0F9FB013D6DB2DCE72369002BDF
:10BCF000E9D0304601F05AFB08B101F0EDFB013DFF
:10BD00006DB2DEE738B50D46044630B91B4B1C4A10
:10BD10001C4840F20D11FFF769FB02F023F9D4E94A
:10BD20000F31226862604B43D0185B1A1344A06045
:10BD3000E3600020FF23A06384F8443084F845309A
:10BD400095B9236963B104F1100001F02FFB38B1FC
:10BD50000D4B4FF080521A60BFF34F8FBFF36F8FC0
:10BD600002F026F9012038BD04F1100002F060FA5B
:10BD700004F1240002F05CFAF2E700BF688A0400D4
:10BD80006B8F0400728A040004ED00E013B51C46BA
:10BD900030B91C4B1C4A4FF4A4711C48FFF726FB1A
:10BDA00023B91B4B184A4FF4A671F6E72AB151B9D3
:10BDB000184B154A4FF4A871EFE721B1164B124A00
:10BDC00040F25111E9E750230193019B502B04D01D
:10BDD000124B0D4A40F25911DFE7002908BF2246F5
:10BDE000019B22600123C4E90F0184F84630194603
:10BDF0002046FFF787FF9DF8103084F84C3020462E
:10BE000002B010BD158B04007E8F0400728A0400FE
:10BE1000398B0400588B0400998B0400DA8B0400E2
:10BE2000F8B50D461746064630B9194B194A4FF476
:10BE3000C3711948FFF7DAFA484381B1B0FBF1F357
:10BE4000B34204D0154B134A4FF4C771F1E710F118
:10BE5000510F04D9124B0F4A40F29111E9E75030CB
:10BE600003F0A0F8044670B1002380F8463065B1B5
:10BE700000F15003C4E90F65236001212046FFF75C
:10BE800041FF84F84C702046F8BD0346F2E700BF3E
:10BE9000158B0400988F0400728A0400F78B04004D
:10BEA000488C040010B50C4630B90A4B0A4A40F2DF
:10BEB000ED210A48FFF79AFA884204D2084B064A55
:10BEC00040F2EE21F5E702220021FFF7A9FF00B1C1
:10BED000846310BD888C0400DE8F0400728A040025
:10BEE0009A8C04002DE9FF47884601921F460446BC
:10BEF00030B94D4B4D4A4FF443714D48FFF776FA38
:10BF000031B9036C23B14B4B484A40F20D31F4E791
:10BF1000022F07D1E36B012B04D0474B434A40F279
:10BF20000E31EAE701F006FB064630B9019B2BB162
:10BF3000424B3E4A40F21131DFE70026DFF800A114
:10BF40004FF0000937E0019D1DB902F031F80020E3
:10BF500050E016B902A801F075FA02F029F800F0D5
:10BF600083FF01F0FFFF94F84430FF2B08BF84F8F3
:10BF7000449094F84530FF2B08BF84F8459002F0B8
:10BF800017F801A902A801F069FA002846D101F0CA
:10BF9000E9FFA26BE36B9A422FD102F009F80199F5
:10BFA00004F1100001F0C2F92046FFF773FE01F022
:10BFB0000FF850B3012601F0D5FFA26BE36B9A4254
:10BFC00001D3022FBFD13A4641462046FFF717FE64
:10BFD000636A1BB104F1240001F0E8F938B1184B91
:10BFE0004FF080521A60BFF34F8FBFF36F8F01F095
:10BFF000DFFF012004B0BDE8F08701F0D9FF204643
:10C00000FFF748FE00F0E4FFD4E74FF08053CAF892
:10C010000030BFF34F8FBFF36F8FCBE72046FFF7A2
:10C0200039FE00F0D5FF92E7688A0400FC8F040017
:10C03000728A0400B98C0400128D0400618D040022
:10C0400004ED00E013B500220B46009011460120DC
:10C05000FFF79CFE044638B1002383600360C36091
:10C060001A461946FFF73EFF204602B010BD0000F9
:10C0700038B5044630B90C4B0C4A0D4840F26D21DE
:10C08000FFF7B4F9856801F04FFA85420AD1E368F9
:10C09000013BE36023B91A4619462046FFF722FF09
:10C0A000012000E0002038BDB68D0400AC8F0400F4
:10C0B000728A040010B5024600210120FFF7B0FE8D
:10C0C000044638B1002383600360C3601A461946F2
:10C0D000FFF708FF204610BD2DE9F843894690463A
:10C0E0001F46044630B92C4B2C4A4FF478712C482B
:10C0F000FFF77CF931B9036C23B12A4B274A40F290
:10C10000E131F4E7022F07D1E36B012B04D0264B7A
:10C11000224A40F2E231EAE702F05AF8EFF31186E0
:10C120004FF0200383F31188BFF36F8FBFF34F8F5E
:10C13000A26BE36B9A4201D3022F2AD194F84550A7
:10C14000A36B6DB23A4649462046FFF758FD6B1C7B
:10C1500013D1636A0BB901200BE004F1240001F054
:10C1600025F90028F7D0B8F1000FF4D00120C8F865
:10C17000000086F31188BDE8F8837F2D04D10B4BB6
:10C18000064A40F26B41B2E701356DB284F8455082
:10C19000E1E70020EDE700BF688A04000E9004008C
:10C1A000728A0400B98C0400128D0400C08D040052
:10C1B00070B50D46044630B9264B274A40F28B41F4
:10C1C0002648FFF713F9036C23B1254B224A40F2AE
:10C1D0008F41F5E7036833B9836823B1214B1E4AC9
:10C1E00040F29441ECE701F0F3FFEFF311864FF0DA
:10C1F000200383F31188BFF36F8FBFF34F8FA26BC0
:10C20000E36B934223D994F845100132FF294BB2D6
:10C21000A26310D1636A0BB9012009E004F1240084
:10C2200001F0C4F80028F7D0002DF5D001202860D7
:10C2300086F3118870BD7F2B04D10B4B064A40F268
:10C240001351BDE701335BB284F84530E4E70020C9
:10C25000EEE700BF688A040027900400728A040099
:10C26000E08D0400FB8D0400C08D04002DE9F04337
:10C2700085B00F460192044630B9464B464A40F21B
:10C280002F514648FFF7B2F831B9036C23B1444B44
:10C29000414A40F23351F4E701F04CF9064630B917
:10C2A000019B2BB13F4B3C4A4FF4A761E9E70026C5
:10C2B000DFF8F4904FF000083BE0019D1DB901F05C
:10C2C00077FE002052E016B902A801F0BBF801F099
:10C2D0006FFE00F0C9FD01F045FE94F84430FF2BDD
:10C2E00008BF84F8448094F84530FF2B08BF84F8D9
:10C2F000458001F05DFE01A902A801F0AFF8002819
:10C300003DD12046FFF770FC98B3019904F1240059
:10C3100001F00CF82046FFF7BDFC00F059FE38B9DB
:10C320004FF08053C9F80030BFF34F8FBFF36F8FCA
:10C33000012601F017FEA56B002DBED03946204620
:10C34000013DFFF791FCA563236963B104F110007F
:10C3500001F02CF838B1144B4FF080521A60BFF343
:10C360004F8FBFF36F8F01F023FE012005B0BDE8B2
:10C37000F0832046FFF78EFC00F02AFED8E7204627
:10C38000FFF788FC00F024FE2046FFF72DFC002874
:10C39000CED096E75E8E040039900400728A0400C5
:10C3A0006C8E0400618D040004ED00E02DE9FF4176
:10C3B0000446019130B9574B574A40F2C151574892
:10C3C000FFF714F8056C25B1554B534A40F2C5519F
:10C3D000F5E701F0AFF8064630B9019B4BB1514B80
:10C3E0004D4A40F2CA51EAE72E46DFF84081002765
:10C3F0004DE00546F9E7019B43B925B14A4B464A52
:10C400004FF4C261DBE701F0D3FD5EE016B902A88C
:10C4100001F018F801F0CCFD00F026FD01F0A2FDBE
:10C4200094F84430FF2B08BF84F8447094F84530EA
:10C43000FF2B08BF84F8457001F0BAFD01A902A8DE
:10C4400001F00CF800284AD12046FFF7CDFB002868
:10C450003FD023683BB901F085FDA06801F07AF870
:10C46000054601F0A5FD019904F1240000F05EFFEE
:10C470002046FFF70FFC00F0ABFD38B94FF08053BA
:10C48000C8F80030BFF34F8FBFF36F8F012601F064
:10C4900069FDA36B002BAED0013BA363236813B9E6
:10C4A00001F050F9A060236963B104F1100000F0BD
:10C4B0007DFF38B11D4B4FF080521A60BFF34F8F94
:10C4C000BFF36F8F01F074FD0125284604B0BDE86D
:10C4D000F0812046FFF7DEFB00F07AFDD6E720462C
:10C4E000FFF7D8FB00F074FD2046FFF77DFB002826
:10C4F000CCD0002DE9D001F035FD616A19B1236B74
:10C500001968C1F10A01A06801F0C2F8002501F024
:10C510004FFDDAE75E8E040047900400728A040043
:10C52000E08D0400618D0400C88E040004ED00E07D
:10C5300037B5044630B90E4B0E4A0F4840F2A521DC
:10C54000FEF754FF8568019100F0EEFF85420199E6
:10C5500005D1E3680133E360012003B030BD20461C
:10C56000FFF724FF0028F8D0E3680133E360F4E725
:10C57000B68D0400C58F0400728A04002DE9F043D3
:10C5800085B00F460192044630B9464B464A40F208
:10C590009A614648FEF72AFF31B9036C23B1444B38
:10C5A000414A40F29E61F4E700F0C4FF064630B90C
:10C5B000019B2BB13F4B3C4A40F2A361E9E70026C7
:10C5C000DFF8F4904FF000083BE0019D1DB901F049
:10C5D000EFFC002052E016B902A800F033FF01F092
:10C5E000E7FC00F041FC01F0BDFC94F84430FF2B67
:10C5F00008BF84F8448094F84530FF2B08BF84F8C6
:10C60000458001F0D5FC01A902A800F027FF002811
:10C610003DD12046FFF7E8FA98B3019904F12400D0
:10C6200000F084FE2046FFF735FB00F0D1FC38B95E
:10C630004FF08053C9F80030BFF34F8FBFF36F8FB7
:10C64000012601F08FFCA36B002BBED0394620469B
:10C65000E568FFF709FB636AE56063B104F1240054
:10C6600000F0A4FE38B1144B4FF080521A60BFF3B3
:10C670004F8FBFF36F8F01F09BFC012005B0BDE829
:10C68000F0832046FFF706FB00F0A2FCD8E7204627
:10C69000FFF700FB00F09CFC2046FFF7A5FA0028FE
:10C6A000CED096E75E8E04005B900400728A040090
:10C6B0006C8E0400618D040004ED00E02DE9F84368
:10C6C00089469046054630B9244B254A40F22F71E1
:10C6D0002448FEF78BFE31B9036C23B1224B204A6C
:10C6E0004FF4E661F4E701F073FDEFF311874FF0CB
:10C6F000200383F31188BFF36F8FBFF34F8FAC6BB1
:10C7000054B395F84460494676B22846FFF7ACFA30
:10C71000013C731CAC6313D12B690BB901200BE0F6
:10C7200005F1100000F042FE0028F7D0B8F1000F2C
:10C73000F4D00120C8F8000087F31188BDE8F88321
:10C740007F2E04D1094B064A40F27371C0E70136CF
:10C7500076B285F84460E1E72046EDE7688A040098
:10C7600066900400728A0400F78E04004B8F040068
:10C7700008B530B9074B084A084840F2EE71FEF799
:10C7800035FE90F846301BB9BDE8084002F018BCF1
:10C7900008BD00BF688A04007B900400728A040010
:10C7A00070B504460D46164601F0DCFB94F84430A3
:10C7B000FF2B04BF002384F8443094F84530FF2B4E
:10C7C00004BF002384F8453001F0F2FBA36B2BB9C2
:10C7D0003246294604F1240000F0C6FD2046BDE89B
:10C7E0007040FFF757BA00002DE9F041044601F010
:10C7F000B9FB2F4B2F4D1A682F4F01321A602E684C
:10C80000002E49D12C601B68012B1FD1B846404631
:10C81000013601F00DFD0A2E08F11408F7D1DFF8FA
:10C82000C480264E404601F003FD304601F000FD75
:10C83000234801F0FDFC234801F0FAFC224801F0F6
:10C84000F7FC224BC3F80080214B1E60214A22498D
:10C850001368086801331360E26A2364012393407C
:10C86000034314200B6000FB0270211D01F0EEFC5D
:10C8700001F09EFB194B1B6863B12B68DA6AE36A0F
:10C880009A4207D2164B4FF080521A60BFF34F8F77
:10C89000BFF36F8FBDE8F081104B1B68002BD5D123
:10C8A0002B68DA6AE36A9A4298BF2C60CEE700BF31
:10C8B0002C2800205827002064270020542800201E
:10C8C00074280020A02800208C2800205C2700204D
:10C8D00060270020382800203C28002088280020DD
:10C8E00004ED00E040280020094B0A4A1B6812684A
:10C8F000D06A58B9084A1268012A08D8012B06D80C
:10C90000064B1868064B1B68C01A7047002070471A
:10C910003C28002058270020642700206828002099
:10C92000B4280020064A13681968064B19B94FF05D
:10C93000FF321A6070471268D2681268F9E700BFC8
:10C940005C270020682800202DE9F843DDE90984F0
:10C950004FEA82094A4606460D46206BA5211F462E
:10C960003AF070FA226BA9F10409914429F0070901
:10C97000002D60D06B1E04F134020B3513F8011F3B
:10C9800002F8011B197809B1AB42F7D1002384F8F2
:10C990003F30089D092D28BF09250021E164E5628B
:10C9A000A564201D01F04FFC04F1180001F04BFCC0
:10C9B000C5F10A050021216504222461A561646294
:10C9C00004F154003AF03EFA0422002104F590608C
:10C9D0003AF038FA0122002104F284403AF032FAA7
:10C9E0004FF48562002104F158003AF02BFA04F567
:10C9F0005173E36504F56B73236604F214436366B5
:10CA000001220023C4E940230C4A0D4BC4E9422310
:10CA10000C4BC4F810310B23A4F814313A463146BC
:10CA2000484601F071FA2060B8F1000F01D0C8F853
:10CA30000040BDE8F88384F83450AAE70E33CDAB4C
:10CA400034126DE6ECDE050010B5044658303AF0BD
:10CA50008BFA94F885343BB9206B02F0B1FA20468A
:10CA6000BDE8104002F0ACBA012BF8D0022B06D082
:10CA7000034B044A044840F68A71FEF7B7FC10BD28
:10CA800088900400C4940400BC900400F8B51B4BCB
:10CA90001B4F1D680446386804300E4601F0F8FB51
:10CAA0003B4640B939681748CF6A02680121B9404E
:10CAB00022EA01020260621C07D136B119681248ED
:10CAC000BDE8F840043101F0C1BB1A682C1954606C
:10CAD00007D30E4A10681968BDE8F840043101F028
:10CAE000C0BB0B4A10681968043101F0BAFB094B4E
:10CAF0001A68A24288BF1C60F8BD00BFB42800209D
:10CB0000582700203C2800208C2800206027002087
:10CB10005C2700206828002070B586B0DDE90B5442
:10CB200035B9154B154A4FF412711548FEF75EFCE6
:10CB300024B9144B114A40F24921F6E74FF49166AB
:10CB40000596059EB6F5916F04D00F4B0B4A40F247
:10CB50005121EAE72563022584F8855404AD019547
:10CB60000A9D02940095059EFFF7EEFE2046FFF712
:10CB70003BFE049806B070BD5F910400C1930400B1
:10CB8000BC9004007F9104009D9104002DE9F043C6
:10CB9000074685B0900088461646994602F002FA8C
:10CBA0000546F0B14FF4916002F0FCF90446A8B1DB
:10CBB000002380F885340D9B056301930C9B029044
:10CBC000009332464B4641463846FFF7BDFE2046AD
:10CBD000FFF70AFE012005B0BDE8F083284602F009
:10CBE000EFF94FF0FF30F6E7F8B50446284D01F0B5
:10CBF000B9F904B92C68261D304601F049FB60B92B
:10CC0000E76A244B142078431B5833B92249012288
:10CC10000B68BA4023EA02030B60A36A1BB104F15C
:10CC2000180001F035FB1D4A1368013313602B68AF
:10CC3000A34219D11A48314601F008FB194A13687A
:10CC40000133136001F0B4F9174B1B68F3B12B6883
:10CC5000A3421BD1154B1B6883B1154B154A1648CF
:10CC600040F2D241FEF7C2FB144A13682046013B52
:10CC70001360FFF7E9FEFFF755FEE3E7104B4FF0B7
:10CC800080521A60BFF34F8FBFF36F8FF8BD00BFA4
:10CC900058270020642700203C2800203828002046
:10CCA000A0280020302800208828002034280020D8
:10CCB000B8910400D3930400BC9004002C280020F9
:10CCC00004ED00E013B5044601F04CF90CB9044B37
:10CCD0001C68E06A019001F06BF9019802B010BD88
:10CCE000582700200929F7B504460D4606D92D4BD3
:10CCF0002D4A2E4840F20B61FEF778FB01F032F925
:10CD00000CB92B4B1C68A26C95423ED0284B41D9E4
:10CD10001968A14243D01B68DE6AAE428CBF002670
:10CD20000126E76AA369A564BA4208BFE562002B41
:10CD3000A4BFC5F10A05A5611E4D6269142303FB5A
:10CD400007539A4218D1211D0846019101F0A0FA1B
:10CD5000194A019928B913680120B84023EA000351
:10CD60001360E06A14680123834023431360142393
:10CD700003FB005001F06AFA3EB1104B4FF08052B5
:10CD80001A60BFF34F8FBFF36F8F03B0BDE8F04061
:10CD900001F00EB91E68331B5E425E41C1E70026FA
:10CDA000BFE700BFD4910400DF930400BC900400EF
:10CDB00058270020642700203C28002004ED00E0D4
:10CDC00010B588B0002407AA06A905A8CDE9054436
:10CDD00000F0E6FF059B0293069B079A1749184847
:10CDE000CDE900432346FFF797FED0B100F010FDD8
:10CDF00001281AD14FF0200383F31188BFF36F8FFE
:10CE0000BFF34F8F0F4B104A1B68583313600F4B03
:10CE10004FF0FF321A600E4B18600E4B1C6001F091
:10CE200053F90D4B1B6808B010BD0130F9D10B4B05
:10CE30000B4A0C4840F63601FEF7D8FAF39104008D
:10CE4000C9D0000058270020682000206828002052
:10CE500088280020B4280020E0110020F891040068
:10CE6000FD930400BC900400024A13680133136070
:10CE7000704700BF34280020014B1868704700BF7E
:10CE8000B428002008B5094B09491A68096802440A
:10CE90008A4206D9074B084A084840F63B21FEF76C
:10CEA000A5FA1A681044186008BD00BFB428002015
:10CEB000682800200C92040020940400BC90040018
:10CEC0002DE9F84F344B1B68002B5ED1334B1E68A5
:10CED00001361E60AEB9324B1A68126832B1314B5E
:10CEE000314A324840F6BC21FEF780FA304A1968D0
:10CEF0001068186011602F4A136801331360FFF740
:10CF000011FD2D4F3B689E424FF0000407D22B4B82
:10CF10001B68002B18BF01242046BDE8F88FDFF8FE
:10CF20008090DFF8A480DFF8A4A0D9F800301B6857
:10CF30001BB94FF0FF333B60E9E7D9F80030DB68FD
:10CF4000DD686B689E42F6D305F1040B584601F08C
:10CF50009FF9AB6A1BB105F1180001F099F9EA6A73
:10CF6000D8F800100123934014200B4300FB02A0CB
:10CF70005946C8F8003001F069F9114BEA6A1B689C
:10CF8000DB6A9A4228BF0124CFE70E4A13680133B7
:10CF900013600024C0E700BF34280020B42800201C
:10CFA0005C270020449204002E940400BC900400EE
:10CFB000602700206C28002068280020B828002066
:10CFC00058270020702800203C28002064270020DB
:10CFD0002DE9F341304C236833B9304B304A3148A6
:10CFE00040F6A901FEF702FA00F0BCFF2368013BFE
:10CFF0002360246834B1002400F0DAFF204602B038
:10D00000BDE8F081284B1B68002BF4D0274D284E3B
:10D01000DFF8B0801FE0EB68DC6804F1180001F075
:10D0200037F9211D0846019101F032F9E26A3068B2
:10D030000199012707FA02F30343142000FB028041
:10D04000336001F003F91B4BE26A1B68DB6A9A420A
:10D0500001D3194B1F602B68002BDCD10CB1FFF7FB
:10D0600061FC164D2C6844B1134E0127FFF728FFD1
:10D0700000B13760013CF9D12C600F4B1B68002BCD
:10D08000B9D00F4B4FF080521A60BFF34F8FBFF3F0
:10D090006F8F0124B0E700BF34280020BC92040049
:10D0A00011940400BC9004002C2800207428002057
:10D0B0003C28002058270020B82800207028002095
:10D0C00004ED00E064270020F8B51A4C1A4F1B4D00
:10D0D000236893B9FFF708FC0128F8D9FFF7C4FECD
:10D0E000174B1A68174B1B689A4219D2164B174AEE
:10D0F000174840F6B551FEF779F900F033FFFB68A9
:10D10000DE68301D01F0C4F82B68013B2B602368FA
:10D11000013B236000F04CFF3046FFF795FCD7E75A
:10D12000FFF7E2FB012801D900F034FEFFF750FFC2
:10D13000CDE700BF30280020A02800202C280020A8
:10D1400068280020B4280020D3920400B89404007A
:10D15000BC90040038B50D46044608B9044B1C6861
:10D1600000F000FF2565BDE8384000F021BF00BF9A
:10D170005827002013B5044608B9054B1C6800F079
:10D18000F1FE206D019000F013FF019802B010BD78
:10D190005827002038B5244B1A68244B12B10122BD
:10D1A0001A6038BD224C1A6023681B6B1A68B2F1F2
:10D1B000A53F0BD15A68B2F1A53F07D19A68B2F1E9
:10D1C000A53F03D1DB68B3F1A53F04D020682168F7
:10D1D000343100F07AFD174B1B68B3FA83F3DBB2EE
:10D1E000C3F11F03142214495A4388188D5835B9C6
:10D1F000124B134A134840F6F731FEF7F7F845682B
:10D2000008326D6845600A44954204BF6A6842600E
:10D21000142202FB03130C4A5B68DB68236023685B
:10D2200058331360BDE700BF34280020B828002021
:10D23000582700203C28002064270020F892040092
:10D2400041940400BC90040068200020F8B5044616
:10D250002B4E00F087FE04B93468251D284601F0E6
:10D2600017F860B9E76A274B142078431B5833B985
:10D27000254901220B68BA4023EA02030B60A36A26
:10D280001BB104F1180001F003F829461F48204D96
:10D2900000F0DCFF94F88434012B04BF002384F8F1
:10D2A000843400F085FE2A682AB100F05BFEFFF7A7
:10D2B00039FB00F07DFE3368A34213D12B6893B194
:10D2C000144B1B6833B1144B144A154840F2F361F8
:10D2D000FEF78CF8134B4FF080521A60BFF34F8F5C
:10D2E000BFF36F8FF8BD094A11680F4A1268914267
:10D2F00001D13360F6E7BDE8F840FFF74BBF00BF50
:10D3000058270020642700203C2800208C2800207B
:10D310008828002034280020B8910400F0930400ED
:10D32000BC90040004ED00E02C28002010B50C4651
:10D3300030B9094B094A0A4840F61141FEF756F840
:10D34000084B1968183100F08CFF20460121BDE818
:10D350001040FFF79BBB00BF3F93040054940400B0
:10D36000BC9004005827002038B50D46144630B94B
:10D370000A4B0B4A0B484FF44461FEF737F80A4B4F
:10D380001968183100F062FF002C21460CBF2846B6
:10D390004FF0FF30BDE83840FFF778BB3F93040003
:10D3A0006A940400BC9004005827002037B5C36875
:10D3B000DC6834B91A4B1B4A1B484FF44761FEF72F
:10D3C00015F804F118010846019100F061FF174BB0
:10D3D00001991B6803BB211D0846019100F058FF0D
:10D3E0001348E26A05680199012393402B430360C7
:10D3F000104B142000FB023000F028FFFFF792FAD8
:10D400000D4BE26A1B68DB6A9A4285BF0B4B012019
:10D410000020186003B030BD094800F017FFEFE7A7
:10D420004D9304008A940400BC900400342800202A
:10D430003C2800206427002058270020B82800201E
:10D4400074280020034B1B680360034B1B68436078
:10D45000704700BF6C280020B428002070B50D462E
:10D46000044630B9164B174A40F6EB411648FDF713
:10D47000BDFF21B9154B134A40F6EC41F6E700F029
:10D4800071FD134B19682B685A1C17D01148266878
:10D4900000686268864208D08A4206D800232B6062
:10D4A000012400F085FD204670BD881A8342F5D91D
:10D4B0005B1A13442B602046FFF7C4FF0024F0E7FB
:10D4C0005E930400A3940400BC9004006A930400DB
:10D4D000B42800206C280020014B01221A607047FC
:10D4E000B82800200B4B1B687BB90B4A106870B939
:10D4F0000A4B1B6863B90A4B18680A4B1B68013B4F
:10D50000984214BF0120022070470020704718463F
:10D51000704700BF74280020B82800207028002021
:10D520008C2800202C280020014B1868704700BF71
:10D5300058270020054B1B6833B1054B1B68002B97
:10D540000CBF02200020704701207047882800206F
:10D5500034280020F7B50446002832D0214AC36A97
:10D560001168C96A8B42164633D282691E4D002A61
:10D57000A1BF3268D26AC2F10A028261142202FBA0
:10D58000035342699A421ED1011D0846019100F0E1
:10D590007FFE164B019930B9E76A1A680120B8403E
:10D5A00022EA00021A6032681E68D26AE26201242E
:10D5B00004FA02F030431860142000FB025000F01F
:10D5C00045FE204603E03368DB6AC362012003B0F6
:10D5D000F0BD1368806CDC6AA0422CBF00200120E3
:10D5E000F5E700BF58270020642700203C280020D2
:10D5F00037B5044610B9002003B030BD1D4B1B6881
:10D60000834206D01C4B1D4A41F23D011C48FDF7E8
:10D61000EDFEDB6C23B91B4B184A41F23E01F5E7E6
:10D62000C16A826C013B9142C364E4D0002BE2D119
:10D63000011D0846019100F02BFE134A019930B9F3
:10D64000E56A13680120A84023EA00031360A36C75
:10D650001568E362C3F10A00A061012404FA03F033
:10D6600028431060094A142000FB032000F0EEFD5F
:10D670002046C1E7582700207A930400D194040083
:10D68000BC900400929304003C28002064270020F2
:10D6900037B50446002845D0C26C32B9224B234A24
:10D6A00041F28D012248FDF7A1FE836C994238BFFB
:10D6B0001946C36A8B4235D0012A33D11D4A1268FC
:10D6C000824204D11C4B194A41F2A801EAE782695F
:10D6D0001A4DC162002A4FF0140202FB0353426943
:10D6E000A4BFC1F10A0181619A421BD1011D084604
:10D6F000019100F0CDFDE46A114A019928B913683F
:10D700000120A04023EA0003136010680123A34016
:10D710000343142000FB0450136003B0BDE8304005
:10D7200000F094BD03B030BD92930400E99404006E
:10D73000BC90040058270020A9930400642700200F
:10D740003C280020044B1A681AB11968CA6C0132CF
:10D75000CA641868704700BF58270020F7B50F4CFF
:10D7600000F000FC25689DB90D4F0E4E384600F0C4
:10D770005FFD304600F05CFD0B4B0C4A1F600C4B0C
:10D780000C211E6014200B4B0095FEF7FFFA206061
:10D7900003B0BDE8F04000F00BBC00BF302A002011
:10D7A000B4290020C8290020BC280020C42800205B
:10D7B000C0280020E0290020914208B541600061A6
:10D7C0000AD8D21A83699A420DD2084B011D1868F3
:10D7D00000F047FD002008BD9A4201D2994202D2D2
:10D7E000034B011DF3E70120F5E700BFC02800202F
:10D7F000BC28002008B5034A034B044840F25F11DF
:10D80000FDF7F4FD319604000D9504002B950400FE
:10D8100010B588B0FFF7A2FF114B1B68B3B100240D
:10D8200007AA06A905A8CDE9054400F0C5FA059B9D
:10D830000293069B019305230093079A09490A481E
:10D840002346FFF769F9094B186030B9084B094ABC
:10D85000094840F20D11FDF7C9FD012008B010BDC7
:10D86000302A0020CF950400ADD90000342A0020D2
:10D87000D79504001B9604002B9504002DE9F04178
:10D8800080462C200D4616461F4601F08BFB0446B1
:10D89000B8B1002380F828300DB9FFF7ABFFFFF7D0
:10D8A0005DFF069BC4F80080C4E906572362201D73
:10D8B00000F0C9FC2EB194F8283043F0040384F83A
:10D8C00028302046BDE8F0817FB5164604461A464A
:10D8D00030B9114B114A12484FF4C171FDF786FD62
:10D8E000104D286880B10529CDE9011603940DDC9F
:10D8F000FFF720FE0023022808BF089A286818BFF7
:10D900001A4601A9FEF7EEFA04B070BD002301A982
:10D91000FEF7E2FBF8E700BFE1950400479604003C
:10D920002B950400302A0020F0B51B4D85B0002750
:10D930002B681A682AB9194A11682960136005B062
:10D94000F0BDDB68DC681E68211D0846039100F00D
:10D950009FFC236A2046984794F82830039913F0D7
:10D96000040FE5D0A36933449E4205D22868636062
:10D97000246100F076FCDBE700230097324619466D
:10D980002046FFF7A1FF0028D2D1054B054A0648E3
:10D9900040F2A931FDF72AFDBC280020C028002054
:10D9A000EA9504008E9604002B9504002DE9F04FB3
:10D9B000744E87B0B1463368D3F800B0BBF1000FA6
:10D9C00028D0DB68D3F800B000246F4D6F4FFFF70D
:10D9D0004BFAFFF751FA2B6898428246A8461BD3B0
:10D9E000286014B36A4B1B681C68B4FA84F4640999
:10D9F00038682246ABEB0A01FEF7D2FEFFF7E8FAE1
:10DA000080B9644A4FF080531360BFF34F8FBFF368
:10DA10006F8F07E00124D8E7FFF786FFC5F800A065
:10DA2000FFF7D6FA4FF0000B6DE08345E0D8FFF723
:10DA3000CFFAD9F80030DB68DD68281D00F028FC3B
:10DA400095F82830580716D5A9695B4652465944BF
:10DA50002846FFF7B1FE90B1009423465A4621466E
:10DA60002846FFF731FF50B94B4B4C4A4FF4057134
:10DA70004B48FDF7BBFC23F0010385F828302B6AE7
:10DA800028469847CEE794F82830A16943F001036F
:10DA900084F82830049B2A4619442046FFF78CFE60
:10DAA00088B3236A2046984794F8283059072AD526
:10DAB000A2690499CDF800B000230A442046194613
:10DAC000FFF702FFF8B9344B364A40F23631CFE760
:10DAD00094F8283023F0010384F8283013E094F8F8
:10DAE00028300499A16143F0010384F8283021B95A
:10DAF0002D4B2C4A40F24F31BAE72B462A46294497
:10DB00002046FFF759FE3868002203A9FEF7AEFB56
:10DB100000283FF450AF039B002BF4DB059C6369A6
:10DB200013B1201D00F0B4FBFFF7A6F9D8F80030C0
:10DB30009842054601D2FFF7F7FE039BC8F8005054
:10DB4000092BE0D801A252F823F000BF87DA0000C9
:10DB500087DA000087DA0000D1DA0000DFDA00009F
:10DB600075DB000087DA000087DA0000D1DA0000F8
:10DB7000DFDA000094F828309A07ABD4204601F091
:10DB80001FFAC0E7BC280020DC290020302A002032
:10DB9000C028002004ED00E0EA9504005C96040033
:10DBA0002B95040073960400F495040013B5044605
:10DBB00030B9094B094A0A4840F2F131FDF716FC29
:10DBC00000F0D0F994F8280000F00100019000F076
:10DBD000EFF9019802B010BDE1950400A29604008F
:10DBE0002B95040038B50823C5182CBF012300234A
:10DBF00000B133B139F0EAF816230360002420465F
:10DC000038BD284601F0CEF9044620B939F0DEF8D7
:10DC10000C230360F3E7C0E900050834EFE713B510
:10DC2000044630B939F0D2F816230360204602B01A
:10DC300010BD01FB00F2B2FBF0F48C4205D039F0CC
:10DC4000C5F88B2303600024F0E710460192FFF72C
:10DC5000C9FF04460028E9D0019A002139F0F2F802
:10DC6000E4E718B150F8080C01F0AAB9704770B594
:10DC70000C46054620B9BDE870400846FFF7B2BF24
:10DC800031B939F0A3F8162303602646304670BD3B
:10DC90000846FFF7A7FF06460028F7D055F8042CE2
:10DCA000083AA24228BF2246294639F0A3F828465E
:10DCB000FFF7D7FFEAE70846FFF794BF0846FFF7EC
:10DCC000D0BF08461146FFF7D2BFFEE738B538F09F
:10DCD000E5FDFFF707FC18B9BDE8384038F0E2BDB4
:10DCE000264B1B685B68984733F076FB430705D5E6
:10DCF000AFF3008030BFAFF30080EDE700F04AFBE8
:10DD00001F4B19680A224FF47A7302FB00F54B434C
:10DD100001219D420446084624BF1D46B3FBF2F490
:10DD200033F060FBA842D7D2164D17482B6823F07A
:10DD30000103A4F118012B6000F064FC124800F00C
:10DD4000EFFB00F071FC0446AFF30080012033F0DC
:10DD500049FEAFF300800C4800F051FC00F064FC79
:10DD60000A23001B58434FF47A73B0FBF3F0FFF71C
:10DD700089F82B6843F005032B60ADE7E80100103C
:10DD8000382A002010E000E0F81E0020FFF76CB8F1
:10DD9000FFF71EB9014B186033F032BB382A002060
:10DDA000034B0360034B0B604FF4807313607047A9
:10DDB000403600203C2A0020034B0360034B0B60DD
:10DDC0004FF4007313607047C83A00203C2E0020C7
:10DDD00040F20000C0F200000068854600F004B880
:10DDE000FEE7FEE7FEE7FEE770B51B4A136843F463
:10DDF0007003136038F0D4F94FF0200383F31188D7
:10DE0000BFF36F8FBFF34F8F144B154A002193421E
:10DE100014D3144A144B9A4202D014498B4210D3A3
:10DE2000134D144C641BA4100026A6420ED1124BB5
:10DE3000124A1A60BDE87040FDF7F0BD43F8041BBC
:10DE4000E5E752F8040B43F8040BE7E755F8043B09
:10DE500098470136E9E700BF88ED00E0D8210020AF
:10DE6000F0530120381C0500E00F0020CC200020DA
:10DE7000507E0400587E040008ED00E00000000021
:10DE80007047000008480068006880F308884FF079
:10DE9000000080F3148862B661B6BFF34F8FBFF302
:10DEA0006F8F00DF00BF000008ED00E0DFF80C001E
:10DEB000016841F4700101607047000088ED00E0E6
:10DEC00007B5002301930C4B1B68013305D00B4BA6
:10DED0000B4A0C48E521FDF789FA4FF0200383F344
:10DEE0001188BFF36F8FBFF34F8F019B002BFCD0C6
:10DEF00003B05DF804FB00BFE4110020B6960400F7
:10DF000020990400D29604004FF0807340F8043C3E
:10DF1000074B40F80C3C21F001016FF0020340F880
:10DF2000081C40F8202C40F8243C4438704700BFBF
:10DF3000C1DE000000000000000000000000000042
:10DF4000074B19680868B0E8F04F80F30988BFF301
:10DF50006F8F4FF0000080F311887047AFF300809F
:10DF60005827002008B54FF0200383F31188BFF332
:10DF70006F8FBFF34F8F094A13680133012B136072
:10DF80000BD1074B1B6813F0FF0F06D0054B064A59
:10DF900006484FF4D271FDF729FA08BDE4110020BC
:10DFA00004ED00E08A97040045990400D29604002D
:10DFB00008B5084A136833B9074B084A084840F2C5
:10DFC000AB11FDF713FA013B13600BB983F3118812
:10DFD00008BD00BFE4110020CE970400589904004A
:10DFE000D2960400000000000000000000000000C5
:10DFF000EFF30980BFF36F8F154B1A681EF0100FF7
:10E0000008BF20ED108A20E9F04F10602DE90900CB
:10E010004FF0200080F31188BFF34F8FBFF36F8F55
:10E02000FFF7B8F84FF0000080F3118809BC1968B9
:10E030000868B0E8F04F1EF0100F08BFB0EC108A6F
:10E0400080F30988BFF36F8F704700BFAFF3008084
:10E050005827002008B54FF0200383F31188BFF341
:10E060006F8FBFF34F8FFEF72BFF18B1034B4FF0AD
:10E0700080521A60002383F3118808BD04ED00E08C
:10E080000B4B0C494BF680321A600B4B40F25D1281
:10E090001A600A4B2D221A60094B00221A600A608E
:10E0A000084A4BF67F31116007221A60704700BFA3
:10E0B0005C3F002018E000E0603F0020583F002057
:10E0C00010E000E014E000E013B5334B334A196868
:10E0D000914206D1324B334A4FF496713248FDF7E4
:10E0E00085F91A68314B9A4204D1314B2D4A40F2DE
:10E0F0002D11F3E72F4B1A78D2B20192FF221A703A
:10E100001B782D4ADBB28DF803309DF8033003F005
:10E1100020031370294A0723136000219DF8030090
:10E12000000603F1FF3408D411B1042B13600DD0A5
:10E13000234B1C4A40F25F11D0E79DF803305B008F
:10E14000DBB28DF8033001212346E7E74FF480630B
:10E150001360019B174ADBB213701A4B1A6842F422
:10E1600060021A601A6842F060421A60FFF788FF86
:10E17000154B00241C60FFF799FE144A136843F006
:10E1800040431360FFF77EFEFFF704F8FFF798FEA9
:10E19000204602B010BD00BF00ED00E071C20F418B
:10E1A000E297040031990400D296040070C20F4136
:10E1B0002498040000E400E0503F0020543F002079
:10E1C0006698040020ED00E0E411002034EF00E048
:10E1D00008B5EFF305830F2B0CD90D4A9B5C0D4A54
:10E1E00012789A4206D90C4B0C4A4FF43F710C48F6
:10E1F000FDF7FCF80B4B0C4A1B68126803F4E06354
:10E20000934204D9094B054A4FF44371EFE708BD27
:10E21000F0E300E0503F0020989804006A99040061
:10E22000D29604000CED00E0543F0020C498040096
:10E2300000F108034FF0FF32C0E90223436003619D
:10E2400000230360704700230361704743684B60FD
:10E250009A688A60516099600861036801330360BD
:10E26000704730B50C68631C0AD103695A684A606C
:10E2700091608B605960086103680133036030BDB1
:10E2800000F10802134652681568A542FAD9EDE775
:10E29000D0E9011203698A60416851605A6882427C
:10E2A00004BF82685A60002202611A68013A1A604B
:10E2B00018687047014B986C00F038BC783F00201C
:10E2C000024A034607CA83E807007047643F0020FC
:10E2D000F0B5204F3D7889B0002D38D11E4C204636
:10E2E00000F082FA012604A8A560C4E92665A4F816
:10E2F000A05084F8A250C4F8946000F001FB4FF0E5
:10E30000FF331649069304AA04F10C0000F000FB49
:10E31000A06401A800F0B0FC0A2301AA10490393ED
:10E3200004F1500000F022FDC4F8900000F0ACFCB5
:10E330000C4DC4F89C002946D4F8900000F070FD04
:10E340006A68094BB3FBF2F3084A3E70136009B0E8
:10E35000F0BD00BF703F0020783F002049E400007E
:10E36000B5E200002040002040420F00284000207D
:10E3700038B500F0D7F9064B05460021D3F89000D8
:10E3800000F054FD0446284600F00EFA204638BD41
:10E39000783F002070B500F0C5F90A4E054600210F
:10E3A000D6F8900000F042FDD6F898301C1AD6F846
:10E3B0009C302846A34238BF002400F0F5F92046DF
:10E3C00070BD00BF783F002070B5064D04460E4674
:10E3D0000146D5F8900000F083FCC5F89440C5F8DC
:10E3E000986070BD783F00202DE9F8430746154836
:10E3F000DFF850900D4600F00CFA4FF0FF3604465F
:10E400004C4502D13046BDE8F883204600F003FABF
:10E41000237D804683B147B1E368AB4205D12369D0
:10E4200063B92375D4E906309847237D23B1E368A7
:10E430005B1B9E4228BF1E464446E1E72B44E36037
:10E44000F0E700BF783F00202DE9F84300F06AF9BB
:10E45000DFF89C8081460121D8F8900000F0E6FCAE
:10E460000123D8F80820D8F89850A8F8A030D8F898
:10E470000830AA1AC31A9A4247464FF0000406D938
:10E4800088F8A0404846BDE8F84300F08DB9461B27
:10E49000484600F089F9254429460120FFF7A4FFEA
:10E4A000B146361B8642A0460446F4D200F03AF943
:10E4B00097F8A130064623B129460020FFF794FFC4
:10E4C0000446631CD7F89C000BD12918FFF77CFF8A
:10E4D000012387F8A230002387F8A030BD603046C2
:10E4E000D1E7A8EB09084444A04228BF2046ECE746
:10E4F000783F002038B5054600F014F90446284658
:10E5000000F09AF92046BDE8384000F04DB910B54A
:10E510000446FFF7EFFF2046BDE81040FFF7A1BB20
:10E52000F8B51C4D044600F0FDF895F8A2300646FB
:10E530002F460BB395F8A030F3B90121D5F8900020
:10E5400000F074FCA968D5F898200346A868591A09
:10E55000121A914210D8A0680122C118E1602275F8
:10E56000D5F89820D31A984201D2FFF72DFF3046F4
:10E57000BDE8F84000F018B9FFF7FAFEA3681844A8
:10E580000123E060237597F8A020002AEFD087F8D8
:10E59000A130ECE7783F0020F8B50E4617461D463F
:10E5A0000446B0B1FFF794FE0B4B0C48002D08BF9A
:10E5B0001D4621466B682361A760A661AB68E361D5
:10E5C0000023237500F029F92B7813B12046FFF7BB
:10E5D000A7FF2046F8BD00BF643F0020783F002021
:10E5E00037B5044620200D460192FFF7FBFA019B48
:10E5F0002A46214603B0BDE83040FFF7CDBF0023D7
:10E6000003757047816070470161704710B5037DE5
:10E6100023B1C468FFF7ACFE201A10BD8068FCE788
:10E62000007D70470A20704738B5FFF751FE00F0B3
:10E6300079F8064B05460021D3F8900000F0F6FB70
:10E640000446284600F0B0F8204638BD783F002048
:10E6500008B54FF0E023094AD3F8043DDBB252F885
:10E66000233053B1D3E901209047054B4FF080523E
:10E670001A60BFF34F8FBFF36F8F08BD2C4000208F
:10E6800004ED00E0F0B50E4685B01C46054618B90D
:10E690000025284605B0F0BD53B901934FF0FF3374
:10E6A000029301238DF80C3001ACC023636002E0BB
:10E6B0001B79FF2BF9D0104B1B68B34202D0636863
:10E6C000E02BE5D00D4B6A6043F826500C4F2368D1
:10E6D0000C49AB6030462E6037F0D2FF3B682179A1
:10E6E0009B6830469847237A002BD2D03B6830464F
:10E6F0001B699847CDE700BFE81100202C4000209F
:10E70000B001001051E6000010B5054B1B6804462F
:10E710005B69006898472068BDE8104037F0CABFC1
:10E72000B001001010B5074B1C6814F0FF0403D1B2
:10E73000FFF718FC204610BD2023EFF3118483F36C
:10E740001188F7E704ED00E0014B1B681B691847CF
:10E75000B0010010034B1868C0B2003818BF012088
:10E76000704700BF04ED00E0044B054A1B681068C9
:10E77000DBB2C31A58425841704700BF04ED00E0B5
:10E78000E811002030B14FF0FF330022C0E9002330
:10E790000123037270470F28C2BF4FF0E0231038E7
:10E7A000C3F8000F70470000044B1B6813F0FF0F05
:10E7B00001D1FFF7FDBB80F31188704704ED00E045
:10E7C00070B504460E461546FFF7ACFFC4E9016577
:10E7D000BDE87040FFF7E8BF024B1B68C9B29B68F9
:10E7E000184700BFB0010010406000607047036828
:10E7F000C31A58425841704738B50446FFF792FF94
:10E8000025682B6823602B685C60FFF7CDFF2846E6
:10E8100038BD006870470068704738B50D4604463B
:10E82000FFF780FF2C6063686B6063681D60656044
:10E83000BDE83840FFF7B8BF436802681A60036854
:10E8400042685A60704737B503220092002203469F
:10E850000D4601201146FDF799FA044628B125B16D
:10E8600000231A461946FDF73DFB204603B030BD94
:10E8700038B50322054600210120FDF7D1FA0446F0
:10E8800028B125B100231A461946FDF72BFB204677
:10E8900038BDFDF76DBF704738B505460C46FFF72C
:10E8A00059FF48B1002211462846FDF707FF0138FD
:10E8B00018BF4FF0FF3038BDFFF7B4FEB0F57A7FD8
:10E8C00007D0A4FB00014FF47A720023FBF7B8FED7
:10E8D000044621462846FDF769FDE8E713B50446DE
:10E8E000FFF738FF034630B9024601462046FDF7E0
:10E8F000F9FA02B010BD01A92046FDF759FCF8E76E
:10E9000000234FF0FF32C0E90033C0E90223704713
:10E910002DE9FF47884615460446002851D0DFF808
:10E92000DC90FFF7FFFE99F80030064603F0FF0782
:10E9300023BB2648FFF758FF2548FFF755FF25481A
:10E94000FFF752FF2448FFF74FFF244B1F60244B73
:10E950001F60244B4FF0010AC3F800A0224B01A80E
:10E960001F70FFF70FFF2149214A09682148E02362
:10E97000029301ABFFF786FE89F800A03046FFF74F
:10E9800013FF1D4B002D08BF1D46AF687B1C03D035
:10E99000032F02D9002414E003272046FFF724FFA9
:10E9A00095E80F0004F10C0686E80F00A3692362C6
:10E9B00000236362054B676103EBC707C4F81C8043
:10E9C000A760204604B0BDE8F08700BF2C410020BE
:10E9D000344100203C410020444100204C410020B3
:10E9E000044100202841002050410020E81100206F
:10E9F00005EB0000084100208C9904002441002010
:10EA000038B50446FFF78EFE05462046FFF714FF93
:10EA1000A068FFF7ECFE38B1064960690B68012277
:10EA2000824023EA02030B602846BDE83840FFF726
:10EA3000BBBE00BF4C41002010B5FFF773FE044B76
:10EA40001C6800221A60FFF7AFFE204610BD00BF11
:10EA5000284100202DE9F047DFF8A0A0DFF8A090C2
:10EA60000546D046DAF800301BB1D9F80030012B4A
:10EA700004D01F4B00221A70BDE8F087DAF800209E
:10EA80000326082312EA030105D1013E701C4FEA58
:10EA90006303F7D10E46174F07EBC6073846FFF75B
:10EAA000ABFE04463846FFF7A2FE40B1D8F800306E
:10EAB000012202FA06F623EA0606C8F800600223DD
:10EAC00063620D4B226A1A60A36923622846FFF72E
:10EAD0006BFEE369D4E903019847FFF723FE636AFD
:10EAE000022B08BF0023054608BF6362BAE700BFD8
:10EAF000504100202C410020044100204C410020C6
:10EB00002841002010B5FFF70DFE0446FFF7A2FFD5
:10EB10002046BDE81040FFF747BE0000014B1868D3
:10EB2000704700BF04410020FFF71EBE70B50446C9
:10EB3000FFF7F8FD636A012B06460ED00F4B6069A4
:10EB400001256562214603EBC000FFF766FE0C4B12
:10EB500061691A688D4015431D600A4C237843B9DA
:10EB6000094B1D68012D04D1084B1868FFF713FEEF
:10EB700025703046BDE87040FFF716BE2C410020DE
:10EB80004C4100205041002028410020E811002085
:10EB900038B504460D46FFF7C5FD236A2B432362B3
:10EBA000FFF702FE2046BDE83840FFF7BFBF000078
:10EBB00070B50446FFF7B6FD0A4B1C600A4B1B6894
:10EBC00005464BB1012C07D1084E337823B9084BC9
:10EBD0001868FFF7E0FD34702846BDE87040FFF785
:10EBE000E3BD00BF284100204C41002050410020DF
:10EBF000E81100204B1C02D0032901D970470321E2
:10EC0000024B416103EBC101816070472C41002040
:10EC100070B5134B134C1D6823684BB1124B1B6826
:10EC200033B1124B4FF480721A6023680120984769
:10EC3000636843B10E4A12682AB10C4A4FF480311E
:10EC40001160022098470B4B1B683BB1074B012218
:10EC50001A60D5E90203BDE87040184770BD00BFD7
:10EC60005C41002054410020A000244304200940BE
:10EC7000C000244380002443024A034607CA83E8B5
:10EC800007007047EC11002008B547F69061D0E905
:10EC900006230020FBF7D4FC0B46002102469942D4
:10ECA0004FF0FF3008BF904238BF0246104608BD03
:10ECB000094B1B68CA1AB2F1004F03F1040303D9D0
:10ECC0001946064B196070475A1A002AF9DB994217
:10ECD00038BF1946F5E700BF302009401820094029
:10ECE00070B5D0E90625A2FB012301FB0533D0E96D
:10ECF0000816551843EB0606290C002241EA064186
:10ED0000FFF7D6FFC0E90A5670BD000038B50546CA
:10ED1000FFF708FD6B680C4AB3F5802F2CBF1B0C66
:10ED200004231360094B1B6804461B680020232141
:10ED30009847074A01231360064A13602046BDE83E
:10ED40003840FFF731BD00BF182009408401001092
:10ED50000420094080022443034B186818B103784B
:10ED60000BB9FFF7D3BF70475C4100202DE9FF418D
:10ED70000E461546044600283BD0DFF89480FFF786
:10ED8000D1FC98F8003007467BB901A8FFF7FAFCE0
:10ED900080230293194A1A4801AB1421FFF772FC31
:10EDA000184B1C60012388F800303846FFF7FCFC44
:10EDB000154B164A002D08BF1D462B7823706B6833
:10EDC000C4E9023600264FF48033C4E904633046B8
:10EDD000A9680023FBF734FC00220023C4E90606DF
:10EDE000C4E90823C4E90A06C4E90C066060FFF719
:10EDF000B3FF204604B0BDE8F08100BF11EC000075
:10EE0000604100205C410020EC11002040420F00D6
:10EE10007C410020014B1B681B6B18478C010010C4
:10EE200000234FF48032C1E900327047F8B505463F
:10EE30000F46FFF7EFFFD5E9064622463346FBF7BC
:10EE4000FFFB3FB16143A4FB002306FB00110B4411
:10EE5000C5E90823F8BD0000F0B5072898BF0820D1
:10EE6000C31C2148214D8468002223F0030308338A
:10EE70002A6011468446644505D102B12960604587
:10EE800012D100201FE066688E4284BF3146012205
:10EE90009E4205DB604505D04768BE42B8BF2046AC
:10EEA000A468E8E72046FBE74168994219DBCA1AE3
:10EEB000102A09DD8118426082505A424A600022BD
:10EEC000CA5001F10800F0BDD0E902239A60D0E9F0
:10EED0000232DA6043685B424360002343500830EB
:10EEE000F1E78068CBE700BFF811002080410020E7
:10EEF00050F8082CA0F10803BAB19B1A50F8041C72
:10EF00005A68521A5A605A681A445168002909DD31
:10EF1000D2E902108160D068C860596852680A441A
:10EF20005A601A445B6813607047064A0260D168F1
:10EF30004160D3604268936050F8042C524240F81C
:10EF4000042CE0E7F811002000230360084B8360E5
:10EF5000DA68C260D860C36821F00301083998609C
:10EF600043184FF00042416041505A60704700BF63
:10EF7000F811002010B5FFF75FFD002460F30F04C7
:10EF8000FFF7D0FB60F31F44204610BD07B501908A
:10EF9000000CFFF709FCBDF80400FFF709FE03B001
:10EFA0005DF804FB38B50446FFF7E4FF054620464C
:10EFB000FFF752FF04462846FFF7E8FF204638BD1A
:10EFC00038B50546FFF7D6FF04462846FFF790FF01
:10EFD0002046BDE83840FFF7D9BF704737B50B462C
:10EFE00011F00101054614465ED000211C2031F0CD
:10EFF00089FF00211D2031F085FF00211E2031F006
:10F0000081FF284636F00CFF2388B3F5C15F4FEA35
:10F01000D07007D043F60702934216D040F60202A2
:10F02000934227D1E37B5A0624D0002180B11C20D3
:10F0300031F054FF32211D2031F050FF2F211E20CE
:10F0400003B0BDE8304031F049BF94F82430EAE71E
:10F050001C2031F043FF00211D2031F03FFF002133
:10F060001E2031F03BFF01211E2003B0BDE83040DF
:10F0700031F048BF48B12F211C2031F02FFF322141
:10F080001D2031F02BFF0021D9E700211C2031F099
:10F0900025FF00211D2031F021FF00211E2031F02D
:10F0A0001DFF01211C20E0E79B0715D51C200191C5
:10F0B00031F028FF01991D2031F024FF01991E2015
:10F0C00031F020FF01991C2031F008FF01991D202B
:10F0D00031F004FF0199B2E703B030BD70B50446CA
:10F0E0000D461646FFF779FF324629462046FFF7C0
:10F0F00075FF70BD38B500210546142031F002FFC0
:10F10000072400210A2031F0FDFE45FA04F101F048
:10F110000101092031F0F6FE01210A2031F0F2FE52
:10F12000082037F0C3FB013CEBD200210A2031F06C
:10F13000E9FE1420012131F0E5FEBDE838404FF42E
:10F140002F7037F0B3BB000008B50A49142031F026
:10F1500073FE0021142031F0D5FE012037F0A6FB0C
:10F160001420012131F0CEFEBDE808404FF40C70B0
:10F1700037F09CBB0162002008B5FFF7E5FF10499E
:10F18000142031F059FE0F490A2031F055FE0D4987
:10F19000092031F051FE0C49082031F04DFEB92014
:10F1A000FFF7A8FF14202CF05FFF0A202CF05CFF73
:10F1B00009202CF059FFBDE8084008202CF054BF6E
:10F1C000016200200062002002200020704708B584
:10F1D00032F0EEFA31F0AAFDFFF7CEFFFFF7F6FFAF
:10F1E00008BD036813F0060F14BF0120002070470C
:10F1F000006810F0010018BF01F00100704708B569
:10F20000FFF7EFFF20B111F0060F14BF012000201F
:10F2100008BDC36A13F0060F14BF01200020704719
:10F2200070478B680120D3E9001210471FB50F4BC0
:10F230000C461B6803934FF0000391B1002201A913
:10F24000104627F055F928B9D4F8B030D4F8B400F6
:10F2500001A99847054B1A68039B5A4004D037F020
:10F2600061FF6FF00800F5E704B010BDD09A04000C
:10F2700008B508461278002137F0E4FD002008BDEB
:10F280000DF0C8BBF0B52C4B89B01B6807934FF04D
:10F29000000350F8D03CDB07A0F1D00542D5D5F8EB
:10F2A000C0300A685B689A423CD10022234C01AF0F
:10F2B0003946104627F01CF9214821462CF0CDFA9A
:10F2C000064638B197E8030084E80300EB69013390
:10F2D000EB6110E0394603A822462CF017FB3C23D3
:10F2E00005A903A8CDE905362CF0A7FA0028EDD032
:10F2F000C4E90066EE61EB69092B13D92CF086F89E
:10F30000012804D90F4A012102202CF085F8D5F8F4
:10F31000C000836800215B69083098470023C4E976
:10F320000033EB61044B1A68079B5A4001D037F059
:10F33000F9FE09B0F0BD00BF009B0400844100202D
:10F34000589E0400D49A040030B5204B056887B05D
:10F3500004461422002168461B6805934FF0000301
:10F3600037F070FDD5F8C030E26804339A421FD000
:10F37000D5F8C43004339A421CD12B689A071BD4A9
:10F3800003F004030093E3798DF8043094F9060048
:10F39000A388ADF80C30AB6880B9DA6819686846A4
:10F3A00090470A4B1A68059B5A400CD037F0BAFEBA
:10F3B0000123E7E70023E5E70223E3E71C691A6876
:10F3C0006946A047EDE707B030BD00BF049B0400CD
:10F3D000D0F8C4306BB103691B7953B103689B0744
:10F3E00007D5D0F8F000036809B1DB6A18471B6B3A
:10F3F000FCE7704710B524F075F90368BDE81040CC
:10F40000DB6818472DE9F34104460D46FFF7F0FE8F
:10F41000A0B92046FFF7E5FE30B12368DB0703D42F
:10F4200094F8283042B14BB929462046FFF7E7FE51
:10F4300020B902B0BDE8F081002BF5D1E36A002AC3
:10F440003AD02B43012DE36239D1002A37D1226310
:10F45000D4F8A400FFF7CEFFE36AD4F8C01013F08D
:10F46000010F054614BFC826002631B10368324695
:10F47000DF68B4F8C8300431B8472046FFF7C9FE4A
:10F48000D4F8C410002814BF6427002741B12B68AA
:10F490003A46D3F80C80B4F8CA3004312846C04745
:10F4A0002BF0B4FF0128C4D902210E4A009733463D
:10F4B00008462BF0B1FFBCE723EA0503C2E7294663
:10F4C0002046FFF79CFE0028C2D094F8E81004EB19
:10F4D00081010B6B1AB143F001030B63B8E723F012
:10F4E0000103FAE7089B040010B524F0FBF8036859
:10F4F000BDE810401B6918472DE9F0472A4B044628
:10F50000D0F8C00086B00D461B6805934FF000038D
:10F5100030B183685E6B08230A4618441121B04756
:10F52000D4F8C43023B1D4F8CC0029460AF0EFFB5C
:10F53000D4F8A40024F0D6F800278146D4F8A4001B
:10F54000FFF7D2FFCDE9027702238DF80830049748
:10F55000036802AE80460096D4342146D3F804A056
:10F5600004AA3B46D047D8F80030009604AA1E688B
:10F5700029463B464046B047D9F8003029465B69EA
:10F580004846984728460DF05FF928686968064B99
:10F5900003C41A68059B5A4001D037F0C3FD3846B2
:10F5A00006B0BDE8F08700BF189B0400FFF7A4BFBA
:10F5B0007FB52B4B1B6803934FF000038369044610
:10F5C000002B44D090F8E53013B1002380F8E530EB
:10F5D00001A9D4F8CC000AF080FB0025D4F8CC00B7
:10F5E0008DF802500DF102010AF032FB9DF8023055
:10F5F000D4F8C0005B1B18BF01238DF8033070B135
:10F60000836809215E6B0DF1030201230830B047C6
:10F61000D4F8C000836829465B690830984723699D
:10F620001B7953B1D4F8C4303BB123689B0704D590
:10F63000D4F8F00003685B6A98479DF8033013B96B
:10F64000012027F007F901A92046FFF755FF044BD9
:10F650001A68039B5A4001D037F064FD04B070BDB6
:10F660001C9B040058B151B14BB1C0E92C328369E5
:10F6700043B10A4600F18C013C3020F0C8BF6FF066
:10F6800008007047184670472DE9F04FADB05A4B4F
:10F690005A4F054600240DF15C0B50222146584676
:10F6A0001B682B934FF00003129437F0CBFBD5F877
:10F6B000A400FFF719FF8046D5F8A400FFF79AFED3
:10F6C000022304948DF810302B68059413F0020F78
:10F6D0000DF1100906463ED0C8233B803B88A5F8B3
:10F6E000CA3013AC2146D5F8CC000AF0F6FAD5F8AA
:10F6F000F000036859465B68984703AA0021D5F8D3
:10F70000CC000AF04BFB102200210EA837F09AFB28
:10F7100005F13C0AD5F8A400CDF834A0CDE90B746E
:10F7200023F0E2FF0223CDE90E0B039A10930BA9FD
:10F7300005F1C4000BF09CF9044680B1304A034641
:10F74000012100202BF068FE2B4B1A682B9B5A409E
:10F750004ED037F0E7FC5B07C0D51323BDE7D5F8E3
:10F76000C400836821465B6808309847254A1068C2
:10F77000516815AB03C3D8F80030CDF80090D3F82A
:10F78000009012AA234615A94046C84704460028FF
:10F79000DAD1D5F8C410336804311B683046984775
:10F7A000044610B1184A0346CAE73368D5F8C410B6
:10F7B000DC683B88642204313046A047044610B11F
:10F7C000124A0346BCE72B691B78002BBCD0D5F846
:10F7D000CC300693D5F8A4300D49CDE9090006AA2E
:10F7E00005F1F400CDE9073A04F024FF0446ABE745
:10F7F00020462DB0BDE8F08F889B04003014002017
:10F80000209B0400647E0400499B0400699B040063
:10F81000A09E0400002270B504460D46012011464A
:10F8200026F066FEE36A003818BF012084F829003C
:10F830004BB3228D3ABB84F8242094F8E6207AB3A7
:10F84000A2696AB3BDB1E968226B914213D12969FB
:10F85000626B91420FD1A16B6A6991420BD194F80E
:10F8600024102A78914206D1AA68934203D1228DAE
:10F87000AB889A4214D0A36804F124005A6919682D
:10F88000BDE87040104794F8E5203AB1DA0705D595
:10F8900094F82820012A01D10322CCE70122CAE7EB
:10F8A00070BD0000F0B5154B89B000F124051B6850
:10F8B00007934FF0000306468C4617460FCD01AC68
:10F8C0000FC495E80300D6F8C43084E803000BB1F8
:10F8D00063450AD13168304601F006013A46FFF728
:10F8E00091FD01A93046FFF795FF044B1A68079B6D
:10F8F0005A4001D037F016FC09B0F0BD8C9B0400D3
:10F9000070B5154B88B000F124061B6807934FF0C3
:10F91000000304460FCE01AD0FC596E80300A369AE
:10F9200085E8030073B1236B012243F00203114603
:10F93000204684F8E5202363FFF764FD01A92046F3
:10F94000FFF768FF044B1A68079B5A4001D037F055
:10F95000E9FB08B070BD00BF909B0400F0B58DB00E
:10F960002D4B8DF8071000F124061B680B934FF008
:10F97000000304460F460FCE05AD0FC596E8030001
:10F9800087F0010385E8030084F8283038460CF03E
:10F9900065FED4F8C00038B183680DF107025D6BD5
:10F9A000092101230830A847236973B11B7963B18A
:10F9B000D4F8C4304BB123689B0706D5D4F8F000C7
:10F9C0009DF8071003689B6A98479DF80730BBB104
:10F9D0002B21072304F1D502012026F0F9FED4F8EB
:10F9E000CC0004F1D4010AF092F905A92046FFF7F2
:10F9F00011FF094B1A680B9B5A400BD037F092FB52
:10FA000003A9D4F8CC000AF068F903A92046FFF74F
:10FA100073FDEAE70DB0F0BD949B040070B5424B56
:10FA20008CB000F124061B680B934FF000030446D2
:10FA30000FCE05AD0FC596E8030085E80300D4F8A6
:10FA4000C40058B123691B79002B64D023689A073E
:10FA500061D5D4F8F00003681B6A984703A9D4F86D
:10FA6000CC000025CDE903550AF037F903A80CF0C6
:10FA7000F7FE03A92046FFF73FFDD4F8C00008B306
:10FA8000836829465B6908309847D4F8C0008368CA
:10FA900008215E6B2A462B460844B047D4F8C000C4
:10FAA0008DF80450836801AA5E6B09210123083098
:10FAB000B047D4F8C00083682A465E6B07212B4606
:10FAC0000830B04740F201120023228501AAE36208
:10FAD00011460120CDE9013326F020FD23691B7971
:10FAE00053B1D4F8C4303BB123689B0704D5D4F894
:10FAF000F0000368DB69984705A92046FFF78AFEF6
:10FB0000A3689A6918689047074B1A680B9B5A407C
:10FB100007D037F007FB836800215B6808309847FF
:10FB20009CE70CB070BD00BF989B040037B5164B26
:10FB300005466A460846002402211B6801934FF0DF
:10FB40000003009420F0D2FED5F8C030009A0433B0
:10FB50009A4210D0D5F8C43004339A420DD12868A7
:10FB600083070CD400F00400074B1A68019B5A402D
:10FB700007D037F0D7FA0120F6E72046F4E7022055
:10FB8000F2E703B030BD00BF9C9B040008B5D0F87D
:10FB9000C4305BB103691B7943B1036813F00203FE
:10FBA00004D0FFF7C3FF821E53425341184608BDDD
:10FBB000F0B5254B8BB000F124061B6809934FF07C
:10FBC000000304460F4694460FCE03AD0FC596E8DA
:10FBD00003002368DB0785E8030021D56146204642
:10FBE000FFF7A4FF012805461AD127B3236B43F082
:10FBF00001032363024601462046FFF703FC94F805
:10FC0000E4306BB10023CDE90133D4F8C00084F8AF
:10FC1000E43083688DF808505B6901A90830984783
:10FC200003A92046FFF7F6FD074B1A68099B5A40C7
:10FC300007D037F077FAD4F8C000836839465B699B
:10FC4000ECE70BB0F0BD00BFA09B0400F8B50F4679
:10FC50001946154606461C46FFF768FF0023012893
:10FC600014BF96F8E8201A460C343A6006F1DC011D
:10FC70002B60204626F0FBFC10B101232B60F8BD61
:10FC80000849204626F0F3FC08B10223F6E72BF0E2
:10FC9000BDFB0128F1D9044A012102202BF0BCFB55
:10FCA000EBE700BFA89E0400A49B0400F0B58DB054
:10FCB000254B8DF8072000F124061B680B934FF0AD
:10FCC000000304460F460FCE05AD0FC596E80300AE
:10FCD00085E80300EFB139462046FFF727FF0128EA
:10FCE00018BF216802460EBF0146012201F006013D
:10FCF0002046FFF787FB3B4603AA04A92046FFF7EF
:10FD0000A5FF9DF81030039904EB83031A6B0A4397
:10FD10001A6305A92046FFF77DFD94F8283053B9F2
:10FD2000D4F8C00038B183680DF107025C6B06217E
:10FD300001230830A047044B1A680B9B5A4001D09E
:10FD400037F0F0F90DB0F0BDD09B0400F0B5474B93
:10FD500089B007461B6807934FF00003A0F1EC043D
:10FD6000114652B1012A7BD06FF005003F4B1A6853
:10FD7000079B5A4078D037F0D5F9A0F1C8060FCECE
:10FD800001AD0FC596E8030057F8EC3CDA0785E8AB
:10FD9000030002D5A369DB0702D494F8283043B1ED
:10FDA000D4F8C00083685D6B00231A460721083031
:10FDB000A84794F8E53013B1002384F8E5300CF03F
:10FDC0002CFD08B10CF026FD0CF031FD08B10CF053
:10FDD0002BFD2046FFF705FA002836D0A36913F063
:10FDE000060F32D094F828307BBBD4F8C030A3B1D2
:10FDF00057F8EC5C15F001050FD1D4F8A400FFF71B
:10FE0000F9FAD4F8C010036804319B689847D4F815
:10FE1000C00003689847C4F8C0502046FFF7F9F9BE
:10FE200098B9D4F8C43013B92046FFF72DFCD4F8A4
:10FE3000C400836801215B6808309847D4F8C40087
:10FE4000836801219B6808309847012120460022E1
:10FE5000FFF7D8FA01A92046FFF7DCFC002085E770
:10FE60002046FFF7CFFAF9E709B0F0BDD49B0400B4
:10FE70002DE9F04F2DED028BC1B0A44B03911B680F
:10FE80003F934FF00003804608B301B38368F3B19A
:10FE90005A68E2B19A68D2B1DA68C2B11A69B2B1ED
:10FEA0005A69A2B19B6993B14168994BA1F5E1529E
:10FEB0009A420CD8036953B11A795AB19B685E1CF7
:10FEC00017D0944AA3F52843C03B934211D96FF051
:10FED0000A0406E0036803F00303022B09D16FF064
:10FEE00005048A4B1A683F9B5A4000F03F8237F066
:10FEF00019F9894A9162D8F8003013F0040F92463C
:10FF0000EDD19D07EBD06FF000429342E7D003F0B4
:10FF10000603062BE3D0814E96F814C03546BCF19B
:10FF2000000F40F0208244460FCC37460FC77C4973
:10FF300023683B60324606F13C00C6F818C020F04A
:10FF4000A3F97849324606F18C0020F0CDFA764AC2
:10FF500092E8030006AB83E8030007F1A800194606
:10FF600024F01AFF2C3704460028BAD101461C227F
:10FF70002BA836F067FF06F1D0032C93D6F8B830E3
:10FF80002D936A4B6A4A2BA906F1A400CDE92E36BF
:10FF900023F01EFB044630B1664A034601210020CF
:10FFA0002BF03AFA9DE7D6F8A40023F09BFB83469A
:10FFB000D6F8A400FFF798FA2394DBF800308146C6
:10FFC0005B69584606F1D4019847CDE908440222FE
:10FFD0008DF82020D9F8002008AB0093D2F800B0AB
:10FFE000234623AA06F1D4014846D84706F1D40B8C
:10FFF000044610B1504A0346D0E7D6F8A4304F4922
:020000021000EC
:10000000324606F1BC0020F067FC044610B14C4AB1
:100010000346C3E7CDE90A00D6F8BC0083680AA905
:100020005B6808309847044610B1464A0346B5E776
:100030003A48FFF7D6F82B68DC0721D4002834D1E2
:10004000414BD5F8A40000264FF00109CDE90C364C
:100050008DF8359023F042FB044624A823F0C7F81E
:100060000823ADF8A03023682046DB680CAA24A939
:1000700098470446002800F09180344A03468DE7F3
:1000800098B9D5F8A4400146242217A836F0DAFE24
:1000900021492F4815AACDE9157409F0A9FE044697
:1000A0000028CDD02B4A034678E7D5F8A4602A4C27
:1000B0002A4B23602422002117A836F0C3FECDE985
:1000C00015762B6920941A791AB19A68501C18BFBA
:1000D00062611B7923762B6813F0020248D0204B13
:1000E000012283F824200023CAF800300A491D4861
:1000F0004C2236F07FFE1A491B4815AA02F09AF8E6
:10010000044600283DD0194A034647E7549D0400A1
:10011000601E090077E0400034140020A012002087
:1001200023F200002DF200006C7E040065F6000052
:10013000709E0400D89B0400F49B0400609E0400A1
:10014000129C0400359C0400E0930400AE9C040063
:100150006C130020579C04008014002081F20000E2
:10016000A4130020E413002090130020779C0400C7
:10017000590741BF804BCAF80020022183F82410A0
:10018000B4E7D5F8F0007D4903689B6898470446BA
:1001900000283FF455AF7A4A0346FFE679498DF8C7
:1001A0001700D5F8CC0009F098FD0DF11701D5F82E
:1001B000CC0009F04DFD9DF817308DF8C990003B3B
:1001C00018BF01238DF8C8302B688DF8CA9003F052
:1001D00001039BE8030083F001038DF8CB303C233F
:1001E000CDE9333735AB83E80300674B3893674B72
:1001F0003993674B3A93674B3B93674B3C93674B01
:100200003D93D5F8A4103795032332A88DF8F83024
:100210000CF048FB064638B10346614A2046494681
:100220002BF0FAF834465CE62146342216A836F064
:1002300009FE5C4B17935C4B1A935C4B1C935C4B15
:100240001D93D5F8CC005B4B159515A91E9309F0AD
:100250008FFD04465848FEF7C4FF18B1D5F8C430E6
:100260005BB300242B689DF81760DA0704D44EB9FD
:10027000D8F800305B0705D5D5F8C090B9F1000F6C
:1002800023D000249DF817304B48B3FA83F30122A2
:100290005B092A7585F8283085F82920FEF7A1FF2B
:1002A00040B1D8F8003013F0040F14BF022301232B
:1002B00085F8E830039B1D6013E63F48FFF7E4F93B
:1002C000044600287FF40DAECBE7D5F8A40023F058
:1002D0000BFAEB68394ACDE9103721238DF84A3003
:1002E0004B23003E8DF84C306B681493CDE90E0B18
:1002F000334BC5F8EC3018BF0126C8270EA9A2F170
:100300002C00ADF848708DF84B6004F007FA0446F5
:1003100010B12C4A034641E6D5F8A400FFF76AF86D
:10032000D5F8C010036804311B6806469847044698
:1003300010B1254A034631E6D5F8C0002349836849
:1003400008309B6998473368D5F8C010DC68B5F869
:10035000C8303A4604313046A0470446002890D0C1
:100360001B4A03461AE66FF01904BAE5204641B06D
:10037000BDEC028BBDE8F08FA41300206C130020AD
:10038000939C040074130020ADF50000B1F500004B
:10039000B1FB000001F900008DFB0000D1F300006B
:1003A000CE9C040071F200001DFA00005DF900000F
:1003B000ADFC0000A5F80000A01200208C13002066
:1003C00084120020E99C0400129D040068130020A0
:1003D000329D0400F0B5554B87B00E461B6805935F
:1003E0004FF000030546002800F09880037D002BA5
:1003F00000F09480002900F0918003688B42C0F0E7
:100400008D800B4000F08A806FF00042914208BF5F
:100410001E46826936EA020300F083803146FEF709
:10042000EEFE00284CD012F0060F49D1D5F8C400DA
:10043000836801215B68083098470446002849D149
:10044000D5F8C400836801219B68083098470127CC
:1004500031462846FEF7CCFE28B995F82830012B06
:100460003FD171073DD5AB69DA073AD4D5F8C00062
:10047000836801215B6808309847044620BBAB695C
:100480003343AB6100242B68B3422DD1002201A974
:10049000104626F02DF80446E0B905F1F80101A850
:1004A0002BF012FA019BB3F5E15F1DD303AA1146AD
:1004B0000120CDE9034426F031F8A8B1044609E053
:1004C00000276FF02704C3E70346194A01210020E3
:1004D0002AF0A2FF154B1A68059B5A4023D036F02C
:1004E00021FE002CCFD1CAE7012385F8E630002198
:1004F0002846FFF78FF92B691B79002BEAD0002FD4
:10050000E8D02B689B07E5D595F82830012BE1D181
:10051000D5F8F0000368DB699847CFE76FF00A046D
:10052000D8E70024D6E7204607B0F0BD709D040050
:10053000589D040070B50E460446002800F0AE80B9
:10054000037D002B00F0AA80002900F0A78003683B
:100550008B42C0F0A3800B4000F0A0806FF00042FF
:10056000914208BF1E463146FEF742FE28B920469A
:10057000FEF745FE002800F09180A56916EA050007
:1005800000F08F80002384F8E63031462046FEF7E5
:100590002FFE28B994F82830012B13D1700711D5FC
:1005A000D4F8C00070B1836800215B6808309847B8
:1005B000054638B13C4A0346012100202AF02CFFB1
:1005C000284670BD31462046FEF719FED8B1236992
:1005D0001B795BB12368990708D594F82830012B63
:1005E00004D1D4F8F00003681B6A9847D4F8C4001B
:1005F00048B1836800215B6808309847054610B110
:100600002A4A0346D8E731462046FEF7F1FD50B1AD
:10061000E36A23F00103E362236B23F00303236304
:100620000023A4F8E43031462046FEF7E8FD98B1F7
:10063000B20742BFE36A23F00203E362730742BFDB
:10064000E36A23F00403E36294F8E83004EB8303E5
:100650001A6B22F003021A632368B3420CD0012301
:10066000002184F8E6302046FFF7D4F8A16921EA9A
:100670000601A1610025A3E704F13C001FF0E5FE9F
:10068000054610B10A4A034696E7024604F1F8010E
:1006900025F02EFF05460028E1D091E76FF00A050E
:1006A0008EE705468CE700BF749D0400939D04000F
:1006B000B29D040010B53C4B86B01B6805934FF00B
:1006C00000030446002867D0037D002B67D090F814
:1006D000283033B903AA11460120CDE9033325F0B0
:1006E0001DFF21682046FFF725FF0CF0CBF8D4F85A
:1006F000BC00836808301B689847D4F8C00020B15C
:10070000036898470023C4F8C03023691B7843B1BD
:10071000D4F8F40028B103681B6898470023C4F894
:10072000F430D4F8C40020B1036898470023C4F81B
:10073000C430D4F8F00038B103681B689847002330
:10074000C4F8F030C4F8CC30D4F8CC0020B109F0B3
:1007500029FB0023C4F8CC30D4F8A40022F0A8FF71
:1007600004F13C0004F18C0101901FF043FF01985B
:100770001FF0A4FED4F8B80008B124F039FB002023
:10078000C4F8C80084F8E8002075074B1A68059B78
:100790005A4007D036F0C6FC6FF00A00F5E76FF05C
:1007A0002700F2E706B010BDC89D040030B1037DFC
:1007B00023B183692BB13C301FF0BCBD6FF00A0040
:1007C00070476FF01C00704720B1037D13B190F9A2
:1007D000200070476FF00A00704738B50C4603469A
:1007E000F8B1057DEDB16FF00045A94219D08D0734
:1007F00017D0FEF7FDFC20B1B3F8C830136000201D
:1008000038BDA10705D519688D0702D5B3F8CA30E0
:10081000F4E7600702D519684907F7D46FF00500BF
:10082000EEE76FF00A00EBE72DE9F04F99466B4BCE
:100830009FB01B681D934FF0000343689DF8A070A4
:100840009C6820460D469046FFF770F94FF0000B6C
:100850000146824603AA2046CDF80CB0FFF7BDFF43
:10086000039B9F420ED900935D4A3B4602215846A6
:100870002AF0D2FD594B1A681D9B5A4000F0A980FE
:1008800036F050FC95F824603EB10D2EF2D1554A59
:10089000012158462AF0C0FDECE72B4604AA05A921
:1008A0002046FFF7D3F995F832301B0728D0049B78
:1008B000022B25D0382231460FA836F0C3FA05F1B5
:1008C0000C010FA820F055F8AB6A1993AB6811938F
:1008D0009DF86E308DF86C6066F303038DF86E3012
:1008E000D4F8BC0003680AAAD3F808B00FA93346AD
:1008F000D847034620B13C4A012130462AF08CFDFE
:10090000002102AA2846ADF808101FF0EFFF0021D1
:1009100010220BA836F096FA049B95F832100C932F
:10092000AB6AADF8343011F00F019DF808308DF846
:10093000393018BF01219DF80930CDF828A0B8F151
:10094000030FCDE906978DF82C808DF838108DF8BF
:100950003A3003D117B901238DF836300DF1370243
:100960000721284604F124061FF0C0FF0FCE0FAD6B
:100970000FC50A9A96E80300012A85E8030015D1FD
:1009800094F8E4306BB10023CDE90833D4F8C0000B
:1009900084F8E43083688DF824205B6908A9083066
:1009A0009847012211462046FEF72CFD9DF8143091
:1009B000049904EB830320461A6B0A431A630FA9B8
:1009C000FEF728FFA36806A99C681A680AA8A04732
:1009D00050E700201FB0BDE8F08F00BF2C9E040040
:1009E000CC9D0400F39D04000C9E040007B5009309
:1009F00013460222FFF718FF03B05DF804FB07B5AA
:100A0000009313460322FFF70FFF03B05DF804FBCA
:100A100007B5009313460122FFF706FF03B05DF808
:100A200004FB07B5009313460022FFF7FDFE03B059
:100A30005DF804FBF0B5754B91B00E4615461B688A
:100A40000F934FF00003044648B96FF00A006F4B54
:100A50001A680F9B5A4000F0D78036F063FB037D85
:100A6000002BF2D00029F0D00B68002BEDD04B68A2
:100A7000013BFE2BE9D8002AE7D0D0F8B80024F0DB
:100A8000BDF9B0F5967F40F2B680AB7B2BB1EA7B27
:100A9000002ADAD02A8A002AD7D02A79032A03D159
:100AA000AA89B2F5804FD0D213B9EB7378232B8289
:100AB00094F8243013B1032B40F0A080E26AD107F0
:100AC00005D42046FEF7A5FB002800F09780296892
:100AD000114200F093806FF0004399420ED0002342
:100AE0006A4620460093FFF778FE0028AFD172686F
:100AF000009B9A420CD96FF00900A8E7B4F8C830FF
:100B0000B4F8CA20934238BF134672689342F2D3B6
:100B1000AF68022F18BF012700213822AF6001A85B
:100B200036F090F9022F0CBF394904F1DC0101A81D
:100B30001FF01FFFE36ADB0723D529682046FEF775
:100B400057FBF0B1AA68236B1A421AD0D4F8C03010
:100B50000433039304F1A803AA7B02939DF8363073
:100B600062F303038DF83630EB7B8DF834302B8A3B
:100B7000ADF838302B79032B43D8DFE803F01C277E
:100B80002C31D4F8C420002A3BD02046FEF741FB8C
:100B9000002836D029682046FEF731FB002830D0E7
:100BA00094F8E83004EB8303196BAB68194228D042
:100BB00004320392CEE7D4F8BC0003681C68337992
:100BC000326801A9A0470B9BAB8140E7D4F8BC0079
:100BD00003685C68F3E7D4F8BC000368DC68EEE700
:100BE000AB89D4F8BC000B93036832689C683379F6
:100BF00001A9A0472BE76FF0030028E76FF027005B
:100C000025E76FF0050022E711B0F0BD309E04002B
:100C1000A89E040040B1037D33B183693BB1D0F895
:100C2000CC00012108F076BE6FF00A0070476FF02B
:100C30001C0070477FB5234B0E461B6803934FF093
:100C40000003054690B3836983B30368DA072DD5A3
:100C500090F82830012B2CD090F82930012B28D087
:100C6000C36ADB0700D539BB174A92E8030001AB22
:100C700083E80300D5F8C00050F8082F8EB1126940
:100C800019469047044670B10346104A01210020DE
:100C90002AF0C2FB0B4B1A68039B5A400FD036F068
:100CA00041FA5269ECE785F8E460F3E76FF00A0473
:100CB000F0E76FF02704EDE76FF01A04EAE720464B
:100CC00004B070BD549E0400747E0400349E040081
:100CD0000B46114638B182692AB121B133B91A469F
:100CE000012025F005BC6FF00A0070476FF0050089
:100CF0007047000000487047484D002008B528B9EB
:100D0000044B054A05486A21FAF770FB044B18604A
:100D100008BD00BF07D904005C9F0400B89E040012
:100D2000484D0020014B93F828007047484D0020A3
:100D300000207047014B002018717047484D00207B
:100D400008B500F03FFA002008BD000010B50446C9
:100D500000F090FC10B9034BDC6210BD6FF0050091
:100D6000FBE700BF484D0020033803289FBF044B1A
:100D700093F937300B70002088BF6FF00100704787
:100D8000484D002008B50F4A92F937309842A8BF65
:100D9000184613681B78012B0AD11428A8BF142009
:100DA00000F056FC00280CBF00206FF0050008BDC5
:100DB000023B012B03D80E28A8BF0E20F0E74FF00E
:100DC000FF30F4E7484D002008B500F0EFFA20B9F5
:100DD000034B022283F8282008BD6FF00500FBE7D3
:100DE000484D002008B500F0FBFA20B9034B012262
:100DF00083F8282008BD6FF00500FBE7484D002070
:100E000008B500F015FB20B9034B052283F8282014
:100E100008BD6FF00500FBE7484D002008B540B164
:100E200039B100F0D7FB00280CBF00206FF005009F
:100E300008BD6FF00100FBE708B500F0E1FB20B949
:100E4000034B042283F8282008BD6FF00500FBE760
:100E5000484D002008B5002100F064FB20B9044B88
:100E6000032283F8282008BD6FF00500FBE700BFD0
:100E7000484D002008B50121002000F053FB20B9A7
:100E8000034B032283F8282008BD6FF00500FBE721
:100E9000484D002007B500230DF10600ADF80630DF
:100EA00000F020FC20B9BDF9060003B05DF804FB9A
:100EB00047F6FF70F9E72DE9F0411E460123337034
:100EC0000F461546FFF742FF044690B9FFF7D2FFE1
:100ED000044670B9012D38BF0125804601202AF053
:100EE0007FFAFFF7D7FFB84208F1010804DD0023BD
:100EF00033702046BDE8F081A845EFD1F9E7000046
:100F0000014BB3F93A007047484D002001380528DD
:100F10009FBF044B93F938300B70002088BF6FF0EF
:100F200001007047484D0020002370B50B800D462E
:100F3000FFF70CFF0446B8B9FFF79CFF044698B9C9
:100F40002026FFF7A7FF2B8818442880013E0120A8
:100F50002AF046FA16F0FF06F3D1B5F90030002B5F
:100F6000B8BF1F335B112B80204670BD431E022B80
:100F7000F0B51CD80F4A11684F7900234FF0060CCA
:100F8000DCB2BC4202D34FF0FF300FE00CFB03F5A4
:100F90008E687419755D854203F10103F0D12368F1
:100FA000C2F83630044BA2889A800020F0BD6FF062
:100FB0000100FBE7484D00207E4D002030B5054B79
:100FC0001D680C3504460FCD0FC42B68236000202C
:100FD00030BD00BF484D002010B50D4C88B182B126
:100FE000C4E90220236821611879FFF7BFFF00F0F0
:100FF00099F948B9FFF7F6FE10B10023C4E90233AE
:1010000010BD6FF00100F8E76FF00500F5E700BFD5
:10101000484D002030B5164B00245C805C609C89F4
:1010200004F0700444F4C0749C81DC7DC8B10425D4
:1010300065F30304DC7580000129197C986121F0B7
:1010400003010CBF41F0020141F001011974197C48
:1010500021F0180141F0080119743AB913229A7568
:1010600030BD012565F30304DC75E5E71122F6E7E1
:10107000C41B0020124B0022C3E901221A7B02F09C
:10108000700262F07F021A730E4A9A6240F2FF7297
:101090001A83DA8922F4417222F0020242F4407289
:1010A000DA81DA7F30B1042161F30302DA7780005C
:1010B00018627047012161F30302DA77F8E700BF95
:1010C000101C00208C4D002010B50446FFF712FEC6
:1010D00028B1C3681BB12046BDE81040184710BDB9
:1010E00070B51D461646FFF705FE816804460022CE
:1010F0000C31104625F0FCF92369C4E9086513B1E9
:10110000BDE87040184770BD70B51D461646FFF724
:10111000F1FD8168044600220C31104625F0E8F903
:101120002369C4E9066513B1BDE87040184770BD76
:1011300010F0F70210B502D010280CD010BD144BDF
:101140001A70144B18680028F8D04FF0FF31BDE832
:10115000104034F0B1BB0E4C237859070AD523F068
:10116000040323700C4BB3F900100A4B00221868DB
:1011700034F0A2FB23789A07E0D523F00203237012
:10118000064BB3F90010034B00221868DFE700BFDD
:10119000884D0020944D00208A4D0020CC56002020
:1011A00002F0020003F0885150EA010306D0044A1D
:1011B000137823F0080343F010031370704700BF47
:1011C000884D002070B5FFF795FD0026044680F895
:1011D000346025F0D9F9A56900220023C4E906236B
:1011E00025F0EAF905F44002334613432DD020469A
:1011F00000F0C4FB064600F085FB26BB0220FFF78B
:1012000063FF05F00202002313433ED125F0BCF931
:10121000256A00220023C4E9082325F0CDF905F052
:101220000202002313430DD01B4B5B88B3F5505FC4
:101230000CBF01200820FFF747FF184A137823F05E
:101240000103137070BD0520D9E7154A33462A40C3
:101250001343F8D105F0020233461343D6D0114BA5
:101260005A8843F201439A4202D10720FFF72CFF2C
:101270000D4B5B8843F20942934203D043F207428D
:10128000934202D10720FFF71FFF044A137823F08F
:1012900002031370BAE700BF401C0020884D0020F5
:1012A00000000E8C101C0020C41B00202DE9F04310
:1012B00085B00023074689469046CDE90133ADF855
:1012C0000C3000F019FB437A027A7A70C3F30011F4
:1012D0001C02002904F4E0640CBF0421022144EA4A
:1012E0000204A4EB0104A4B20CBF0A260826FF2CBA
:1012F00028BFFF243B700546224600F10A014846FC
:1013000035F078FD291932460A3101A835F072FD11
:1013100004AB1E44204616F8123C88F8003005B095
:10132000BDE8F08330B500208BB0FFF701FF40F639
:101330000903009315491648012340F6140200F0F2
:10134000EBFA0446F8B9134D134834F0CDFA286887
:1013500010B134F0BDF92C600F4B104A1049114800
:1013600034F0CEFA286002A834F024F800220023DA
:10137000CDE900230C492868002302AA34F048FA7A
:1013800020460BB030BD0324FAE700BFB84E002062
:101390008C4D0020944D0020984E0020E01B002032
:1013A000601C0020984D00209C1B002038B50A4D81
:1013B0002B6873B1094C237813F0F70F09D008207C
:1013C000FFF7B6FE286834F035FA237843F00803B7
:1013D0002370002038BD00BF944D0020884D0020B0
:1013E00030B50F4D2C688BB0A4B10E4B1C7814F0A7
:1013F000F70412D102A833F0DDFF02220023CDE969
:1014000000230949094B286802AA33F0DFFF0028AE
:10141000B8BF032420460BB030BD0024FAE700BF5C
:10142000944D0020884D0020B41B0020A111010024
:10143000F0B50C468BB005461020FFF779FEB4F5E9
:10144000807F53D007D8012C16D0102C3DD064B12A
:1014500000200BB0F0BD40F201139C424DD0B4F51A
:10146000887FF5D10122002131E022460121284662
:10147000FFF7D0FD002613E0002221462846FFF7A3
:10148000C9FD0020FFF7F6FD1D4A1E4C1E4E00232D
:1014900053801E4B5A605A7B022161F303025A7338
:1014A00002A8002733F086FFCDE9006718481749E6
:1014B0000068234602AA33F089FF164B164A1880AB
:1014C000137843F020031370C2E701221146284627
:1014D000FFF7A0FD114A124C002353800B4B5A60BA
:1014E0005A7B032161F303025A73C3E700221146BA
:1014F0002846FFF78FFD0024BCE700221146BDE718
:10150000101C0020091101000000CE84C41B002023
:10151000944D0020CC560020884D0020401C002017
:10152000E1100100F0B58BB00E460446FFF7E2FB78
:1015300005461020FFF7FCFD95F834701D4D3FB3B4
:101540002046FFF797FD2C462EB1AB7B23F0060318
:1015500043F00603AB7302A833F02CFF164A17487A
:101560000023CDE90023214602AA154B006833F081
:101570002DFF0028134BA8BF134A1880A3BF137870
:10158000002043F002030320A8BF13700BB0F0BD8E
:101590003A46012120460D4CFFF73CFD0C48FFF771
:1015A00069FD627B6F80022161F3030265606273F3
:1015B000CAE700BF101C00200000CE84944D00201C
:1015C00009110100CC560020884D0020C41B0020CA
:1015D000400D030038B5084D0C460A460146284622
:1015E00035F008FC054B1A7B1C826FF30302DD61AA
:1015F0001A73002038BD00BFCE560020401C0020CA
:1016000000B510208BB0FFF793FD02A833F0D2FE97
:1016100000220023CDE9002309480A4B0A4900684B
:1016200002AA33F0D3FE0028A1BF084A1378002095
:1016300043F00103B4BF032013700BB05DF804FB4B
:10164000944D0020E1100100401C0020884D002036
:1016500010B5064B014606481C6834F019FC0146DB
:10166000204634F0CBFB002010BD00BF944D00207D
:10167000081D002030B58BB058B31749B0FBF1F509
:101680004FF47A7401FB1500B0FBF4F3C3EB034293
:1016900004FB1303B2FBF4F2C3EB03430F4CB3FBA5
:1016A000F1F31344013302A82382E58133F082FE73
:1016B00000220023CDE9002309480023006802AA84
:1016C000214633F083FE0028ACBF002003200BB07E
:1016D00030BD0220FBE700BF40420F009C1B0020F2
:1016E000944D002010B5044B0446186834F070FA8D
:1016F0002080002010BD00BF944D0020042910B5AB
:1017000019D842180023904210D10C4A93610C4A18
:1017100013610C4A937DC900C9B203F03F008842AF
:1017200002D061F305039375002005E010F8014B2A
:1017300044EA0323E7E7032010BD00BF401C00205C
:10174000101C0020E01B002010B50446FFF7D2FA61
:1017500023683E4A934231D03D4A934252D04CF2E4
:101760005032934270D13B4A136923F0604323F017
:10177000FF03B3F5000F13460AD1D18921F0070109
:101780008904890CB1F5487F02D1127D552A13D006
:101790001A694FF4004161F31C221A61DA8964214D
:1017A00061F3CD02DA8155221A752B4ADA6122687B
:1017B0002A4BB3FBF2F30363002046E0254A13698A
:1017C00023F0604323F0FF03B3F1C07F13460AD137
:1017D000D18921F007018904890CB1F5E46F02D1A8
:1017E000127D592AE8D01A694FF4C03161F31C22E6
:1017F0001A61DA89E42161F3CD02DA8159221A757E
:10180000174AD3E7134A136923F0604323F0FF0319
:10181000B3F1207F13460AD1D18921F00701890451
:10182000890CB1F5FA6F02D1127D5C2AC4D01A6915
:101830004FF4203161F31C221A61DA89FA2161F335
:10184000CD02DA815C22DAE7022010BDF049020005
:1018500090D00300E01B0020B81C002040420F0085
:10186000981C002038B50446FFF744FA0E4AE17888
:10187000937D03F03F058D421CBF61F30503937513
:101880002288036B5343094AD17C04259B0065F3EE
:101890000301D17453612388202B9CBF012380F85E
:1018A0003430002038BD00BFE01B0020401C002069
:1018B0000388C2780179103313448279002918BF54
:1018C0000132C179012908D011F0FB0F14BF0220A9
:1018D0000120104403EBC00070470020F9E710B569
:1018E0000C46FFF7E5FF23684FF47A715A1E01FB9F
:1018F0000020B0FBF3F010BD014B1868704700BF2B
:10190000F0380120034A1368002119711B68136025
:1019100018797047F03801202DE9F041BDF81860C2
:1019200006F0030406F10807C4F1040404EB0708F9
:1019300008FB03F5AA421DDB00250A468E46AC468D
:1019400057FA84F4AB4208DC0B4BCEF80010C0E928
:10195000001C19600020BDE8F081577982F804C0AE
:1019600027F00F075771A7189646D68017600135E4
:101970004244E7E70120EEE7F038012013B5846820
:1019800000230DF1030204F1140101A8ADF80430A5
:101990008DF80330FFF78AFCC0B284F81301A8B1B8
:1019A0000C499DF9032091F900306BB1134403EB0E
:1019B000D37343F347030B7002F15A012172A272F1
:1019C0006372002002B010BD1346F4E76FF0070009
:1019D000F8E700BFCD5E002003684CF2503293421E
:1019E0000AD1426846F2A8139A4221D1437A1A2BAF
:1019F00014BF0020032070470E4A93420AD1426868
:101A000049F27C239A4213D1437A192B14BF002048
:101A100004207047084A93420AD142684FF2244397
:101A20009A4205D1437A092B14BF00200520704744
:101A300000207047F049020090D0030000B3042951
:101A40000ED0052914D003291AD146F2A8134CF25E
:101A5000503CC0E900C341F60B23038100207047CE
:101A6000094949F27C23C0E9001341F60913F4E760
:101A7000064A4FF22443C0E9002340F60913ECE77D
:101A80006FF00100704700BFF049020090D00300E2
:101A9000C8B10168B9B14368ABB1C2689AB1552009
:101AA00010708978002914BF6F21902151704E2148
:101AB000917040F205325A80FF2200209A71012273
:101AC00098809A8170476FF00100704770B50028C8
:101AD00044D00468002C41D04368002B3ED0C2683B
:101AE000002A3BD00069002838D09979002935D0E8
:101AF0001D88002D32D0257865BBFB292ED85525B1
:101B00001570A578002D14BF6F25902555704E25B2
:101B100095704FF441725A808D1C00229A80EDB26C
:101B200001229D719A8122781201D2B242706678A8
:101B3000002E14BF082600263244427022780AB9CB
:101B40000431CDB200F8025B9A79996835F052F908
:101B5000002070BD012DD2D1FD29CFE76FF001002B
:101B6000F7E708B5FFF7CAFD002814BF6FF00500BE
:101B7000002008BD002070471FB588B1D0E90023C0
:101B8000CDE901230389ADF80C3001A8FFF7DCFD96
:101B900000280CBF00206FF0050005B05DF804FBC5
:101BA0006FF00100F9E71FB538B303888288ADF8FC
:101BB0000820012B83BF03F1FF33DB009BB200231E
:101BC000ADF8043083788DF80630C378DB008DF8EB
:101BD000073083798DF80A30037B8DF80B30437B17
:101BE0008DF80C3001A8FFF73DFE00280CBF002047
:101BF0006FF0050005B05DF804FB6FF00100F9E738
:101C00007FB540B351B3D0E90023CDE90323038965
